:100000000C94A0060C94BB060C94BB060C94BB0687
:100010000C94BB060C94BB060C94BB060C94BB065C
:100020000C94BB060C9470170C94BB060C94BB0686
:100030000C94682C0C94BB060C94BB060C94BB0669
:100040000C94BB060C94BB060C9405160C94BB06D2
:100050000C947D0D0C94BB060C94470D0C94BB06C0
:100060000C946A1C0C94BB060C94232B0C94BB06BA
:100070000C9419680C94BB060C943366951C9A1C5E
:100080009F1CA81CBF1CD61CE61CF61C131D6D1F54
:10009000D61C2F1E401E6F1E8D1EAA1E041F5F1F22
:1000A0003D21B6217222E9225223F523002667263C
:1000B000E1262B277627C32710286A28D7287129FD
:1000C0006B2A462B782B872BB22BE42BF42B342C6A
:1000D000342C212C0C2C0E2C282C162C212C112CE1
:1000E000132C282C162C212C232C252C282C2C2CA2
:1000F0000A0D426174743A0020332043656C6C73BE
:1001000020200020342043656C6C73202000204C9C
:100110006F77207761726E696E67206C6576656CAB
:100120003A2025642E2564000A0D47656E657261CC
:1001300074696E672064656661756C74204D6978BA
:100140006572205461626C65000A0D4D69786572B4
:100150002D436F6E6669673A20272573272028256F
:1001600075204D6F746F727329000A0D466F756E9E
:100170006420424C2D4374726C3A200025642000A8
:100180000A0D0A0D2121204D495353494E47204263
:100190004C2D4354524C3A202564202121000A0D55
:1001A0003D3D3D3D3D3D3D3D3D3D3D3D3D3D3D3D7F
:1001B0003D3D3D3D3D3D3D3D3D3D3D3D3D3D3D3D6F
:1001C0003D3D3D000A0D496E69742E204545505253
:1001D0004F4D003A2047656E65726174696E672005
:1001E00044656661756C742D506172616D657465EE
:1001F00072207573696E67206F6C64205374696335
:100200006B2053657474696E6773000A0D466C69E0
:100210006768742D74696D65202575206D696E2081
:1002200020546F74616C3A2575206D696E000A0D5B
:10023000414343206E6F742063616C696272617424
:1002400065642021000A0D5573696E672070617224
:10025000616D65746572736574202564000A0D43D1
:10026000616C6962726174696E6720707265737324
:100270007572652073656E736F722E2E004F4B0A78
:100280000D000A0D436F6E74726F6C3A2000486562
:100290006164696E67486F6C64004E6F726D616C6B
:1002A00020284143432D4D6F646529000A0D3D3DD3
:1002B0003D3D3D3D3D3D3D3D3D3D3D3D3D3D3D3D6E
:1002C0003D3D3D3D3D3D3D3D3D3D3D3D3D3D3D3D5E
:1002D0003D0A0D00416E676C654E69636B202020FE
:1002E00020202020416E676C65526F6C6C202020AE
:1002F000202020204163634E69636B202020202052
:1003000020202020416363526F6C6C20202020202D
:10031000202020205961774779726F2020202020EB
:10032000202020204865696768742056616C7565D7
:10033000202020204163635A2020202020202020DC
:1003400020202020476173202020202020202020F2
:1003500020202020436F6D706173732056616C758F
:1003600065202020566F6C74616765205B302E31EC
:10037000565D20205265636569766572204C65760E
:10038000656C20204779726F20436F6D70617373C5
:10039000202020204D6F746F7220312020202020DB
:1003A000202020204D6F746F7220322020202020CA
:1003B000202020204D6F746F7220332020202020B9
:1003C000202020204D6F746F7220342020202020A8
:1003D000202020202020202020202020202020201D
:1003E000202020202020202020202020202020200D
:1003F00020202020566172696F4D6574657220203F
:10040000202020204D4B334D61672043616C537495
:1004100061746520536572766F2020202020202093
:1004200020202020486F766572676173202020208D
:100430002020202043757272656E74205B302E314F
:10044000415D20204361706163697479205B6D4177
:10045000685D202020202020202020202020202017
:10046000202020202020202020202020202020208C
:10047000202020202020202020202020202020207C
:10048000202020202020202020202020202020206C
:10049000202020204932432D4572726F7220202087
:1004A000202020202020202020202020202020204C
:1004B000202020204750535F4E69636B202020206E
:1004C000202020204750535F526F6C6C202020204A
:1004D0002020202021212120494E434F4D504154BE
:1004E00049424C4520212121002E000A0D20444183
:1004F00043206F7220493243204552524F522120EF
:10050000436865636B204932432C2033567265661D
:100510002C2044414320616E6420424C2D43747270
:100520006C005B25695D005B25695D002B204D69D2
:100530006B726F4B6F70746572202B0048573A5680
:1005400025642E25642053573A25642E256425639F
:100550000053657474696E673A25642025730049F9
:100560003243204552524F52212121004D6973736D
:10057000696E6720424C2D4374726C3A25642121C8
:10058000004865696768743A20202535690053651D
:1005900074706F696E743A253569005072657373B3
:1005A0007572653A253569004F66667365743A2041
:1005B000202535690048656967687420636F6E742B
:1005C000726F6C0044495341424C45440048656990
:1005D00067687420636F6E74726F6C004449534196
:1005E000424C4544006163742E2062656172696EFD
:1005F00067004E69636B3A20202020202025356952
:1006000000526F6C6C3A2020202020202535690094
:10061000436F6D706173733A202020253569004B5C
:10062000313A25346920204B323A25346920004B79
:10063000333A25346920204B343A25346920004B65
:10064000353A25346920204B363A25346920004B51
:10065000373A25346920204B383A25346920004E3A
:10066000693A2534692020526F3A253469200047C1
:10067000733A253469202047693A253469200050AF
:10068000313A253469202050323A2534692000500F
:10069000333A253469202050343A25346920004704
:1006A00079726F202D2053656E736F72004E6963EF
:1006B0006B25346920282533692E25692900526F5E
:1006C0006C6C25346920282533692E25692900475B
:1006D000696572253469202825336929004E6963CC
:1006E0006B2025346920282533692E25782900526E
:1006F0006F6C6C2025346920282533692E257829D4
:100700000059617720202534692028253369290084
:100710004E69636B202534692028253369292825F3
:1007200033692900526F6C6C2025346920282533E9
:1007300069292825336929005961772020253469E2
:10074000202825336929282533692900414343207E
:100750002D2053656E736F72004E69636B202534D4
:100760006920282533692900526F6C6C2025346973
:10077000202825336929005A20202020253469208B
:10078000282533692900566F6C746167653A20200B
:10079000202533692E253169560043757272656EC6
:1007A000743A2020202533692E2531694100506F8D
:1007B0007765723A2020202020253469570044694B
:1007C000736368617267653A202535696D41680019
:1007D00052656365697665720052432D52535349E1
:1007E0003A202020202534690052432D5175616C38
:1007F0006974793A202534690052432D4368616E4B
:100800006E656C733A25346900436F6D7061737364
:100810000048656164696E673A2020253569005695
:10082000616C75653A20202020253569005374617C
:1008300072743A2020202025356900506F74693188
:100840003A202025336900506F7469323A20202500
:10085000336900506F7469333A20202533690050A2
:100860006F7469343A202025336900506F746935FC
:100870003A202025336900506F7469363A202025CC
:10088000336900506F7469373A202025336900506E
:100890006F7469383A202025336900536572766F8A
:1008A000202000536574706F696E742020253369B1
:1008B00000506F736974696F6E3A20253369005276
:1008C000616E67653A2533692D2533690045787473
:1008D00065726E436F6E74726F6C2020004E693AC1
:1008E0002534692020526F3A253469200047733A35
:1008F000253469202047693A253469200048693A3F
:10090000253469202043663A2534692000424C2D65
:100910004374726C204572726F72732000253364C9
:1009200020253364202533642025336420002533BB
:10093000642025336420253364202533642000257A
:10094000336420253364202533642025336420005C
:10095000424C2D4374726C20666F756E64200020CB
:1009600025632020202563202020256320202025AA
:10097000632000202563202020256320202025637C
:10098000202020256320002025632020202D2020EA
:10099000202D2020202D2000313000313100313237
:1009A00000466C696768742D54696D652020005499
:1009B0006F74616C3A2535756D696E004163743AE8
:1009C00020202535756D696E002872657365742960
:1009D000000A0D506C6561736520636F6E6E656310
:1009E00074205370656B7472756D207265636569F0
:1009F00076657220666F722062696E64696E672028
:100A00004E4F572E2E2E006F6B2E0A0D0054696D1F
:100A1000656F75742E0A0D0000008F001E01AD0178
:100A20003B02CA025803E603740402058F051B0645
:100A3000A7063307BE074808D2085B09E3096B0A1B
:100A4000F20A780BFD0B810C040D860D070E870E44
:100A5000060F840F00107B10F5106E11E5115B126C
:100A6000CF124213B31323149214FE146A15D31534
:100A70003B16A11605176717C81727188318DE1825
:100A800037198E19E319361A871AD61A231B6E1BCB
:100A9000B61BFD1B411C831CC31C001D3C1D751D8A
:100AA000AB1DE01D121E421E6F1E9A1EC31EE91EC4
:100AB0000D1F2E1F4D1F691F841F9B1FB01FC31FBB
:100AC000D31FE11FEC1FF51FFB1FFF1F00200301B9
:100AD00000000A6200020101CA62010302023963D6
:100AE0000200030396632532692E253169560025DD
:100AF0003033646D20253033642563005374617492
:100B000075730025346920202532693A2530326911
:100B1000002534696D004E69636B20526F6C6C2048
:100B200020596177002534692025346920253469EE
:100B3000002532692E2531695620202533692E255E
:100B40003169410025346957202536696D416800B7
:100B50005361743A25303264004E6F466978003232
:100B600044466978003344466978003F3F466978D7
:100B7000002F4447505300486F6D653A2530336469
:100B80006D20253033642563004E6F204E617669F9
:100B90004374726C21000A0D7777772E4D696B7262
:100BA0006F4B6F707465722E64652028632920482E
:100BB0006953797374656D7320476D6248000A0D3F
:100BC00074686520757365206F662074686973208A
:100BD000736F667477617265206973206F6E6C79CC
:100BE000207065726D6974746564200A0D6F6E20E3
:100BF0006F726967696E616C204D696B726F4B6FC4
:100C0000707465722D48617264776172650041434A
:100C1000542044534C004A65746920736174656CB8
:100C20006C6974005370656B7472756D20736174B8
:100C3000656C6C697420284C6F77207265736F6CDB
:100C40007574696F6E29005370656B7472756D20D1
:100C5000736174656C6C69742028323034382900F3
:100C60005370656B7472756D20736174656C6C691B
:100C700074004D756C74697369676E616C205050B7
:100C80004D000A0D52656365697665723A200075FC
:100C90006E6B6E6F776E2E205573696E67205050A5
:100CA0004D2E2E2E006E6F7420737570706F7274DF
:100CB00065642062792068617264776172652100E1
:100CC0000A0D3D3D3D3D3D3D3D3D3D3D3D3D3D3DB7
:100CD0003D3D3D3D3D3D3D3D3D3D3D3D3D3D3D3D44
:100CE0003D3D3D3D3D000A0D466C69676874436FAC
:100CF0006E74726F6C0A0D48617264776172653A46
:100D000025642E25640A0D536F6674776172653A07
:100D10005625642E2564256320000A0D3D3D3D3D8A
:100D20003D3D3D3D3D3D3D3D3D3D3D3D3D3D3D3DF3
:100D30003D3D3D3D3D3D3D3D3D3D3D3D3D3D3D0020
:100D400011241FBECFEFD0E1DEBFCDBF11E0A0E088
:100D5000B1E0ECE4FEED02C005900D92A03DB107BC
:100D6000D9F717E0A0EDB1E001C01D92A63CB10794
:100D7000E1F70C94E7070C940000282FFB01815049
:100D8000853008F023E0842F992733272150304005
:100D9000829FD001839FB00D929FB00D1124AC595A
:100DA000BF4F019724F00E94086F0192FACF0E9472
:100DB000545E0895863010F085E002C0882329F043
:100DC000A2E0B0E0082E0E94156F0895582F8630DB
:100DD00010F055E002C0882339F1842F9927252F80
:100DE000332721503040829FD001839FB00D929FC6
:100DF000B00D1124AC59BF4FFB01019724F00190B5
:100E00000E94156FFACFA2E6B0E0042E0E94156F83
:100E1000A0E5B0E08CE0FB01182E0E94216F852F29
:100E20000E94DA060E94545E0895CF93A2E0B0E0DB
:100E30000E94086F802DC82F8150853020F0C3E0BC
:100E40008C2F0E94DA068C2F9927CF9108958091DC
:100E50005606E82FFF27EE0FFF1FE951FA4F80815A
:100E600091818D5E9F4F14F01092030180819181DA
:100E70008A5B9F4FCCF4809103018823A9F481E021
:100E800080930301809113048F5F80931304853056
:100E900038F088EE93E09093FF018093FE0104C048
:100EA00066E970E00E94EF2F8091130499279093D8
:100EB0008D0580938C0508951F93CF93DF93182F92
:100EC000882389F080EF90E09F938F9387E293E1EE
:100ED0009F938F93E0919203F091930309950F9064
:100EE0000F900F900F9080917806823308F046C0E3
:100EF00084EF91E00E94F016EC01112329F0CE015D
:100F00000E94F9168823D9F380912501909126013A
:100F1000209178068238910584F433E0239FC00144
:100F2000112480930001112359F168EC70E0832FA4
:100F30000E94EF2F88EF90E011C0822F9927880F31
:100F4000991F880F991F809300011123C9F068EC45
:100F500070E084E00E94EF2F83E091E09F938F93F5
:100F600087E293E19F938F93E0919203F091930333
:100F700009950F900F900F900F9002C08093000181
:100F8000112309F1809100016AE00E945B6E892FB4
:100F900099279F938F93809100010E945B6E992700
:100FA0009F938F938EE091E09F938F9387E293E1DD
:100FB0009F938F93E0919203F091930309958DB7DE
:100FC0009EB708968DBFDF91CF911F910895CFEF07
:100FD000D0E1DEBFCDBF6624772410E014B915B987
:100FE00087EEC82E83E0D82E8EEC9FEFC80ED91E58
:100FF000D7FEFACF189B06C0199B02C08DE007C030
:101000008BE005C0199B02C084E101C08AE0809397
:10101000020181E887B93E9A8FEF88B98BE184B9E4
:1010200081E085B98EE38AB987E48BB9469A84B7A3
:10103000877F84BF809160008861809360001092F8
:10104000600080ED97E09093FF018093FE01109285
:101050007D0210927C021092EC051092EB0510922A
:101060007F0210927E0210928102109280022091E3
:101070000201243128F088E894E0A0E0B0E004C048
:101080008BE095E0A0E0B0E08093790190937A0145
:10109000A0937B01B0937C012A3011F0243111F42C
:1010A000289801C0289A0E9459170E942A170E9466
:1010B0002F130E944C2C0E94381B0E94E22A0E948F
:1010C0005F5A0E9496640E945667809102018C309C
:1010D00010F4299A01C0299878944DE066E576E0ED
:1010E00083E00E94BD06C8EED3E0DE010E94086FD7
:1010F000802D8130D9F4DE01A75EB3400E94086FD5
:10110000802D8F3F99F0E4E9F3E08DE4DE01182EA5
:101110000E94106FE1EAF3E09FE080813496181698
:101120000CF41F5F915097FFF8CF51C088E291E017
:101130009F938F9387E293E19F938F93E091920324
:10114000F091930309950F900F900F900F9024E961
:1011500033E0F9018FE0158616861786108A8150D4
:10116000349687FFF8CF80E48093A1038093A20395
:101170001092A3038093A4038093A50390EC909313
:10118000A6031092A7038093A8038093A90310924B
:10119000AA039093AB039093AC038093AD0310929A
:1011A000AE038093AF039093B00381E080939403E8
:1011B0008BE0A4E0B1E0E5E9F3E00D9001928A95BF
:1011C000E1F78DE4DE01F901182E0E94216F812FD5
:1011D00099279F938F9385E993E09F938F9389E459
:1011E00091E09F938F9307E2A02E03E1B02EBF9270
:1011F000AF92E0919203F091930309958DB79EB75A
:1012000008968DBF8AE691E09F938F93BF92AF922D
:10121000E0919203F0919303099510924802109285
:1012200002020E94AA3B0F900F900F900F908091A6
:1012300002028823E1F31092480280ED97E00E94B9
:10124000F0166C01C0E0D0E017EBE12E15E0F12EB6
:101250008E01109202020E94AA3B80910202882312
:10126000E1F3F801EC56FC4F85851816ACF408C084
:10127000909302020E94AA3B809102028823E1F32C
:10128000C6010E94F916982F882331F4F801EA5418
:10129000FA4F8181882364F7F701808187FF13C0AB
:1012A0002196DF93CF9321978CE791E09F938F93C3
:1012B000BF92AF92E0919203F091930309958DB79D
:1012C0009EB706968DBF21960C5F1F4FE4E0F0E0BD
:1012D000EE0EFF1ECC30D10508F4BBCFC0E0D0E04D
:1012E00006EB15E0B1EAEB2EB3E0FB2EF8018181AD
:1012F00087FD1CC0F70180811816C4F42196DF9386
:10130000CF93219780E891E09F938F9387E293E1B9
:101310009F938F93E0919203F0919303099581E05D
:101320008093FC018DB79EB706968DBFF801818131
:1013300080788183219684E090E0E80EF91E080F02
:10134000191FCC30D10590F28EE991E09F938F93D5
:10135000A7E2EA2EA3E1FA2EFF92EF92E091920328
:10136000F091930309950E94AA3B0F900F900F9064
:101370000F9001E010E0D8010E94086F802D8235A7
:1013800009F4DAC00E94652D84EC91E09F938F935D
:10139000FF92EF92E0919203F09193030995C1E0DF
:1013A0000F900F900F900F90C23039F0C33019F4A6
:1013B0000E940B2F04C0C43010F00E94392E80917F
:1013C0000201843168F085E08093750610929606DC
:1013D0008BE1809371068EE480939306809394064C
:1013E000A0E5B0E0AD010E94086F802D8C3008F0C0
:1013F0008FC0DA011196FD010E94086F802D8C309C
:1014000008F086C0DA011296BD010E94086F802D97
:101410008C3008F07DC0DA0113969D010E94086FA0
:10142000802D8C3008F074C0DA010E94086F802D86
:1014300080935606DF010E94086F802D8093570627
:10144000DB010E94086F802D80935806D9010E940D
:10145000086F802D80935906DA0114960E94086F58
:10146000802D80935A06DA0115960E94086F802D10
:1014700080935B06DA0116960E94086F802D809398
:101480005C06DA0117960E94086F802D80935D0636
:10149000DA0118969D010E94086F802D8F3FD1F0D0
:1014A000D9010E94086F802D80935E06DA0119969B
:1014B0000E94086F802D80935F06DA011A960E94C1
:1014C000086F802D80936006DA011B960E94086FDA
:1014D000802D0AC089E080935E068AE080935F06D3
:1014E0008BE0809360068CE080936106C13091F4BC
:1014F00083ED91E09F938F93FF92EF92E09192039F
:10150000F091930309950F900F900F900F9002C0E8
:101510000E94402D4CE666E576E08C2F0E94E606A0
:10152000CF5FC63008F440CF83E00E94DA0682E540
:10153000D801082E0E94156F0EE010E0D8010E941D
:10154000086F802D9927582F442748010894811C43
:10155000911CD4010E94086F802D480F511D50939B
:10156000D5014093D401ECEFAE2EEFEFBE2EA00ECE
:10157000B11ED5010E94086F802D9927982F8827CA
:101580006DEFE62E6FEFF62EE00EF11ED7010E94F2
:10159000086F202D820F911D9093D3018093D2016B
:1015A0008F5F9F4F19F04F5F5F4F41F41092D5014D
:1015B0001092D4011092D3011092D2018091D201E5
:1015C0009091D3019F938F938091D4019091D501F5
:1015D0009F938F938BE092E09F938F93C7E2D3E129
:1015E000DF93CF93E0919203F091930309958DB728
:1015F0009EB708968DBFA4E0B0E00E94086F802DD2
:10160000853078F08EE292E09F938F93DF93CF93B3
:10161000E0919203F091930309950F900F900F9032
:101620000F900E9415074CE666E576E00E94BD0625
:101630000E94150799279F938F9385E492E09F93CB
:101640008F93DF93CF93E0919203F09193030995E9
:10165000EDB7FEB73696EDBF8DE592E09F938F9381
:10166000DF93CF93E0919203F0919303099588EE75
:1016700093E00E94F0166C010E943E1B0F900F90A9
:101680000F900F90C6010E94F9168823D9F38DE7B9
:1016900092E09F938F93DF93CF93E0919203F09129
:1016A000930309950E945B39809102010F900F907E
:1016B0000F900F908A3011F0843111F4289801C0F6
:1016C000289A80ED97E09093FF018093FE0185E5D5
:1016D0008093150482E892E09F938F93DF93CF93DA
:1016E000E0919203F09193030995809162060F9027
:1016F0000F900F900F90E0919203F091930382FF6F
:1017000007C08EE892E09F938F93DF93CF9308C03A
:101710008AE992E09F938F9387E293E19F938F935F
:1017200009950F900F900F900F900E94B42088E8B9
:1017300093E19093A00180939F0181E08093140432
:101740000E945C070E94AD668CEA92E09F938F93A3
:10175000DF93CF93E0919203F0919303099580ED8D
:1017600097E00E94F0166C018AEF90E00E94F0165C
:10177000EC010F900F900F900F90CE010E94F91680
:10178000882339F084E690E00E94F016EC010E9474
:10179000086880910202882309F471C180911701C1
:1017A000882309F46CC110920202809113048823EB
:1017B00019F00E94270702C00E94FB3D0E94AA3B2D
:1017C000209102012A3011F0243111F4289801C02F
:1017D000289A80918302882331F08091830281507E
:1017E0008093830205C080916F00806280936F00B8
:1017F00080919F019091A00101979093A001809307
:101800009F0180919F019091A001892B21F08091EF
:1018100047028823A1F180919F019091A001892B1B
:10182000B1F40E94F82A85E090E09093A0018093A3
:101830009F0180919E0590919F05019690939F0531
:1018400080939E058091520280688093520280911D
:101850001001909111018F5F9F4F19F580917902CE
:101860008823F9F080E197E29093FF018093FE01D5
:1018700080E890E0909311018093100112C02A300B
:1018800011F0243111F4289801C0289A8091FE01AA
:101890009091FF01892B29F4809152028F778093D8
:1018A000520280910202882321F0809179028823DC
:1018B00011F40E946A130E94BB0FC6010E94F91620
:1018C000882309F4D8C084E190E0C80ED91E809125
:1018D0000D01882321F0815080930D0125C0809354
:1018E0001F0410925E0210925D0210925C02109230
:1018F0005B0210925A02109259028091100190914D
:1019000011018F5F9F4F81F480918302882361F4DE
:1019100088E99AE39093FF018093FE0180E09CE0C8
:10192000909311018093100180916803882339F00E
:10193000815080936803809152028F7B11C0109276
:101940006603109265031092640310926303809102
:10195000FE019091FF01892B29F48091520280644D
:101960008093520280910001282F33278091250116
:101970009091260182179307CCF4809152028062E5
:101980008093520280911001909111018F5F9F4FBF
:10199000C1F480E797E19093FF018093FE0180E01E
:1019A00093E090931101809310010BC08091FE0190
:1019B0009091FF01892B29F4809152028F7D8093B1
:1019C00052020E94885D84E08093FD01809179023B
:1019D000882329F45AEA652E55E0752E12C08091AD
:1019E000D6018F5F8093D601813359F41092D601CE
:1019F0008091D0019091D10101969093D101809373
:101A0000D0010894611C711C22E762162BE072065B
:101A100091F5662477242091D4013091D5012F5F70
:101A20003F4F3093D5012093D4018091D201909102
:101A3000D30101969093D3018093D201832F9927EC
:101A4000D801082E0E94156F8091D401D401082E70
:101A50000E94156F8091D301D501082E0E94156F49
:101A60008091D201D701082E0E94156F84E190E089
:101A70000E94F0166C010E94635E0E94AB6480912C
:101A8000FD01882309F079CE0E94C95D76CE1F92B0
:101A90000F920FB60F9211248F939F93EF93FF93A2
:101AA00080910F018823E1F48091F0019091F10180
:101AB00001969093F1018093F001FC01EC53FB4FF0
:101AC000E081ED3019F0803A910539F41092F1017E
:101AD0001092F00181E080930F01E093C60004C0F2
:101AE0001092F1011092F001FF91EF919F918F916F
:101AF0000F900FBE0F901F9018951F920F920FB668
:101B00000F9211242F933F934F935F936F937F9383
:101B10008F939F93AF93BF93CF93EF93FF9390E0F7
:101B20008091C6008093E8015091F601503A10F080
:101B30009093F7018091E8018D3009F065C08091A4
:101B4000F701823009F060C09093F701852F992743
:101B50008E5D9B4FFC01329740812091F2013091C4
:101B6000F301241B3109DC0111978C91281B3109E9
:101B7000C9019F709093F3018093F20146E096951E
:101B800087954A95E1F7982F935C9093F4012F7312
:101B90003070235C2093F5018081981729F48C9193
:101BA000281711F491E006C090E08091E5018F5F65
:101BB0008093E501C091E701CC2309F074C099231B
:101BC00009F471C081E08093E701580F5093E4015C
:101BD0005150E52FFF27EE5DFB4F8DE08083809114
:101BE0002404823509F05FC00E94B42088E190E0AF
:101BF0002CE00FB6F894A895809360000FBE209358
:101C00006000C093FC014FC02091F701822F9927FB
:101C100081309105F9F0823091051CF4892B21F077
:101C200040C0029711F13DC08091E801833239F440
:101C30008091E701882319F481E08093F701809176
:101C4000E8018093220481E08093F6018091E8010D
:101C5000992722C02F5F2093F701E52FFF27EE5D24
:101C6000FB4F8091E801808309C0E52FFF27EE5DDF
:101C7000FB4F8091E8018083503A20F45F5F5093DE
:101C8000F60102C01092F7012091E8018091F20163
:101C90009091F301820F911D9093F3018093F201D3
:101CA00002C01092F701FF91EF91CF91BF91AF91D8
:101CB0009F918F917F916F915F914F913F912F9164
:101CC0000F900FBE0F901F901895AC01A0E0B0E0F0
:101CD0009D01A817B90748F4E4ECF4E08191280FBE
:101CE000311D1196A417B507C8F33F70FD01EC53E1
:101CF000FB4FC90156E0969587955A95E1F7835CAD
:101D000080831196FD01EC53FB4F2F733070822FAF
:101D1000835C8083AB53BB4F8DE08C9310920F019B
:101D20008091C4048093C6000895A0E0B0E0EBE980
:101D3000FEE00C94D46E2C859D850E85BB2483E239
:101D40008093C4049F599093C5042093C60433E044
:101D5000E32EF12C002309F49EC0CF84D888BE0165
:101D60006D5E7F4FA989BA890150109709F493C01D
:101D70001097B9F0F601EB0DF11DB3949081119716
:101D800091F4002349F1FB016E5F7F4FDB01C080BE
:101D9000D1806E5F7F4F0D90BC91A02DBB24015070
:101DA00002C090E019C01097B9F0F601EB0DF11DDB
:101DB000B3944081119791F4002341F1FB016E5FD0
:101DC0007F4FDB01C080D1806E5F7F4F0D90BC9153
:101DD000A02DBB24015002C040E018C01097B1F004
:101DE000F601EB0DF11DB3941081119781F40023DE
:101DF00071F0FB013296DB01CD90DC90BF016E5F8C
:101E00007F4FA081B181BB24015001C010E0F701D8
:101E1000EC53FB4F892F86958695835C80830894CD
:101E2000E11CF11CF701EC53FB4F892F99278370BC
:101E3000907024E0880F991F2A95E1F755279A01A1
:101E400094E0369527959A95E1F7822B835C808301
:101E50000894E11CF11CF701EC53FB4F4F705070DC
:101E6000440F551F440F551F812F992726E0969543
:101E700087952A95E1F7842B835C80830894E11C85
:101E8000F11CF701EC53FB4F1F73135C1083089494
:101E9000E11CF11C6ACFC7010E94650EE9E00C94B9
:101EA000F06EA3E07A2F4091E4014650442309F4F8
:101EB00058C0E72FFF27EE5DFB4F80818D537F5F7A
:101EC000E72FFF27EE5DFB4F20812D537F5FE72F2C
:101ED000FF27EE5DFB4F30813D537F5FE72FFF27EC
:101EE000EE5DFB4F60816D537F5F9927880F991FCF
:101EF000880F991F522F52955F70582B822F992768
:101F00008F709070F4E0880F991FFA95E1F7232FF6
:101F100026952695282B832F992783709070E6E0CD
:101F2000880F991FEA95E1F7682B41504F3FC9F0A0
:101F3000EA2FFF27EE5DFB4F5083AF5F41504F3FCD
:101F400081F0EA2FFF27EE5DFB4F2083AF5F41500A
:101F50004F3F39F0EA2FFF27EE5DFB4F6083AF5F05
:101F6000A5CF85E294E09093E3018093E201A35032
:101F7000A093E1010895A2E0B0E0E1ECFFE00C9451
:101F8000DB6E8091E701882309F45DC30E94510F45
:101F900080912304823609F01FC28091240499277E
:101FA0008037910509F4ACC081379105A4F48636D9
:101FB000910509F470C18736910524F48B3491059D
:101FC000F1F00AC28D36910509F468C08E3691058C
:101FD00009F453C001C28337910509F4EDC0843779
:101FE00091052CF48137910509F491C0F5C184372E
:101FF000910511F18937910509F48AC1EDC1E0918C
:10200000E201F091E30180819181909396028093A7
:1020100095022091930230919402821B930B845E6F
:102020009D4F68E671E00E947B6E845B90409093C8
:10203000920280939102D0C18091E401A091E201CB
:10204000B091E301853140F080E1EDEFF3E00D90D8
:1020500001928A95E1F70DC08D919D910D90BC91F3
:10206000A02D8093FD039093FE03A093FF03B093F4
:10207000000480EF8093DF0146C080910F01882328
:10208000E1F38DE490E09F938F9384E993E09F9335
:102090008F9381E08F938F938EE42AC080910F01FC
:1020A0008823E1F34091E2015091E301DA019C9130
:1020B000913089F464E973E08DE4FB01282F0D90E1
:1020C00001922A95E1F7A8EEB3E0FB01182E0E94D9
:1020D000216F998301C0198281E090E09F938F93D3
:1020E000CE0101969F938F9381E08F938F938DE420
:1020F0008F930E94950E8DB79EB707968DBF6CC1CA
:1021000081E08093EA018FEF80930D0165C1E0913A
:10211000E201F091E30180818F3F39F40E941507BD
:10212000E091E201F091E3018083E091E201F0911E
:10213000E3018081882311F481E003C0863010F030
:1021400085E08083E091E201F091E3014CE666E5F1
:1021500076E080810E94BD0680910F018823E1F323
:10216000E091E201F091E3018081898382E58A8335
:102170008CE690E09F938F9386E596E09F938F93F4
:1021800021E030E03F932F93CE0102969F938F93EF
:102190003F932F93CE01820F931F9F938F9383E0E2
:1021A0008F9381E08F9381E58F930E94950EADB759
:1021B000BEB71F96ADBF10C12091E2013091E3017F
:1021C000F90180818150853008F04CC081818235D1
:1021D00009F048C066E576E08CE62E5F3F4FDB01F4
:1021E000F901982F01900D929A95E1F72250304015
:1021F000482FD9018C910E94E60680919306992779
:10220000AA27BB27BC01CD0124EC39E040E050E017
:102210000E943C6EDC01CB018093990190939A015E
:10222000A0939B01B0939C01809194069927AA27C3
:10223000BB27BC01CD010E943C6EDC01CB01809329
:10224000950190939601A0939701B0939801E09126
:10225000E201F091E30180810E94DA060E941507F5
:10226000898301C0198280910F018823E1F381E005
:1022700090E09F938F93CE0101969F938F9381E07F
:102280008F938F9383E58F930E94950EEDB7FEB7E2
:102290003796EDBF2EC0E091E201F091E301E081BD
:1022A0008E2F8150853018F48E2F0E94DA06E0912F
:1022B000E201F091E301808189834CE666E576E0F6
:1022C0000E94BD0680910F018823E1F381E090E038
:1022D0009F938F93CE0101969F938F9381E08F936D
:1022E0008F9386E48F930E94950E8DB79EB70796C5
:1022F0008DBF80917902882329F46EE670E0898190
:102300000E94EF2F80E00E945C070E94AD6664C0CF
:10231000E091E201F091E3018081992787FD90959A
:1023200090930206809301068181992787FD9095FD
:1023300090930406809303068281992787FD9095E8
:1023400090930606809305068381992787FD9095D3
:1023500090930806809307068481992787FD9095BE
:1023600090930A06809309068581992787FD9095A9
:1023700090930C0680930B068681992787FD909594
:1023800090930E0680930D068781992787FD90957F
:102390009093100680930F068085992787FD90956E
:1023A00090931206809311068185992787FD909559
:1023B00090931406809313068285992787FD909544
:1023C00090931606809315068385992787FD90952F
:1023D00090931806809317068091240499278436D9
:1023E000910509F4C5C085369105ACF48136910597
:1023F00009F479C0823691052CF48B34910509F4E7
:1024000055C019C18236910509F47AC08336910509
:1024100009F489C010C18C36910509F4F7C08D36D6
:1024200091054CF48736910509F402C1883691056F
:1024300009F4BCC000C18437910529F086379105A5
:1024400009F4F2C0F8C08091E401A091E201B091DA
:10245000E301853140F080E1EDEFF3E00D90019272
:102460008A95E1F70DC08D919D910D90BC91A02DA5
:102470008093FD039093FE03A093FF03B0930004A9
:1024800080910F018823E1F31F9280910C018F93BB
:1024900084E58F930E94950E8AEF8093DF018FEF82
:1024A00080930D010F900F900F90C5C0E091E20155
:1024B000F091E3018081918190939602809395023F
:1024C0002091930230919402821B930B845E9D4F66
:1024D00068E671E00E947B6E845B9040909392026C
:1024E00080939102A8C0E091E201F091E301808124
:1024F00080930E01803298F08FE180930E010FC01F
:10250000A091E201B091E3018BE0E5E1F4E00D90F0
:1025100001928A95E1F780911E048093A6058FEFC2
:1025200080930D0188C08091DB019091DC01892BA3
:1025300089F4E091E201F091E301E081EE2351F0B2
:102540008AE0E89FC00111240E94F0169093F003E6
:102550008093EF03E091E201F091E30190818AE042
:10256000989FC00111249093DC018093DB0115C07A
:102570008FEF80930D01E091E201F091E3019081F2
:102580008AE0989FC00111249093DE018093DD01C1
:10259000892B19F081E08093EC0180EA9FE00E9492
:1025A000F0169093D8018093D70145C08FEF8093A8
:1025B0000D01E091E201F091E301908197FD08C0E7
:1025C00082E08093E9011092DA011092D9011AC0D9
:1025D000909580914202892B8093420291818AE0FA
:1025E000989FC00111249093DA018093D90184E06F
:1025F0008093E90180EA9FE00E94F0169093D80151
:102600008093D70181E08093ED0115C08FEF809317
:102610000D01E091E201F091E3018081809343029A
:1026200081E08093EE0107C081E08093EB0103C05D
:1026300081E08093EF011092E7011092E301109284
:10264000E2011092E101E2E0CE5F0C94F76E982F68
:102650008091C00085FFFCCF9093C600089588E16B
:102660008093C1008091C00082608093C0008091FF
:10267000C10080688093C1008091C1008064809314
:10268000C1008AE28093C4008091DD019091DE0157
:102690000E94F0169093F2038093F1038CED90E08A
:1026A0000E94F01690932104809320041092F3036B
:1026B0008EE48093F40381E08093F7038BE08093B2
:1026C000F5031092F6031092E3011092E2011092CA
:1026D000E1010895A0E1B0E0E0E7F3E10C94D76EEA
:1026E00080910F01882309F48CC28091D7019091C9
:1026F000D8010E94F916882361F01092DA01109235
:10270000D9011092DE011092DD011092DC011092CD
:10271000DB018091D9019091DA01892B41F0809100
:10272000C2049091C3040E94F916882329F4809171
:10273000ED01882309F460C080910F01882309F41A
:102740005BC08091E90108E211E08430A8F00E94AA
:10275000C82080E590E09F938F931F930F9381E0B3
:102760008F938F9388E48F930E94950E2DB73EB779
:10277000295F3F4F2DBF34C01092440284ED94E096
:102780009F938F938DEB90E29F938F93E0919203B1
:10279000F0919303099584E190E09F938F931F93A9
:1027A0000F9381E090E09F938F9389EE91E09F9348
:1027B0008F9382E08F9381E08F9388E48F930E94C0
:1027C000950E8091E901982F8F5F8093E9012DB7D5
:1027D0003EB7215F3F4F2DBF943010F01092E901BA
:1027E0008091D9019091DA010E94F0169093C30470
:1027F0008093C2041092ED018091EE01882351F183
:1028000080910F01882331F10E94C82080E590E07B
:102810009F938F9388E291E09F938F9321E030E024
:102820003F932F9387E291E09F938F933F932F9352
:1028300083E492E09F938F9383E08F9381E08F9363
:102840008CE48F930E94950E1092EE018DB79EB787
:102850000F968DBF8091EB018823D1F080910F01FD
:102860008823B1F08AE090E09F938F9383EF93E009
:102870009F938F9381E08F938F9386E58F930E9430
:10288000950E1092EB012DB73EB7295F3F4F2DBF3C
:102890008091EF018823D9F080910F018823B9F04E
:1028A0008BE090E09F938F9385E194E09F938F93CB
:1028B00081E08F9380910C018F9387E48F930E9426
:1028C000950E1092EF018DB79EB707968DBF809140
:1028D0002004909121040E94F916882309F461C014
:1028E00080910F01882309F45CC0809171069927BB
:1028F000880F991F880F991F7C010027F7FC00950E
:10290000102F8091CF029091D002A091D102B0916E
:10291000D202BC01CD01A80197010E94B06E309394
:102920000E0420930D048091C7029091C802A091DB
:10293000C902B091CA02BC01CD01A80197010E9451
:10294000B06E3093100420930F0480916602809340
:102950001104809165028093120488E090E09F93B7
:102960008F938DE094E09F938F9381E08F9383E02A
:102970008F9387E78F930E94950E809113042DB754
:102980003EB7295F3F4F2DBF853018F086E080931A
:10299000130483E690E00E94F01690932104809344
:1029A00020048091DD019091DE01892B41F080911E
:1029B000F1039091F2030E94F916882321F480918B
:1029C000EC01882329F180910F01882309F182E429
:1029D00090E09F938F9384E695E09F938F9381E09F
:1029E0008F938F9384E48F930E94950E1092EC0145
:1029F0008DB79EB707968DBF8091DD019091DE0166
:102A0000009731F00E94F0169093F2038093F10347
:102A10008091DB019091DC01892B09F485C08091C4
:102A2000EF039091F0030E94F916882309F47CC00B
:102A300080910F01882309F477C08091710699274E
:102A4000880F991F880F991F7C010027F7FC0095BC
:102A5000102F8091CF029091D002A091D102B0911D
:102A6000D202BC01CD01A80197010E94B06E309343
:102A7000E2032093E1038091C7029091C802A091E4
:102A8000C902B091CA02BC01CD01A80197010E9400
:102A9000B06E3093E4032093E30320911D0730913F
:102AA0001E0740911F0750912007DA01C90103E07A
:102AB000880F991FAA1FBB1F0A95D1F7820F931F7A
:102AC000A41FB51F820F931FA41FB51F209179016A
:102AD00030917A0140917B0150917C01BC01CD0184
:102AE0000E94B06E3093E6032093E5038EE090E001
:102AF0009F938F9381EE93E09F938F9381E08F93C9
:102B00008F9383E48F930E94950E8091DB019091C7
:102B1000DC010E94F0169093F0038093EF032DB731
:102B20003EB7295F3F4F2DBF80910E018F3F71F15E
:102B3000992714E0880F991F1A95E1F78C529D4F41
:102B400040E150E0BC01CE0101960E94486D80E159
:102B500090E09F938F93CE0101969F938F9381E096
:102B600090E09F938F938EE091E09F938F9382E00C
:102B70008F9381E08F9381E48F930E94950E8FEF66
:102B800080930E018DB79EB70B968DBF8091A605E1
:102B90008823D1F080910F018823B1F081E090E08B
:102BA0009F938F9386EA95E09F938F9381E08F9315
:102BB0008F9382E48F930E94950E1092A6052DB7F5
:102BC0003EB7295F3F4F2DBF8091EA018823C9F0AE
:102BD00080910F018823A9F084E390E09F938F9365
:102BE00087EE95E09F938F9381E08F938F9380E59D
:102BF0008F930E94950E1092EA018DB79EB70796AB
:102C00008DBFE6E0C05F0C94F36E1F920F920FB67B
:102C10000F9211242F933F935F936F937F938F9322
:102C20009F93AF93BF93EF93FF938091FD01882310
:102C300029F08091FD0181508093FD018091760300
:102C4000882319F08150809376038091050281508A
:102C5000809305028F3FB9F489E08093050280914B
:102C600012018F5F817080931201882319F481E033
:102C70008093020280910302909104020196909346
:102C80000402809303028091FE019091FF01892B41
:102C9000C9F08091FE019091FF0101979093FF018F
:102CA0008093FE018091FE019091FF01209110011F
:102CB0003091110182239323892B11F021E009C067
:102CC00020E007C020E08FEF9FEF909311018093E9
:102CD000100180910201222331F08A3011F45A9AB6
:102CE00007C0479A05C08A3011F45A9801C0479826
:102CF00080916803882309F063C08091620683FF96
:102D00005FC086B19927FC01E071F07084FF0AC0B2
:102D100080910002909101020196909301028093AC
:102D200000024EC08091000290910102892B09F4AB
:102D300043C080910002909101028A569140E0F5D3
:102D4000809100029091010269E270E00E94676E3A
:102D50008091000290910102860F971F90930102CB
:102D60008093000280910002909101020B9750F035
:102D700080910002909101020A97909396028093AD
:102D8000950204C0F0939602E0939502809195021B
:102D9000909196022091930230919402821B930BA2
:102DA000845E9D4F68E671E00E947B6E845B90407C
:102DB000909392028093910210920102109200026D
:102DC000FF91EF91BF91AF919F918F917F916F9103
:102DD0005F913F912F910F900FBE0F901F9018950C
:102DE0002091030230910402280F391FC901019676
:102DF00008952091030230910402821B930B892FC6
:102E000099278695807490700895CF93DF930E94E0
:102E1000F016EC01CE010E94F9168823D9F3DF9158
:102E2000CF910895CF93DF930E94F016EC0109C073
:102E300080911701882329F0909317018FEC8093DC
:102E40007A00CE010E94F916982F882389F3DF912A
:102E5000CF9108959FB7F8945F983E9A469A8091D3
:102E6000B0008F708093B0008091B0008360809339
:102E7000B0008091B1008B738093B1008091B1005C
:102E80008B608093B1001092B2008FEF8093B300FB
:102E90008091B00080688093B000809170008A7F3C
:102EA00080937000809170008260809370009FBF5B
:102EB00008958AE090E00E94F01690930D028093AE
:102EC0000C0282E085BD83EA84BD17BC88E788BD1B
:102ED00086E086BD80916E00816080936E000895CB
:102EE0001F920F920FB60F9211242F933F934F937F
:102EF0005F936F937F938F939F93AF93BF93CF9382
:102F0000DF93EF93FF938091020190910602843149
:102F100008F011C1992309F064C38091B00086FFC5
:102F2000ECC08091B0008F7B8093B00089EA93E081
:102F300090930802809307028091130190911401ED
:102F40009C01220F331F280F391F8091850199277B
:102F5000880F991F880F991F280F391F37FF02C04C
:102F60002D5F3F4FC90195958795959587959093CE
:102F70001401809313019093FB018093FA018091D7
:102F8000B406609182062091CF023091D002409128
:102F9000D1025091D20280FF2CC077278827992731
:102FA000EA01D90157FF04C0A158BF4FCF4FDF4FEF
:102FB000E7E0D595C795B795A795EA95D1F79D0117
:102FC000AE010E943C6E9B01AC0197FF04C0215CE6
:102FD0003F4F4F4F5F4F66E0559547953795279583
:102FE0006A95D1F78091FA019091FB01820F931FAE
:102FF0002BC0772788279927EA01D90157FF04C0FA
:10300000A158BF4FCF4FDF4F27E0D595C795B79554
:10301000A7952A95D1F79D01AE010E943C6E9B01B8
:10302000AC0197FF04C0215C3F4F4F4F5F4FF6E06C
:103030005595479537952795FA95D1F78091FA01DF
:103040009091FB01821B930B9093FB018093FA01FB
:1030500080918306282F3327220F331F220F331F1F
:103060008091FA019091FB01821793077CF0809187
:103070008406282F3327220F331F220F331F8091FE
:10308000FA019091FB012817390724F43093FB01D2
:103090002093FA0120910702309108028091FA01F1
:1030A0009091FB01280F391F2050324030930802C5
:1030B000209307028091FA019091FB0197FD0396FE
:1030C00095958795959587959093FB018093FA0147
:1030D00045E02D3D340718F08CED95E005C02757ED
:1030E000314030F487E791E0909308028093070223
:1030F000809107029091080241C28091B0008064E3
:103100008093B00080918906282F33278DED96E0BB
:10311000289FA001299F500D389F500D1124CA01EE
:103120002091090230910A02821B930B90930802AE
:103130008093070253C2992309F053C28091B000D3
:1031400086FF21C28091B0008F7B8093B000E09118
:103150000B02EE23F1F480918906282F33278DEDA1
:1031600096E0289FA001299F500D389F500D1124F3
:10317000CA012091090230910A02821B930B90939D
:1031800008028093070210920A0210920902469ADE
:1031900025C289EA93E090930802809307028E2F5C
:1031A00099278330910509F4A4C1843091053CF43A
:1031B0008130910561F0029709F4D2C0A8C1843032
:1031C000910509F499C1059709F49EC1A0C18091A8
:1031D0001301909114019C01220F331F280F391FF6
:1031E000809185019927880F991F880F991F280FB3
:1031F000391F37FF02C02D5F3F4FC9019595879555
:103200009595879590931401809313019093FB01FA
:103210008093FA018091B406609182062091CF02DA
:103220003091D0024091D1025091D20280FF2CC047
:10323000772788279927EA01D90157FF04C0A158A9
:10324000BF4FCF4FDF4F27E0D595C795B795A795CF
:103250002A95D1F79D01AE010E943C6E9B01AC0105
:1032600097FF04C0215C3F4F4F4F5F4FA6E055953D
:10327000479537952795AA95D1F78091FA019091B6
:10328000FB01820F931F27C077278827992757FFB5
:1032900004C021583F4F4F4F5F4FF7E0559547957A
:1032A00037952795FA95D1F70E943C6E9B01AC01AA
:1032B00097FF04C0215C3F4F4F4F5F4FE6E05595AD
:1032C000479537952795EA95D1F78091FA01909126
:1032D000FB01821B930B9093FB018093FA01809179
:1032E0008306282F3327220F331F220F331F80918D
:1032F000FA019091FB01821793077CF0809184067C
:10330000282F3327220F331F220F331F8091FA01FA
:103310009091FB012817390724F43093FB01209387
:10332000FA0180910702909108022091FA013091F0
:10333000FB01820F931F805092409093080280936C
:1033400007028091FA019091FB0197FD03969595F4
:103350008795959587959093FB018093FA01EAC034
:1033600080911501909116019C01220F331F280FA7
:10337000391F809184019927880F991F880F991F01
:10338000280F391F37FF02C02D5F3F4FC9019595A8
:103390008795959587959093160180931501909345
:1033A000F9018093F8018091B40660918606A0919E
:1033B000C702B091C802C091C902D091CA0281FF70
:1033C0002AC07727882799279D01AE01D7FF04C01F
:1033D00021583F4F4F4F5F4FA7E055954795379581
:1033E0002795AA95D1F70E943C6E9B01AC0197FFEF
:1033F00004C0215C3F4F4F4F5F4FF6E05595479516
:1034000037952795FA95D1F78091F8019091F901B8
:10341000820F931F29C07727882799279D01AE0126
:10342000D7FF04C021583F4F4F4F5F4FE7E05595FE
:10343000479537952795EA95D1F70E943C6E9B01F9
:10344000AC0197FF04C0215C3F4F4F4F5F4F66E0D8
:1034500055954795379527956A95D1F78091F8014D
:103460009091F901821B930B9093F9018093F801DD
:1034700080918706282F3327220F331F220F331FF7
:103480008091F8019091F901821793077CF0809167
:103490008806282F3327220F331F220F331F8091D6
:1034A000F8019091F9012817390724F43093F901B4
:1034B0002093F80180910702909108022091F80171
:1034C0003091F901820F931F80509240909308022F
:1034D000809307028091F8019091F90197FD03967E
:1034E00095958795959587959093F9018093F80127
:1034F00021C08091E90602C0809155069927880F66
:10350000991F87559C4F12C08091F306F7CFFF2774
:10351000EE0FFF1FE951FA4F20813181220F331F37
:103520008091070290910802820F931F90930802E6
:1035300080930702809107029091080255E08D3D2B
:10354000950718F08CED95E005C08757914030F451
:1035500087E791E090930802809307022091070289
:10356000309108022C5B3040309308022093070210
:103570008091090290910A02820F931F90930A0290
:10358000809309022BC08091B00080648093B000CA
:103590008CEB90E0909308028093070280910902DF
:1035A00090910A0284549F4F90930A0280930902DB
:1035B0008091FC01882331F080918302853B10F0DB
:1035C000469801C0469A80910B028F5F80930B0250
:1035D00090918906981710F410920B0281E0809365
:1035E0000602209107023091080241E02F3734078C
:1035F00030F08FEF8093B3002F5F30400FC02F3F2C
:103600003105C9F0C0F0A9014F5F50404F37510557
:1036100050F480E88093B300205830403093080283
:103620002093070212C08FEF8093B30050930802DB
:10363000409307020AC0809107028093B300109262
:1036400008021092070210920602FF91EF91DF919B
:10365000CF91BF91AF919F918F917F916F915F912A
:103660004F913F912F910F900FBE0F901F90189583
:1036700010927C008FEC80937A0008950F931F9333
:10368000CF93DF9303E010E0D8010E94086F802DF4
:10369000C82FDD27C531D10508F02A97C7BD109284
:1036A000150284E690E00E94121780911B01909110
:1036B0001C018052934010F4C0E0D0E0CA3FD10515
:1036C000F8F4C7BD82E390E00E94121789EE94E0FF
:1036D0009F938F9387E293E19F938F93E09192035F
:1036E000F0919303099580911B0190911C010F901B
:1036F0000F900F900F908052934010F02196DECFE4
:10370000D8010C2E0E94156FC093B3058CE291E096
:103710000E941217DF91CF911F910F910895EF92A0
:10372000FF921F93CF93C0E0C0931002C0930F028B
:10373000C0930E0280ED97E00E94F0167C011CE819
:10374000C33019F41B3008F019E0C0E08091250265
:10375000909126028C5F934024F480911A0181504D
:103760000AC080912502909126028750944034F03F
:1037700080911A018F5F80931A0101C0C1E080918E
:103780002302909124028C5F934024F480911901CC
:1037900081500AC080912302909124028750944066
:1037A00034F0809119018F5F8093190101C0CF5FC0
:1037B00080912102909122028C5F934024F48091A9
:1037C000180181500AC080912102909122028750F5
:1037D0009440C4F0809118018F5F8093180113C04A
:1037E0008BEE94E09F938F9387E293E19F938F9367
:1037F000E0919203F091930309950F900F900F9031
:103800000F904DC0CF5F88E080934A020E94E82A63
:1038100080911A018A3030F481E0809310028AE0AE
:1038200080931A0180911A01863F30F081E08093E5
:10383000100285EF80931A01809119018A3030F4CB
:1038400081E080930F028AE0809319018091190131
:10385000863F30F081E080930F0285EF809319015D
:10386000809118018A3030F481E080930E028AE062
:103870008093180180911801863F30F081E0809399
:103880000E0285EF8093180180914A02882339F057
:10389000C7010E94F916882309F0A2CFF5CF109234
:1038A00017018FEC80937A00809117018823E1F350
:1038B0001A3020F48AE090E00E941217115009F0AB
:1038C0003FCF86E490E00E941217CF911F91FF90A6
:1038D000EF9008951F920F920FB60F921124AF929E
:1038E000BF92CF92DF92EF92FF920F931F932F938D
:1038F0003F934F935F936F937F938F939F93AF9378
:10390000BF93EF93FF9380912E02282F33274427F4
:1039100055278F5F80932E02F9012231310508F07F
:10392000FAC3E25CFF4F0C94026F80917800909193
:10393000790046C080917800909179009AC1809179
:103940007800909179009093300280932F02C5C146
:103950008091DB029091DC02209178003091790017
:10396000821B930B9093A8058093A7058091A705D0
:103970009091A80590933A0280933902CCC180912E
:103980007800909179002091DD023091DE02821B57
:10399000930B9093B2058093B1058091B1059091FE
:1039A000B20590933C0280933B02B7C380913302EF
:1039B000909134022091780030917900820F931F0A
:1039C000909334028093330281E0A8C38091310246
:1039D000909132022091780030917900820F931FEC
:1039E000909332028093310284E098C38091250144
:1039F000909126019C01220F331F280F391F8091BF
:103A000078009091790063E070E00E94676E260F65
:103A1000371F3695279536952795309326012093A5
:103A2000250185E07BC38091780090917900AA27D9
:103A300097FDA095BA2FBC01CD010E94C26D7B01FC
:103A40008C018091D5029091D602A091D702B091BD
:103A5000D8029C01AD01C801B7010E94626DDC0172
:103A6000CB01BC01CD010E94A56DDC01CB0190937F
:103A70001C0280931B0280911B0290911C020297F2
:103A80000CF446C08091D5029091D602A091D70245
:103A9000B091D80220E030E84BE354E4BC01CD0102
:103AA0000E94CC6D88230CF088C08091D502909143
:103AB000D602A091D702B091D8022AE037ED43EAAE
:103AC0005CE3BC01CD010E94636DDC01CB018093FE
:103AD000D5029093D602A093D702B093D8028091DA
:103AE000530290915402845F914008F066C0809127
:103AF000D5029091D602A091D702B091D8022DECB8
:103B00003CEC4CEC5DE3BC01CD010E94636D4BC00D
:103B100080911B0290911C028F5F9F4F0CF04DC053
:103B20008091D5029091D602A091D702B091D8028F
:103B300020E030E849E054E4BC01CD010E94CF6DA3
:103B40001816DCF58091D5029091D602A091D7028B
:103B5000B091D8022AE037ED43EA5CE3BC01CD0125
:103B60000E94626DDC01CB018093D5029093D60256
:103B7000A093D702B093D80280915302909154023F
:103B8000845F9140D0F48091D5029091D602A091AB
:103B9000D702B091D8022DEC3CEC4CEC5DE3BC01BB
:103BA000CD010E94626DDC01CB018093D502909320
:103BB000D602A093D702B093D80281E080931A0274
:103BC00080917800909179009093AA058093A9053F
:103BD00080911B0290911C029C01442737FD409567
:103BE000542F8091970290919802A0919902B091E0
:103BF0009A02820F931FA41FB51F80939702909380
:103C00009802A0939902B0939A0220919702309162
:103C100098024091990250919A0257FF04C0215096
:103C20003C4F4F4F5F4F0AE0559547953795279585
:103C30000A95D1F78091970290919802A0919902EC
:103C4000B0919A02821B930BA40BB50B8093970241
:103C500090939802A0939902B0939A022EC18091FA
:103C60003102909132022091780030917900820FD8
:103C7000931F909332028093310210922D0250C212
:103C8000809102018A3071F48091780090917900DE
:103C900020912F0230913002820F931F019696954A
:103CA000879517C040912F0250913002843159F40A
:103CB0002091780030917900240F351F8FEF97E025
:103CC000821B930B06C08091780090917900840F3D
:103CD000951F909322028093210286E01FC280915B
:103CE000DB029091DC022091780030917900821BF8
:103CF000930B9093A8058093A7058091A7059091B9
:103D0000A8052091390230913A02820F931F9093B7
:103D1000200280931F0287E001C280917800909179
:103D200079002091DD023091DE02821B930B90938B
:103D3000B2058093B1058091B1059091B2052091B3
:103D40003B0230913C02820F931F90931E0280939E
:103D50001D02E3C12091330230913402809178003A
:103D600090917900280F391F309334022093330249
:103D7000809102018A3019F4220F331F04C0220FF0
:103D8000331F220F331F30933402209333022091CC
:103D9000330230913402C90137FD0796A3E09595AF
:103DA0008795AA95E1F7909326028093250280914A
:103DB000350290913602820F931F97FD01969595DB
:103DC000879590933602809335022091E7023091D7
:103DD000E802821B930B909324018093230120918E
:103DE0002B0230912C028091230190912401280F05
:103DF000391F37FF02C02F5F3F4F3595279530930E
:103E00002C0220932B02E0CD20913102309132021E
:103E10008091780090917900280F391F30933202F9
:103E200020933102809102018A3019F4220F331F4E
:103E300004C0220F331F220F331F3093320220930E
:103E400031022091310230913202C90137FD0796CB
:103E500063E0959587956A95E1F7909324028093A6
:103E600023028091370290913802820F931F97FDB1
:103E7000019695958795909338028093370220910B
:103E8000E5023091E602821B930B9093220180930E
:103E900021012091290230912A02809121019091E3
:103EA0002201280F391F37FF02C02F5F3F4F359582
:103EB000279530932A022093290283E02FC1109284
:103EC0002E0281E0809317018091110290911202DD
:103ED0000196909312028093110280917800909144
:103EE000790090931C0180931B0180911B0190919C
:103EF0001C01AA27BB27A0903D02B0903E02C090B3
:103F00003F02D0904002A80EB91ECA1EDB1EA0922E
:103F10003D02B0923E02C0923F02D0924002809198
:103F200041028F5F80934102823108F4F6C0809194
:103F30001D0190911E01A0911F01B09120017C01F3
:103F40008D0123E0EE0CFF1C001F111F2A95D1F7F5
:103F5000E81AF90A0A0B1B0BEA0CFB1C0C1D1D1DB1
:103F600080911502992787FD9095A92FB92FBC0143
:103F7000CD0126EC34E240E050E00E943C6EDC01D2
:103F8000CB01E81AF90A0A0B1B0BD801C7010496EA
:103F9000A11DB11DB7FF05C0D801C7010B96A11D1A
:103FA000B11D13E0B595A795979587951A95D1F70B
:103FB00080931D0190931E01A0931F01B0932001D7
:103FC0008091AB059091AC057C010027F7FC009532
:103FD000102F80911D0190911E01A0911F01B091A1
:103FE0002001E81AF90A0A0B1B0BE0927502F09205
:103FF0007602009377021093780220911602309196
:104000001702409118025091190257FF04C0215F16
:104010003F4F4F4F5F4FF4E05595479537952795A4
:10402000FA95D1F78091160290911702A09118028B
:10403000B0911902821B930BA40BB50B809316024F
:1040400090931702A0931802B09319028091160260
:1040500090911702A0911802B09119028E0D9F1D28
:10406000A01FB11F8093160290931702A09318020D
:10407000B09319028091130290911402AC01E4E014
:10408000440F551FEA95E1F7481B590B8091160222
:1040900090911702A0911802B0911902B7FF03C0C6
:1040A0000F96A11DB11D74E0B595A79597958795BD
:1040B0007A95D1F72091750230917602281B390B41
:1040C00063E0220F331F6A95E1F7240F351F37FF96
:1040D00002C0215F3F4F44E0359527954A95E1F7AF
:1040E0003093140220931302D601C501D7FE03C0FA
:1040F0000196A11DB11DB595A795979587958093BC
:104100003D0290933E02A0933F02B093400289E0AB
:104110008093410202C010922E0282E080932D0211
:1041200080912D0280937C0080912E02882319F0CB
:104130008FEC80937A00FF91EF91BF91AF919F91A7
:104140008F917F916F915F914F913F912F911F912F
:104150000F91FF90EF90DF90CF90BF90AF900F90B6
:104160000FBE0F901F90189590E2E8E2F1E08FE407
:104170009193815087FFFCCF089590914402E8E22B
:10418000F1E0E90FF11D80839F5F90934402089551
:10419000EF92FF920F931F93CF93DF9320914202F0
:1041A00020FF0AC080914302882311F0815002C091
:1041B000809127018093430221FF0CC0909143021C
:1041C00080912701981719F41092430203C09F5F52
:1041D00090934302822F992780FF04C081FF02C081
:1041E000109243020E94B42080914302282F33276B
:1041F000CDEBEC2EC0E2FC2EC0919203D091930344
:104200008A3098F481E1809344023F932F9382E2B5
:1042100095E09F938F93FF92EF92FE0109952DB742
:104220003EB72A5F3F4F2DBF11C080E1809344020B
:104230003F932F9387E295E09F938F93FF92EF92A6
:10424000FE0109958DB79EB706968DBF209143025A
:10425000822F9927AA27BB27FC01419710F00C94C5
:10426000D22AE05BFF4FBDEBEB2EB0E2FB2EC091FC
:104270009203D09193030C94026F109244028CE24B
:1042800095E09F938F93FF92EF92FE01099584E151
:10429000809344020F900F900F900F9082E690E071
:1042A0009F938F938EE490E09F938F931F921F9222
:1042B000809102016AE00E945B6E892F99279F938B
:1042C0008F93809102010E945B6E99279F938F9339
:1042D0008CE395E09F938F93FF92EF92E09192038E
:1042E000F0919303099588E2809344022DB73EB77D
:1042F000225F3F4F2DBF85E993E09F938F930E94EC
:10430000150799279F938F9381E595E09F938F934E
:10431000FF92EF92E0919203F091930309958091BF
:104320009F019091A0012DB73EB7285F3F4F2DBF51
:10433000069730F48CE3809344028FE595E0CDC07E
:1043400090914702992311F40C94DB2A8CE380931B
:104350004402892F99279F938F938CE695E09F9332
:104360008F938DEB90E29F938F9377C0809162063D
:10437000ADEBEA2EA0E2FA2EC0919203D091930306
:1043800080FF74C010924402809175029091760271
:10439000A0917702B0917802BC01CD0125E030E018
:1043A00040E050E00E94B06E3F932F9381E895E08B
:1043B0009F938F93FF92EF92FE01099584E1809382
:1043C00044022DB73EB72A5F3F4F2DBF8091710247
:1043D00090917202A0917302B0917402BC01CD0160
:1043E00025E030E040E050E00E94B06E3F932F9314
:1043F0008EE895E09F938F93FF92EF92E091920366
:10440000F0919303099588E2809344028DB79EB79B
:1044100006968DBF80911B0190911C019F938F93F5
:104420008BE995E09F938F93FF92EF92E091920337
:10443000F091930309958CE3809344022DB73EB726
:104440002A5F3F4F2DBF87B599279F938F9388EAA7
:1044500095E09F938F93FF92EF92E0919203F091FA
:10446000930309958DB79EB7069639C710924402FB
:1044700085EB95E09F938F93FF92EF92FE01099554
:1044800084E1809344020F900F900F900F9084EC82
:1044900095E09F938F93FF92EF92E0919203F091BA
:1044A0009303099588E2809344020F900F900F9038
:1044B0000F908DEC95E09F938F93FF92EF92E09198
:1044C0009203F091930309958CE3809344020F903B
:1044D0000F900F900F908CED95E09F938F93FF922C
:1044E000EF92EFC71092440285EE95E09F938F9371
:1044F0000DEB10E2FF92EF92FE01099584E18093AB
:1045000044020F900F900F900F908091CF029091E6
:10451000D002A091D102B091D202B7FF04C0815065
:104520009C4FAF4FBF4FFAE0B595A79597958795EC
:10453000FA95D1F7BF93AF939F938F9382EF95E056
:104540009F938F931F930F93E0919203F0919303A6
:10455000099588E2809344022DB73EB7285F3F4F0C
:104560002DBF8091C7029091C802A091C902B0915D
:10457000CA02B7FF04C081509C4FAF4FBF4FEAE063
:10458000B595A79597958795EA95D1F7BF93AF9382
:104590009F938F9381E096E09F938F931F930F9348
:1045A000E0919203F091930309958CE38093440288
:1045B0008DB79EB708968DBF809195029091960217
:1045C0009F938F9380E196E09F938F931F930F9318
:1045D000EEC3109244028091EB059091EC059F93FD
:1045E0008F938091E9059091EA059F938F938FE1D6
:1045F00096E09F938F93FF92EF92FE01099584E1DD
:10460000809344028DB79EB708968DBF8091EF05C9
:104610009091F0059F938F938091ED059091EE0519
:104620009F938F938FE296E09F938F93FF92EF92E9
:10463000E0919203F0919303099588E280934402FC
:104640002DB73EB7285F3F4F2DBF8091F305909166
:10465000F4059F938F938091F1059091F2059F93BC
:104660008F938FE396E09F938F93FF92EF92E09169
:104670009203F091930309958CE3809344028DB7E4
:104680009EB708968DBF8091F7059091F8059F938E
:104690008F938091F5059091F6059F938F938FE40A
:1046A00096E076C51092440280915706E82FFF27C6
:1046B000EE0FFF1FE951FA4F808191819F938F93F5
:1046C00080915606E82FFF27EE0FFF1FE951FA4FA2
:1046D000808191819F938F938FE596E09F938F9335
:1046E000FF92EF92FE01099584E1809344028DB719
:1046F0009EB708968DBF80915906E82FFF27EE0FD1
:10470000FF1FE951FA4F808191819F938F93809190
:104710005806E82FFF27EE0FFF1FE951FA4F80815F
:10472000918188589F4F9F938F938FE696E09F9338
:104730008F93FF92EF92E0919203F091930309958A
:1047400088E2809344022DB73EB7285F3F4F2DBFCC
:1047500080915B06E82FFF27EE0FFF1FE951FA4F0C
:104760008081918182599F4F9F938F9380915A06A8
:10477000E82FFF27EE0FFF1FE951FA4F808191814B
:1047800082599F4F9F938F938FE796E09F938F93CC
:10479000FF92EF92E0919203F091930309958CE3DD
:1047A000809344028DB79EB708968DBF80915D06B9
:1047B000E82FFF27EE0FFF1FE951FA4F808191810B
:1047C00082599F4F9F938F9380915C06E82FFF271C
:1047D000EE0FFF1FE951FA4F8081918182599F4F5F
:1047E0009F938F938FE896E0D3C4109244028FE991
:1047F00096E09F938F930DEB10E2FF92EF92FE01F4
:104800000995809102010F900F900F900F908A30C0
:1048100009F0A1C084E1809344028091E702909165
:10482000E8029C0197FF02C0295F3F4F287F821B4F
:10483000930B9F938F938091E7029091E80297FDED
:10484000079673E0959587957A95E1F79F938F93F7
:104850002091E7023091E80237FF02C0295F3F4F05
:1048600063E0359527956A95E1F78091250290914F
:104870002602821B930B9F938F938DEA96E09F9362
:104880008F931F930F93E0919203F09193030995F7
:1048900088E2809344028DB79EB70A968DBF8091BF
:1048A000E5029091E6029C0197FF02C0295F3F4F0D
:1048B000287F821B930B9F938F938091E5029091A9
:1048C000E60297FD079653E0959587955A95E1F78F
:1048D0009F938F932091E5023091E60237FF02C04B
:1048E000295F3F4F43E0359527954A95E1F7809141
:1048F000230290912402821B930B9F938F938EEB44
:1049000096E09F938F931F930F93E0919203F09102
:10491000930309958CE3809344022DB73EB7265F3D
:104920003F4F2DBF8091E3029091E4029F938F93BC
:104930008091E3029091E4022091210230912202C1
:10494000821B930B9F938F938FEC96E09F938F9393
:104950001F930F93B6C38B3019F0843109F0ADC0AB
:1049600084E1809344028091E7029091E8029C01E7
:1049700097FF02C0215F3F4F207F821B930B97FD63
:104980000196959587959F938F938091E7029091DB
:10499000E80297FD0F9624E0959587952A95E1F713
:1049A0009F938F932091E7023091E80237FF02C076
:1049B000295F3F4F83E0359527958A95E1F78091F0
:1049C000250290912602821B930B9F938F938DED6E
:1049D00096E09F938F931F930F93E0919203F09132
:1049E0009303099588E2809344022DB73EB7265F72
:1049F0003F4F2DBF8091E5029091E6029C0197FF09
:104A000002C0215F3F4F207F821B930B97FD0196D1
:104A1000959587959F938F938091E5029091E602FB
:104A200097FD0F96B4E095958795BA95E1F79F931A
:104A30008F932091E5023091E60237FF02C0295F93
:104A40003F4FA3E035952795AA95E1F78091230282
:104A500090912402821B930B9F938F938FEE96E08D
:104A60009F938F931F930F93E0919203F091930381
:104A700009958CE3809344028DB79EB70A968DBF4B
:104A80008091E3029091E40297FD019695958795B8
:104A90009F938F938091E3029091E40220912102F1
:104AA00030912202821B930B9F938F9381E097E0BA
:104AB0009F938F931F930F936FC38D3009F07BC526
:104AC00084E18093440280911A0199279F938F93E8
:104AD0008091E7029091E80297FD0F96E4E09595AA
:104AE0008795EA95E1F79F938F932091E7023091A4
:104AF000E80237FF02C0295F3F4F73E035952795E5
:104B00007A95E1F78091250290912602821B930B02
:104B10009F938F9380E197E09F938F931F930F93C1
:104B2000E0919203F0919303099588E28093440207
:104B30008DB79EB70A968DBF8091190199279F93D3
:104B40008F938091E5029091E60297FD0F9664E0C5
:104B5000959587956A95E1F79F938F932091E5024C
:104B60003091E60237FF02C0295F3F4F53E0359591
:104B700027955A95E1F78091230290912402821B98
:104B8000930B9F938F9384E297E09F938F931F9350
:104B90000F93E0919203F091930309958CE3809336
:104BA00044022DB73EB7265F3F4F2DBF80911801BD
:104BB00099279F938F938091E3029091E40297FD50
:104BC0000196959587959F938F938091E30290919D
:104BD000E4022091210230912202821B930B9F93C9
:104BE0008F9388E397E09F938F931F930F93E091A8
:104BF0009203F091930309958DB79EB70A966FC300
:104C0000109244028CE497E09F938F93FF92EF926F
:104C1000FE01099584E1809344020F900F900F905C
:104C20000F908091DD029091DE029F938F9380918F
:104C30001D0290911E029F938F9389E597E09F93A9
:104C40008F93FF92EF92E0919203F0919303099575
:104C500088E2809344022DB73EB7285F3F4F2DBFB7
:104C60008091DB029091DC029F938F9380911F02D1
:104C7000909120029F938F9388E697E09F938F9364
:104C8000FF92EF92E0919203F091930309958CE3E8
:104C9000809344028DB79EB708968DBF8091D50250
:104CA0009091D602A091D702B091D802BC01CD015B
:104CB0000E94A56DDC01CB019F938F938091DE064E
:104CC0009091DF069F938F9387E797E061C21092E0
:104CD000440280912501909126016AE070E00E94D3
:104CE0007B6E9F938F9380912501909126016AE0BE
:104CF00070E00E947B6E7F936F9386E897E09F93AE
:104D00008F93FF92EF92FE01099584E18093440214
:104D10008DB79EB708968DBF8091930790919407A9
:104D20006AE070E00E94676E9F938F938091930773
:104D3000909194076AE070E00E94676E7F936F9392
:104D40008AE997E09F938F93FF92EF92E09192030D
:104D5000F0919303099588E2809344022DB73EB702
:104D6000285F3F4F2DBF80919507909196079F93A5
:104D70008F938EEA97E09F938F93FF92EF92E0914B
:104D80009203F091930309958CE3809344028DB7CD
:104D90009EB706968DBF80919707909198079F9335
:104DA0008F938EEB97E09F938F93FF92EF92E0911A
:104DB0009203F091930309952DB73EB72A5F3F4FB9
:104DC000F4C11092440280ED97E09F938F93FF927D
:104DD000EF92FE01099584E1809344020F900F90B9
:104DE0000F900F908091E7059091E8059F938F9326
:104DF00089ED97E09F938F93FF92EF92E09192035A
:104E0000F0919303099588E2809344028DB79EB791
:104E100006968DBF8091830299279F938F9389EE89
:104E200097E09F938F93FF92EF92E0919203F0911E
:104E3000930309958CE3809344022DB73EB72A5F14
:104E40003F4F2DBF8091E605992701979F938F9340
:104E500089EF97E0FECA1092440289E098E09F93A0
:104E60008F93FF92EF92FE01099584E180934402B3
:104E70000F900F900F900F9080919102909192025D
:104E80009F938F9381E198E09F938F93FF92EF928E
:104E9000E0919203F0919303099588E28093440294
:104EA0002DB73EB72A5F3F4F2DBF8091950290915D
:104EB00096029F938F938FE198E09F938F93FF9239
:104EC000EF92E0919203F091930309958CE3809324
:104ED00044028DB79EB706968DBF80919302909144
:104EE00094029F938F938DE298E05DCF10924402DD
:104EF0008091840299279F938F938BE398E09F93EF
:104F00008F93FF92EF92FE01099584E18093440212
:104F10008DB79EB706968DBF8091850299279F9386
:104F20008F9387E498E09F938F93FF92EF92E091A5
:104F30009203F0919303099588E2809344022DB780
:104F40003EB72A5F3F4F2DBF8091860299279F93DE
:104F50008F9383E598E09F938F93FF92EF92E09178
:104F60009203F091930309958CE3809344028DB7EB
:104F70009EB706968DBF8091870299279F938F9346
:104F80008FE598E010CF1092440280918802992713
:104F90009F938F938BE698E09F938F93FF92EF926E
:104FA000FE01099584E1809344028DB79EB7069671
:104FB0008DBF8091890299279F938F9387E798E00F
:104FC0009F938F93FF92EF92E0919203F09193035E
:104FD000099588E2809344022DB73EB72A5F3F4F80
:104FE0002DBF80918A0299279F938F9383E898E041
:104FF0009F938F93FF92EF92E0919203F09193032E
:1050000009958CE3809344028DB79EB706968DBFB9
:1050100080918B0299279F938F938FE898E0C3CE5E
:10502000109244028BE998E09F938F93FF92EF9246
:10503000FE01099584E1809344020F900F900F9038
:105040000F908091850199279F938F9383EA98E031
:105050009F938F93FF92EF92E0919203F0919303CD
:10506000099588E2809344028DB79EB706968DBF5E
:105070008091FA019091FB019F938F9381EB98E0CF
:105080009F938F93FF92EF92E0919203F09193039D
:1050900009958CE3809344022DB73EB72A5F3F4FBA
:1050A0002DBF8091840699279F938F9380918306CB
:1050B00099279F938F938FEB98E09F938F93FF9205
:1050C000EF92E0919203F091930309958DB79EB70B
:1050D000089605C1109244028DEC98E09F938F933F
:1050E000FF92EF92FE01099584E1809344020F90B4
:1050F0000F900F900F9080911904992787FD90953C
:105100009F938F9380911804992787FD90959F9383
:105110008F938DED98E09F938F93FF92EF92E091A4
:105120009203F0919303099588E2809344022DB78E
:105130003EB7285F3F4F2DBF80911A04992787FD06
:1051400090959F938F9380911B0499279F938F93A2
:105150008DEE98E09F938F93FF92EF92E0919203F0
:10516000F091930309958CE3809344028DB79EB729
:1051700008968DBF80911F0499279F938F938091EC
:105180001C04992787FD90959F938F938DEF98E04E
:105190009F938F93FF92EF92E0919203F09193038C
:1051A00009952DB73EB7285F3F4F2DBF04C210921F
:1051B00044028DE099E09F938F93FF92EF92FE015E
:1051C000099584E1809344020F900F900F900F9007
:1051D0008091C30599278F7790709F938F938091CB
:1051E000BF0599278F7790709F938F938091BB0510
:1051F00099278F7790709F938F938091B705992708
:105200008F7790709F938F938DE199E09F938F9309
:10521000FF92EF92E0919203F0919303099588E257
:10522000809344028DB79EB70C968DBF8091D305B5
:1052300099278F7790709F938F938091CF059927AF
:105240008F7790709F938F938091CB0599278F775D
:1052500090709F938F938091C70599278F77907057
:105260009F938F938EE299E09F938F93FF92EF929B
:10527000E0919203F091930309958CE380934402AB
:105280002DB73EB7245F3F4F2DBF8091E30599278F
:105290008F7790709F938F938091DF0599278F77F9
:1052A00090709F938F938091DB0599278F779070F3
:1052B0009F938F938091D70599278F7790709F93B5
:1052C0008F938FE399E09F938F93FF92EF92E091FA
:1052D0009203F091930309958DB79EB70C968DBFFD
:1052E0006AC11092440280E599E09F938F930DEB81
:1052F00010E2FF92EF92FE01099584E1809344024F
:105300000F900F900F900F908091C305881F8827F2
:10531000881F97E0899FC00111248D969F938F93DA
:105320008091BF05881F8827881F96E0899FC0014C
:1053300011248D969F938F938091BB05881F88279A
:10534000881F95E0899FC00111248D969F938F93AC
:105350008091B705881F8827881F9927880F991F74
:10536000880F991F8D969F938F938FE599E09F9358
:105370008F93FF92EF92E0919203F091930309953E
:1053800088E2809344022DB73EB7245F3F4F2DBF84
:105390008091D305881F8827881F9BE0899FC001C3
:1053A00011248D969F938F938091CF05881F882716
:1053B000881F9AE0899FC00111248D969F938F9337
:1053C0008091CB05881F8827881F99E0899FC0019D
:1053D00011248D969F938F938091C705881F8827EE
:1053E000881F992723E0880F991F2A95E1F78D964A
:1053F0009F938F9383E799E09F938F93FF92EF9210
:10540000E0919203F091930309958CE38093440219
:105410008DB79EB70C968DBF8091D705881F8827C2
:10542000881F9CE0899FC00111248D969F938F93C4
:1054300087E899E09F938F93FF92EF92E091920318
:10544000F091930309958091DB052DB73EB72A5F54
:105450003F4F2DBF87FF12C080E48093440288E94C
:1054600099E09F938F93FF92EF92E0919203F091D6
:10547000930309950F900F900F900F908091DF0587
:1054800087FF12C084E4809344028BE999E09F93E4
:105490008F931F930F93E0919203F09193030995DB
:1054A0000F900F900F900F908091E30587FF83C0BE
:1054B00088E4809344028EE999E09F938F931F9331
:1054C0000F93E0919203F091930309950F900F9041
:1054D0000F900F9070C01092440281EA99E09F9360
:1054E0008F93FF92EF92FE01099584E1809344022D
:1054F0000F900F900F900F908091D2019091D30157
:105500009F938F938FEA99E09F938F93FF92EF92EF
:10551000E0919203F0919303099588E2809344020D
:105520008DB79EB706968DBF8091D4019091D5011D
:105530009F938F938CEB99E09F938F93FF92EF92C1
:10554000E0919203F0919303099589E480934402DA
:105550002DB73EB72A5F3F4F2DBF89EC99E09F934F
:105560008F93FF92EF92E0919203F091930309954C
:10557000809142020F900F900F900F9083FF1BC0FD
:105580001092D5011092D401AEE0B0E080E0082E78
:105590000E94156FAFE0B0E08091D401082E0E9408
:1055A000156F09C080912701281719F42150209305
:1055B00027011092430210924202E6E0CDB7DEB717
:1055C0000C94F36E1092B9008AE28093B8000895AB
:1055D00085EA8093BC00089584E98093BC00089517
:1055E0001092B9008093BB0085E88093BC000895B9
:1055F0000E94EC2A10924A028091BB00109249024C
:1056000080E88093BC001092BD001092BA00109206
:10561000BB001092B9001092B8000E94E22A0E94CA
:10562000E82A80E00E94F02A08958093BB0085E874
:105630008093BC00089585EC8093BC00089585E8B4
:105640008093BC0008951F920F920FB60F92112401
:105650002F933F934F935F936F937F938F939F937A
:10566000AF93BF93EF93FF9380914A02282F332784
:10567000442755278F5F80934A02F901273131056E
:1056800008F0F2C0EF59FF4F0C94026F20914902CD
:10569000E22FFF27EE0FFF1FEE0FFF1FEC56FC4F10
:1056A00085851816A4F02C3090F4922F9F5FE92F77
:1056B000FF27EE0FFF1FEE0FFF1FEC56FC4F8585F7
:1056C00018161CF0292F9C3080F39093490280918A
:1056D00049028C3051F41092490283E080934A02CF
:1056E00080914802880F8D5AB4C0880F8E5AB1C07D
:1056F00080914902E82FFF27EE0FFF1FEE0FFF1FDB
:10570000EA54FA4F8F5F809349028081A2C0809152
:10571000B9008033E1F480914B02882321F4809119
:10572000490280934B0280914902E82FFF27EE0F38
:10573000FF1FEE0FFF1FED54FA4F2081822F992794
:105740008F7790708F37910514F42F5F20830E941C
:10575000EC2A8AE090E09093A00180939F01109240
:105760004A026CC08091B900909148028034C1F027
:10577000E92FFF27EE0FFF1FEE0FFF1FEA54FA4F2E
:1057800081818F778183892F8F5F809348028C304E
:1057900010F0109248020E94EC2A10924A020DC0AA
:1057A000E92FFF27EE0FFF1FEE0FFF1FEA54FA4FFE
:1057B0008181806881830E941B2B80914B028093A2
:1057C000470210924B0252C080914802E82FFF27F7
:1057D000EE0FFF1FEE0FFF1FEA54FA4F8091BB0040
:1057E00082830E941F2B42C090914802E92FFF271D
:1057F000EE0FFF1FEE0FFF1FEA54FA4F8091BB0020
:105800008383892F8F5F809348028C3010F0109231
:1058100048020E94EC2A28C080E11BC080911A0136
:1058200018C082E116C08091190113C00E94EC2AB1
:105830008AE090E09093A00180939F010E94E82A63
:1058400015C088E906C084E104C08091180101C038
:1058500080E80E94F02A0AC00E94EC2A8AE090E0C8
:105860009093A00180939F0110924A028091BC0006
:1058700080688093BC00FF91EF91BF91AF919F91A1
:105880008F917F916F915F914F913F912F910F90E9
:105890000FBE0F901F90189589E1ABE1B6E0E7EEDF
:1058A000F5E011821082329611961C921E92129689
:1058B000815087FFF6CF1092E4021092E30210921B
:1058C000E6021092E5021092E8021092E7020895B3
:1058D0001F920F920FB60F9211240F931F932F93C5
:1058E0003F934F935F936F937F938F939F93AF9368
:1058F000BF93CF93DF93EF93FF9340918600509136
:10590000870080914D0290914E02481B590BCA01AD
:1059100057FD0196AC015595479580918600909171
:10592000870090934E0280934D02CA018959984096
:10593000A0914F02B0915002875E954338F41497BE
:1059400014F01092780181E090E081C0AD30B10593
:105950000CF081C0CA018B5F90408356944008F0E0
:1059600071C0425C5340FD01EA0FFB1FE951FA4F41
:1059700080819181FA01E81BF90BCF01F7FF03C089
:10598000909581959F4F06974CF480918302883CB7
:1059900028F480918302865F80938302FD01EA0FE1
:1059A000FB1FE951FA4F808191819C01220F331F27
:1059B000280F391F240F351F37FF02C02D5F3F4FBF
:1059C000E901D595C795D595C795CA0101968C175C
:1059D0009D0714F4219706C041505040C417D507C5
:1059E0000CF4219680918302833CD8F08D010A0F3C
:1059F0001B1FF801E951FA4F808191819E01281BFC
:105A0000390BC90163E070E00E947B6ECB01880F07
:105A1000991F860F971F055E194FF80191838083A8
:105A200007C0AA0FBB1FA55EB94F11961C921E920C
:105A3000E0914F02F0915002EE0FFF1FE951FA4F33
:105A4000D183C08380914F02909150020196909330
:105A5000500280934F02FF91EF91DF91CF91BF9160
:105A6000AF919F918F917F916F915F914F913F91F6
:105A70002F911F910F910F900FBE0F901F901895AF
:105A800081E08093580682E08093570683E08093FC
:105A9000560684E08093590685E080935A0686E096
:105AA00080935B0687E080935C0688E080935D06C8
:105AB00089E080935E068AE080935F068BE08093A6
:105AC00060068CE08093610608951F938AE68093B8
:105AD000620661E06093B5065EE1509363068FEF66
:105AE000809365068AE0809366065093640650931F
:105AF000680685E08093690680E480936A061092C8
:105B00006B0684E1809367068EE080936C06F0E17B
:105B1000F0936D061CE010936E06A8E0A0936F064C
:105B200086EE809370065093710680E8809372062B
:105B300040E54093730696E99093740683E0809362
:105B40007506409376069093770681E280937806F7
:105B500083E28093790650937A0670E270937C0614
:105B600010927D0610927E0610927F06109280069B
:105B7000109298061092990610929A0610929B061F
:105B800024E62093810638E2309382066093B406BF
:105B90001092830697EF90938406E6E0E0938906DF
:105BA0008DE780938A0680938B0680938C062093E2
:105BB000850630938606109287069093880682E3C6
:105BC00080938D069AE590938E0680938F061092AF
:105BD000B30690939006409391066093920685E5F4
:105BE0008093930680939406F0939506709396069F
:105BF000209397068FE580939C0683EF80939E0603
:105C00008AEA8093A0068093A1068FE080939D0688
:105C100080939F068EEF8093A2062093A306909315
:105C2000A4069093A5069093A6068BE48093A706FE
:105C30008093A8068093A9061092AA06E093AB066B
:105C4000A093AC069093AD065093AE062093AF069A
:105C50002093B00684E08093B10660937B06A1EAAE
:105C6000B1E0E6EBF6E00D9001921A95E1F71F9195
:105C700008958AE680936206E1E0E093B5066EE15E
:105C8000609363068FEF809365069AE090936606B3
:105C9000609364066093680685E08093690680E4FB
:105CA00080936A0610926B068FE08093670690934C
:105CB0006C0680E180936D0676E070936E06F8E0E6
:105CC000F0936F0686EE809370066093710680E80D
:105CD000809372062AE52093730698E790937406E2
:105CE00083E080937506209376069093770681E291
:105CF0008093780683E28093790660937A0650E277
:105D000050937C0610927D0610927E0610927F06BC
:105D100010928006109298061092990610929A0698
:105D200010929B0644E64093810638E23093820647
:105D3000E093B4061092830697EF909384067093D5
:105D400089068DE780938A0680938B0680938C0664
:105D500040938506309386061092870690938806B6
:105D600082E380938D0620938E0680938F06109297
:105D7000B3062093900680E5809391068CE3809390
:105D8000920685E58093930680939406509395063A
:105D9000509396069BE4909397068FE580939C061C
:105DA00083EF80939E068AEA8093A0068093A106E3
:105DB00084E180939D0680939F068EEF8093A206D8
:105DC0004093A3062093A4062093A5062093A6063D
:105DD0009093A7069093A8069093A9061092AA06FE
:105DE0007093AB06F093AC062093AD066093AE06BD
:105DF0004093AF064093B00684E08093B106E093F1
:105E00007B068CE0A8EAB1E0E6EBF6E00D900192AB
:105E10008A95E1F708958AE68093620671E07093AF
:105E2000B5064EE1409363068FEF809365068AE0E6
:105E300080936606409364064093680685E08093ED
:105E4000690680E480936A0610926B068FE0809367
:105E5000670668E060936C0620E120936D0656E0CB
:105E600050936E0660936F0686EE809370064093A3
:105E7000710680E88093720634E63093730698E7E3
:105E80009093740683E08093750630937606909322
:105E9000770681E28093780683E28093790684E135
:105EA00080937A0620937C0610927D0610927E06DF
:105EB00010927F0610928006109298061092990612
:105EC00010929A0610929B063093810628E2209346
:105ED00082067093B4061092830697EF909384061F
:105EE000509389068DE780938A0680938B06809372
:105EF0008C06309385062093860610928706909331
:105F0000880692E390938D062AE520938E0690935F
:105F10008F061092B3062093900680E58093910639
:105F200086E48093920685E5809393068093940699
:105F300080E28093950680939606909397068FE56E
:105F400080939C0683EF80939E068AEA8093A00646
:105F50008093A10640939D0640939F068EEF809309
:105F6000A2063093A3062093A4062093A5062093AF
:105F7000A6068BE48093A7068093A8068093A906C3
:105F80001092AA065093AB066093AC062093AD0620
:105F90004093AE063093AF063093B00684E0809312
:105FA000B10670937B068CE0A0EBB1E0E6EBF6E087
:105FB0000D9001928A95E1F708956817790754F4D6
:105FC000680F791F77FF02C06F5F7F4FCB019595F8
:105FD00087950895681B790B861B970B08951F936F
:105FE000CF93DF93182FEB01809179028823A1F4DE
:105FF00011501F3F89F0D093FF01C093FE018091A3
:10600000FE019091FF01892BD1F7CE018C0F9D1FCE
:106010000E940517115078F7DF91CF911F910895D5
:10602000A3E1B0E0E6E1F0E30C94CB6E8091E302F3
:106030009091E4022091210230912202821B930B65
:10604000909317078093160780912B0290912C0252
:1060500097FD07969C0153E0359527955A95E1F7F2
:106060003093D4062093D3068091290290912A027E
:1060700097FD079643E0959587954A95E1F79093AC
:10608000C5068093C4063093E1062093E006909302
:10609000D7068093D6068091110790911207AA2700
:1060A00097FDA095BA2F7C018D01EE0CFF1C001FFF
:1060B000111FE80EF91E0A1F1B1F80911D029091EF
:1060C0001E029C01442737FD4095542FDA01C90177
:1060D000F2E0880F991FAA1FBB1FFA95D1F7820F14
:1060E000931FA41FB51F820F931FA41FB51FE80E97
:1060F000F91E0A1F1B1F17FF08C023E030E040E015
:1061000050E0E20EF31E041F151FE2E015950795FF
:10611000F794E794EA95D1F7F0921207E09211070D
:106120008091210790912207AA2797FDA095BA2F69
:106130007C018D01EE0CFF1C001F111FE80EF91EE3
:106140000A1F1B1F80911F02909120029C0144276F
:1061500037FD4095542FDA01C90162E0880F991F7D
:10616000AA1FBB1F6A95D1F7820F931FA41FB51FEB
:10617000820F931FA41FB51FE80EF91E0A1F1B1FD5
:1061800017FF08C083E090E0A0E0B0E0E80EF91E41
:106190000A1F1B1F82E015950795F794E7948A95CF
:1061A000D1F7F0922207E09221078091DE069091CC
:1061B000DF06AA2797FDA095BA2F9C01AD01220FFB
:1061C000331F441F551F280F391F4A1F5B1F809123
:1061D0001B0290911C02AA2797FDA095BA2F280FA9
:1061E000391F4A1F5B1F57FF04C02D5F3F4F4F4FA2
:1061F0005F4FF2E05595479537952795FA95D1F77A
:106200003093DF062093DE0620911D0230911E029E
:10621000C901880F991F880F991F820F931F820F42
:10622000931F9C01442737FD4095542F8091BF0256
:106230009091C002A091C102B091C202820F931F3F
:10624000A41FB51F8093BF029093C002A093C10208
:10625000B093C20220911F0230912002C901880F21
:10626000991F880F991F820F931F820F931F9C0104
:10627000442737FD4095542F8091BB029091BC027A
:10628000A091BD02B091BE02820F931FA41FB51F43
:106290008093BB029093BC02A093BD02B093BE0258
:1062A0008091EA069091EB0620911D0230911E022A
:1062B000820F931F9093EB068093EA068091190753
:1062C00090911A0720911F0230912002820F931F94
:1062D00090931A07809319078091D9029091DA025E
:1062E00001969093DA028093D9028091B70290913F
:1062F000B802A091B902B091BA02BC01CD010E94CE
:10630000C26D5B016C018091A9059091AA05AA2735
:1063100097FDA095BA2FBC01CD010E94C26D7B01F3
:106320008C018091D5029091D602A091D702B091B4
:10633000D8029C01AD01C801B7010E94626DDC0169
:10634000CB019C01AD01C601B5010E94636DDC016A
:10635000CB01BC01CD010E94A56DDC01CB01809376
:10636000B7029093B802A093B902B093BA028FEC2F
:1063700080937A00109217012091A7023091A80211
:106380004091A9025091AA0229873A874B875C87DE
:1063900029543B46414050402CF028E43BE641E084
:1063A00050E00DC089859A85AB85BC85885B944992
:1063B000AE4FBF4F4CF428EB34E94EEF5FEF2D8327
:1063C0003E834F83588708C089859A85AB85BC85F5
:1063D0008D839E83AF83B8872091AF023091B00246
:1063E0004091B1025091B2022D873E874F87588B62
:1063F00029543B46414050402CF028E43BE641E024
:1064000050E00DC08D859E85AF85B889885B944925
:10641000AE4FBF4F4CF428EB34E94EEF5FEF2983CA
:106420003A834B835C8308C08D859E85AF85B88990
:1064300089839A83AB83BC83A0911607B091170719
:10644000BA8BA98BFD01CF01AA2797FDA095BA2F82
:10645000A0909F02B090A002C090A102D090A20292
:10646000A80EB91ECA1EDB1EA0929F02B092A00207
:10647000C092A102D092A202E0901D07F0901E07E8
:1064800000911F0710912007E80EF91E0A1F1B1F1D
:10649000E0921D07F0921E0700931F07109320073C
:1064A000F0916C02FB8BFF2309F098C180916B0285
:1064B000882309F093C18091620686FF8FC1809185
:1064C000C4069091C506AA2797FDA095BA2FBC01D6
:1064D000CD0129813A814B815C810E943C6E9B01F8
:1064E000AC0197FF04C02150384F4F4F5F4F6BE016
:1064F00055954795379527956A95D1F780918101F4
:10650000682E772488249924CA01B901A401930133
:106510000E943C6EDC01CB018093F3029093F40265
:10652000A093F502B093F602B7FF04C08150904FDC
:10653000AF4FBF4F1C012D013CE055944794379459
:1065400027943A95D1F72092F3023092F4024092C8
:10655000F5025092F6028091D3069091D406AA27B4
:1065600097FDA095BA2FBC01CD012D813E814F81B1
:1065700058850E943C6E97FF04C06150784F8F4F42
:106580009F4F2BE095958795779567952A95D1F73D
:10659000A40193010E943C6EDC01CB018093F702C1
:1065A0009093F802A093F902B093FA02B7FF04C0E7
:1065B0008150904FAF4FBF4F9C01AD018CE055957E
:1065C0004795379527958A95D1F72093F702309311
:1065D000F8024093F9025093FA028091F3029091ED
:1065E000F4029093500680934F068091F7029091A9
:1065F000F8029093540680935306221933094409F4
:1066000055092093F7023093F8024093F902509312
:10661000FA02E20EF31E041F151FE0921D07F0920E
:106620001E0700931F071093200780918001882385
:10663000B1F457FF04C02F5F3F4F4F4F5F4F559549
:10664000479537952795A21AB30AC40AD50AA0928E
:106650009F02B092A002C092A102D092A202298908
:106660003A8979010027F7FC0095102F8091F702F5
:106670009091F802A091F902B091FA02E80EF91E89
:106680000A1F1B1FC801B70129813A814B815C8118
:106690000E943C6E9B01AC0197FF04C02150384F13
:1066A0004F4F5F4FBBE05595479537952795BA9566
:1066B000D1F780918201A82EBB24CC24DD24CA010D
:1066C000B901A60195010E943C6EDC01CB018093CB
:1066D000EB029093EC02A093ED02B093EE02B7FFB1
:1066E00004C08150904FAF4FBF4F3C014D01ACE013
:1066F0009594879477946794AA95D1F76092EB026A
:106700007092EC028092ED029092EE02C801B70105
:106710002D813E814F8158850E943C6E97FF04C0B9
:106720006150784F8F4F9F4FFBE0959587957795F8
:106730006795FA95D1F7A60195010E943C6EDC01A0
:10674000CB018093EF029093F002A093F102B093FB
:10675000F202B7FF04C08150904FAF4FBF4FAC0162
:10676000BD01ECE07595679557954795EA95D1F78A
:106770004093EF025093F0026093F1027093F202A3
:1067800029893A8937FF03C0309521953F4F21343D
:106790003105E4F1D401C30197FE07C0B095A0957F
:1067A000909581959F4FAF4FBF4F81389105A105BF
:1067B000B10584F4DB01CA0177FF07C0B095A0954D
:1067C000909581959F4FAF4FBF4F81389105A1059F
:1067D000B105E4F081E080938F0218C01092540656
:1067E000109253061092500610924F061092EF022C
:1067F0001092F0021092F1021092F2021092EB024B
:106800001092EC021092ED021092EE028091EF02D3
:106810009091F002A091F102B091F202BC01CD0181
:1068200024E630E040E050E00E94B06EE090EB02E1
:10683000F090EC02E21AF30AF092D206E092D1064E
:106840008091EB029091EC02A091ED02B091EE02EA
:10685000BC01CD0124E630E040E050E00E94B06E83
:10686000DA01C9012091EF023091F0028C01021B84
:10687000130B1093C7060093C6068091790190917F
:106880007A01A0917B01B0917C01BC01CD0128E689
:1068900031E040E050E00E943C6E20911D073091B5
:1068A0001E0740911F0750912007261737074807FA
:1068B000590764F0261B370B480B590B20931D0713
:1068C00030931E0740931F075093200720911D0708
:1068D00030911E0740911F075091200757FF0CC0B1
:1068E000260F371F481F591F20931D0730931E077F
:1068F00040931F07509320076091C4067091C5060E
:106900006E0D7F1D9B01442737FD4095542F8091CC
:10691000A3029091A402A091A502B091A602820FB9
:10692000931FA41FB51F8093A3029093A402A0936A
:10693000A502B093A60280916F0290917002681B2D
:10694000790BCB01AA2797FDA095BA2F29853A8507
:106950004B855C85820F931FA41FB51F8093A702F0
:106960009093A802A093A902B093AA02C0909501A7
:10697000D0909601E0909701F0909801C816D90642
:10698000EA06FB06C4F488EA91E6A0E0B0E08C19C0
:106990009D09AE09BF098093A7029093A802A09316
:1069A000A902B093AA028093A3029093A402A09399
:1069B000A502B093A60222273327A9012C193D096D
:1069C0004E095F098091A7029091A802A091A902A7
:1069D000B091AA0282179307A407B507B4F4D701B0
:1069E000C601885A9146A040B0408093A702909378
:1069F000A802A093A902B093AA028093A302909345
:106A0000A402A093A502B093A6026091D306709150
:106A1000D406600F711F9B01442737FD4095542F0A
:106A20008091AB029091AC02A091AD02B091AE0208
:106A3000820F931FA41FB51F8093AB029093AC02EB
:106A4000A093AD02B093AE0280916D0290916E0260
:106A5000681B790BCB01AA2797FDA095BA2F2D852E
:106A60003E854F855889820F931FA41FB51F8093C1
:106A7000AF029093B002A093B102B093B202E09043
:106A80009901F0909A0100919B0110919C01E816E8
:106A9000F9060A071B07C4F488EA91E6A0E0B0E013
:106AA0008E199F09A00BB10B8093AF029093B00297
:106AB000A093B102B093B2028093AB029093AC0268
:106AC000A093AD02B093AE0222273327A9012E195D
:106AD0003F09400B510B8091AF029091B002A09101
:106AE000B102B091B20282179307A407B507B4F4BC
:106AF000D801C701885A9146A040B0408093AF02A8
:106B00009093B002A093B102B093B2028093AB0213
:106B10009093AC02A093AD02B093AE0280919F021D
:106B20009091A002A091A102B091A2028093B30221
:106B30009093B402A093B502B093B6028091AF02D5
:106B40009091B002A091B102B091B2028093CF02B5
:106B50009093D002A093D102B093D2028091A70269
:106B60009091A802A091A902B091AA028093C702B5
:106B70009093C802A093C902B093CA028091AB025D
:106B80009091AC02A091AD02B091AE028093CB0285
:106B90009093CC02A093CD02B093CE028091A30239
:106BA0009091A402A091A502B091A6028093C30285
:106BB0009093C402A093C502B093C60280912301B2
:106BC0009091240197FD079633E0959587953A9526
:106BD000E1F79093D4068093D306809121019091A0
:106BE000220197FD079623E0959587952A95E1F771
:106BF0009093C5068093C406809125029091260249
:106C00000F9734F488E19CEF9093D4068093D306D9
:106C10008091250290912602079734F480E398EF43
:106C20009093D4068093D306209102012A30A9F4D0
:106C30008091250290912602835F934034F088EE84
:106C400093E09093D4068093D3068091250290918F
:106C500026028A5F9340DCF014C080912502909157
:106C60002602815D974034F088EE93E09093D4063D
:106C70008093D3068091250290912602805E9740F2
:106C800034F080ED97E09093D4068093D306809102
:106C90002302909124020F9734F488E19CEF9093A3
:106CA000C5068093C4068091230290912402079721
:106CB00034F480E398EF9093C5068093C4062A309D
:106CC000A9F48091230290912402835F934034F0D1
:106CD00088EE93E09093C5068093C40680912302CA
:106CE000909124028A5F9340DCF014C080912302CB
:106CF00090912402815D974034F088EE93E0909368
:106D0000C5068093C4068091230290912402805E80
:106D1000974034F080ED97E09093C5068093C406C9
:106D2000E0918C01EE2309F4B7C04091230150910A
:106D300024018091FB029091FC02481B590B509357
:106D40000203409301032091230130912401280F75
:106D5000391F37FF02C02F5F3F4F3595279530937E
:106D6000FC022093FB02413851051CF080E890E0C2
:106D700005C040585F4F34F480E89FEF90930203C2
:106D8000809301038E2F9927A0910103B0910203F4
:106D9000A89FA001A99F500DB89F500D112457FF27
:106DA00002C0415F5F4F84E0559547958A95E1F7B2
:106DB0008091D3069091D406840F951F9093D406AA
:106DC0008093D30660912101709122018091FD0290
:106DD0009091FE02681B790B709300036093FF0291
:106DE0004091210150912201480F591F57FF02C0C5
:106DF0004F5F5F4F559547955093FE024093FD02BC
:106E0000613871051CF080E890E005C060587F4F44
:106E100034F480E89FEF909300038093FF022E2FBD
:106E200033278091FF0290910003829FB001839FDE
:106E3000700D929F700D1124AB0177FF02C0415F6E
:106E40005F4F14E0559547951A95E1F78091C40678
:106E50009091C506840F951F9093C5068093C40634
:106E6000A29FC001A39F900DB29F900D11249C0181
:106E70008091230190912401820F931F909324010C
:106E8000809323018091210190912201860F971F09
:106E900090932201809321010091D6061091D7068C
:106EA00080914F0690915006101611065CF59C01DA
:106EB00097FF04C022273327281B390BC901AA27B3
:106EC00097FDA095BA2F209180013327442755279D
:106ED000BC01CD010E943C6E9B01AC0197FF04C038
:106EE000215C3F4F4F4F5F4FF6E0559547953795E3
:106EF0002795FA95D1F78091D1069091D206820F0D
:106F0000931F27C097FF03C0909581959F4FAA2795
:106F100097FDA095BA2F209180013327442755274C
:106F2000BC01CD010E943C6E9B01AC0197FF04C0E7
:106F3000215C3F4F4F4F5F4FE6E0559547953795A2
:106F40002795EA95D1F78091D1069091D206821BC0
:106F5000930B9093D2068093D106E090E006F090D8
:106F6000E10680915306909154061E141F045CF5AF
:106F70009C0197FF04C022273327281B390BC90126
:106F8000AA2797FDA095BA2F209180013327442787
:106F90005527BC01CD010E943C6E9B01AC0197FFBF
:106FA00004C0215C3F4F4F4F5F4F76E055954795AA
:106FB000379527957A95D1F78091C6069091C706A7
:106FC000820F931F27C097FF03C0909581959F4F15
:106FD000AA2797FDA095BA2F209180013327442737
:106FE0005527BC01CD010E943C6E9B01AC0197FF6F
:106FF00004C0215C3F4F4F4F5F4F66E0559547956A
:10700000379527956A95D1F78091C6069091C70666
:10701000821B930B9093C7068093C60680916206ED
:1070200087FF44C09B89992309F040C080916B027F
:107030008823E1F5A1E0EA16A1E0FA064CF0809180
:10704000D3069091D4068E0D9F1D805091400DC0A7
:10705000B0E0EB16BFEFFB0664F48091D30690918D
:10706000D4068E0D9F1D80509F4F9093D406809321
:10707000D306E1E001301E074CF08091C4069091E8
:10708000C506800F911F805091400CC0FFEF00306B
:107090001F0764F48091C4069091C506800F911F6C
:1070A00080509F4F9093C5068093C406A4E8B2E039
:1070B0006AE576E057E0FB018191BF01E82FFF27E9
:1070C000EE0FFF1FE951FA4F0190F081E02DE259D8
:1070D000FF4FEF3FF10521F01CF0EFEFF0E004C0AF
:1070E000F7FF02C0E0E0F0E04C91242F3327E217D5
:1070F000F307B1F0CF01821B930B97FD079633E0A6
:10710000959587953A95E1F7242F280F2C93822F98
:107110009927E817F90714F4215001C02F5F2C9329
:107120005150119657FFC7CFE2E1CD5E0C94E76E48
:10713000CF93DF93809102018D3011F40E948F1B59
:1071400010927A0080912502909126029093D406A5
:107150008093D30680912302909124029093C506D8
:107160008093C40680912102909122029093170788
:107170008093160780911D0290911E029C01442766
:1071800037FD4095542FDA01C90172E0880F991F2D
:10719000AA1FBB1F7A95D1F7820F931FA41FB51F9B
:1071A000820F931FA41FB51F90931207809311079E
:1071B00080911F02909120029C01442737FD409549
:1071C000542FDA01C90162E0880F991FAA1FBB1F63
:1071D0006A95D1F7820F931FA41FB51F820F931FCB
:1071E000A41FB51F909322078093210780911B0253
:1071F00090911C029093DF068093DE068FEC8093C3
:107200007A00A4E8B2E0CAE5D6E097E08991E82FD9
:10721000FF27EE0FFF1FE951FA4F0190F081E02D9B
:10722000E259FF4F1E161F061CF0E0E0F0E005C01B
:10723000EF3FF10514F0EFEFF0E08C91282F3327AA
:10724000E217F30714F4815004C02E173F0714F41B
:107250008F5F8C939150119697FFD8CF80919306B2
:107260009927AA27BB27BC01CD0124EC39E040E0D7
:1072700050E00E943C6EDC01CB0180939901909319
:107280009A01A0939B01B0939C0180919406992749
:10729000AA27BB27BC01CD010E943C6EDC01CB01BB
:1072A0008093950190939601A0939701B0939801D4
:1072B000DF91CF910895A0E0B0E0E1E6F9E30C940E
:1072C000CF6EC0E0D0E07E016E01469AD093DE0220
:1072D000C093DD02D093DC02C093DB0280E090E03B
:1072E000A0E0B0E08093D5029093D602A093D7029D
:1072F000B093D802D093E802C093E702D093E6029D
:10730000C093E502D093E402C093E302D093F20667
:10731000C093F10610928201109281011092150221
:107320000E94983884E690E00E9412170E949838D4
:107330008091620680FF10C080911B0190911C011A
:10734000875B934038F480911B0190911C018E5E05
:10735000924010F40E943E1B1FE18AE090E00E94E0
:1073600012178091210290912202C80FD91F80919B
:10737000250290912602E80EF91E80912302909139
:107380002402C80ED91E115017FFE7CFA701405F96
:107390005F4F56954795569547955093E802409311
:1073A000E7029601205F3F4F369527953695279542
:1073B0003093E6022093E502CE01409615E09695C3
:1073C00087951A95E1F79093E4028093E3029093F6
:1073D000F2068093F1063093E2022093E10250938B
:1073E000E0024093DF0244E050E0DA010E94086FBF
:1073F000802D853038F1809121079091220797FFE9
:1074000003C0909581959F4F6CE070E00E947B6E69
:107410007093DC026093DB02809111079091120758
:1074200097FF03C0909581959F4F6CE070E00E949C
:107430007B6E7093DE026093DD028091A9059091CE
:10744000AA0534C0DA010E94086F802D9927982F71
:107450008827DA0111960E94086F202D820F911D56
:107460009093DE028093DD02DA0112960E94086F8B
:10747000802D9927982F8827DA0113960E94086F8C
:10748000202D820F911D9093DC028093DB02DA01A4
:1074900014960E94086F802D9927982F8827DA016B
:1074A00015960E94086F202D820F911DAA2797FD27
:1074B000A095BA2FBC01CD010E94C26DDC01CB01A9
:1074C0008093D5029093D602A093D702B093D802AE
:1074D0001092D4061092D3061092C5061092C406DC
:1074E000109217071092160784E690E00E94121778
:1074F00080911D0290911E02AA2797FDA095BA2F98
:107500009C01AD01F2E0220F331F441F551FFA9575
:10751000D1F7280F391F4A1F5B1F280F391F4A1F39
:107520005B1F309312072093110780911F029091E7
:107530002002AA2797FDA095BA2F7C018D01E2E0D9
:10754000EE0CFF1C001F111FEA95D1F7E80EF91E83
:107550000A1F1B1FE80EF91E0A1F1B1FF0922207AD
:10756000E092210780917106682E7724882499245F
:10757000C9019C01442737FD4095542FC401B30134
:107580000E943C6E5B016C016093CF027093D0024D
:107590008093D1029093D2029701442737FD409502
:1075A000542FC401B3010E943C6EDC01CB018093D7
:1075B000C7029093C802A093C902B093CA02A092D6
:1075C000AB02B092AC02C092AD02D092AE028093F8
:1075D000A3029093A402A093A502B093A6021092D6
:1075E0009F021092A0021092A1021092A20280911A
:1075F0001D0190911E01A0911F01B0912001909357
:10760000AC058093AB0510921402109213021092F5
:107610009702109298021092990210929A02809109
:1076200095029091960290939402809393020E9407
:10763000355A82E390E09093FF018093FE018091A0
:1076400093069927AA27BB27BC01CD0124EC39E07A
:1076500040E050E00E943C6EDC01CB018856954C26
:10766000AF4FBF4F8093990190939A01A0939B01D4
:10767000B0939C01809194069927AA27BB27BC014F
:10768000CD010E943C6EDC01CB018856954CAF4F7A
:10769000BF4F8093950190939601A0939701B0936B
:1076A000980110927E0110927D0180919502909137
:1076B0009602AA2797FDA095BA2F209179013091C3
:1076C0007A0140917B0150917C01BC01CD010E9467
:1076D0003C6EDC01CB0180931D0790931E07A093A5
:1076E0001F07B093200710928E0210928D0281E046
:1076F000809301010E94545E8091520284608093C5
:1077000052028FEF80938E0710928F0780E2809352
:107710009007C4E8D2E0AAE5B6E017E08D91E82F23
:10772000FF27EE0FFF1FE951FA4F808191818259A7
:107730008993115017FFF2CF84E6809383028091E2
:10774000FC01882311F0469A579AEEE0CDB7DEB7D8
:107750000C94EB6E809179028823F9F480915202A7
:107760008C7F80935202A6EBB5E0EDEFF3E09BE057
:107770008091DF01882309F4808381918C93149692
:10778000915097FFF5CF8091DF01882359F08091C8
:10779000DF0181508093DF0105C08091520281603A
:1077A000809352028091B605992790937F0580932C
:1077B0007E058091BA059927909381058093800575
:1077C0008091BE05992790938305809382058091CF
:1077D000C2059927909385058093840510924A02EB
:1077E000109249020E94E82A089580916406883F19
:1077F00038F0EFEFF0E0E81BF109EC57FD4F808126
:107800008093920180919201882329F0843618F0A8
:1078100084E68093920180916606883F38F0EFEF0E
:10782000F0E0E81BF109EC57FD4F80818093900157
:1078300080919001882329F0843618F084E68093A3
:10784000900180917306883F38F0EFEFF0E0E81B7D
:10785000F109EC57FD4F808180938B0180918B0162
:107860008B3010F48AE002C08F3F11F480938B01BB
:1078700080919D06883F38F0EFEFF0E0E81BF109BA
:10788000EC57FD4F80818093EC068091EC068230AE
:1078900010F481E002C08F3F11F48093EC068091D8
:1078A0009F06883F38F0EFEFF0E0E81BF109EC5756
:1078B000FD4F80818093140780911407823010F46B
:1078C00081E002C08F3F11F48093140780918A06F3
:1078D000883F38F0EFEFF0E0E81BF109EC57FD4F7F
:1078E00080818093E90680918B06883F38F0EFEF26
:1078F000F0E0E81BF109EC57FD4F808180935506BD
:1079000080918C06883F38F0EFEFF0E0E81BF1093A
:10791000EC57FD4F80818093F30690916506983F68
:1079200018F49093910109C0EFEFF0E0E91BF10921
:10793000EC57FD4F808180939101983F18F490930C
:10794000910109C0EFEFF0E0E91BF109EC57FD4FA1
:1079500080818093910180916806883F38F0EFEF35
:10796000F0E0E81BF109EC57FD4F808180938F0117
:1079700080916A06883F38F0EFEFF0E0E81BF109EC
:10798000EC57FD4F808180938D0180917206883F76
:1079900038F0EFEFF0E0E81BF109EC57FD4F808184
:1079A00080938E0180917406883F38F0EFEFF0E00D
:1079B000E81BF109EC57FD4F808180938A0180918B
:1079C0007506883F38F0EFEFF0E0E81BF109EC575F
:1079D000FD4F808180938C0180917606883F38F03E
:1079E000EFEFF0E0E81BF109EC57FD4F8081809349
:1079F000890180917706883F38F0EFEFF0E0E81BCF
:107A0000F109EC57FD4F80818093880180917C06BD
:107A1000883F38F0EFEFF0E0E81BF109EC57FD4F3D
:107A200080818093860180917D06883F38F0EFEF5A
:107A3000F0E0E81BF109EC57FD4F8081809366026E
:107A400080917E06883F38F0EFEFF0E0E81BF10907
:107A5000EC57FD4F80818093650280917F06883FBF
:107A600038F0EFEFF0E0E81BF109EC57FD4F8081B3
:107A70008093640280918006883F38F0EFEFF0E059
:107A8000E81BF109EC57FD4F8081809363028091E0
:107A90009806883F38F0EFEFF0E0E81BF109EC576B
:107AA000FD4F80818093620280919906883F38F073
:107AB000EFEFF0E0E81BF109EC57FD4F8081809378
:107AC000610280919A06883F38F0EFEFF0E0E81B02
:107AD000F109EC57FD4F80818093600280919B06F5
:107AE000883F38F0EFEFF0E0E81BF109EC57FD4F6D
:107AF000808180935F0280918106883F38F0EFEFAC
:107B0000F0E0E81BF109EC57FD4F8081809385017F
:107B100080918506883F38F0EFEFF0E0E81BF1092F
:107B2000EC57FD4F80818093840180918D06883FC2
:107B300038F0EFEFF0E0E81BF109EC57FD4F8081E2
:107B40008093830180919006883F38F0EFEFF0E05A
:107B5000E81BF109EC57FD4F8081809382018091F1
:107B60009106883F38F0EFEFF0E0E81BF109EC57A1
:107B7000FD4F80818093810180919206883F38F08B
:107B8000EFEFF0E0E81BF109EC57FD4F80818093A7
:107B9000800180919706883F38F0EFEFF0E0E81B16
:107BA000F109EC57FD4F808180937F018091B206EF
:107BB000883F38F0EFEFF0E0E81BF109EC57FD4F9C
:107BC00080818093240780918601282F33272F5F9F
:107BD0003F4F8CE398E2B9010E947B6E7093940151
:107BE00060939301809170068093150780916F06D2
:107BF0008093D8060895A4E1B0E0E1E0FEE30C94A0
:107C0000CB6E80915102815080935102882319F4E8
:107C100085E0809351020E941030309102013C3087
:107C200010F4299A01C02998E0907A02F0907B0222
:107C3000FA82E9828091D80699270A96E816F90611
:107C400014F49A83898380918302843608F05CC09F
:107C500080911F0390912003009731F0019790933A
:107C6000200380931F0307C0109279028091520273
:107C70008F7E809352023A3011F0343111F4289AF9
:107C800001C028988091530290915402895E9340DC
:107C9000C0F180917906282F33273A832983809178
:107CA000520280618093520280915606A82FBB2712
:107CB000AA0FBB1FFD01E55EF94F11821082809172
:107CC0005706282F3327220F331FC901855E994F8E
:107CD000FC0111821082A951BA4F11961C921E927A
:107CE00029513A4FD90111961C921E928091590642
:107CF000E82FFF27EE0FFF1FE951FA4F1182108284
:107D0000E8C210927902E5C2809183028D3808F4AE
:107D1000E0C2809152028F7E8093520290917A0647
:107D200082E3989FC00111249093200380931F0346
:107D3000E981FA81B9978CF080917902882369F002
:107D40008091530290915402FFEF8F3F9F0729F0DB
:107D50000196909354028093530280915302909124
:107D600054028F3F910509F038F5109203031092E9
:107D70000403109205031092060310920703109259
:107D800008031092090310920A038A3F9105C9F46F
:107D900081E08093250310920B0310920C03109244
:107DA0000D0310920E0310929F021092A0021092E7
:107DB000A1021092A20205C08091520282608093BB
:107DC000520280915806E82FFF27EE0FFF1FE9515E
:107DD000FA4F80819181813591050CF4A6C12091E3
:107DE0007902222309F0A1C180915906E82FFF27CB
:107DF000EE0FFF1FE951FA4F808191818C3491057C
:107E00000CF404C1809121038F5F80932103893C8E
:107E100008F48BC13C3010F4299801C0299A1092C3
:107E20007902109221031092540210925302309161
:107E30005606E32FFF27EE0FFF1FE951FA4F80810F
:107E4000918187349105B4F480915706E82FFF277C
:107E5000EE0FFF1FE951FA4F808191810190F0816F
:107E6000E02DF7FF03C0F095E195FF4FE734F105F2
:107E70000CF478C041E020915706A22FBB27AA0F2F
:107E8000BB1FA951BA4F8D919C91119787349105D1
:107E900044F0E32FFF27EE0FFF1FE951FA4F8081D7
:107EA00091818D919C918734910574F08091560653
:107EB000E82FFF27EE0FFF1FE951FA4F80819181D4
:107EC000873491050CF042E0E22FFF27EE0FFF1FF1
:107ED000E951FA4F808191818634910574F4809143
:107EE0005606E82FFF27EE0FFF1FE951FA4F80815A
:107EF0009181873491050CF043E0E22FFF27EE0FCC
:107F0000FF1FE951FA4F808191818A5B9F4F74F482
:107F100080915606E82FFF27EE0FFF1FE951FA4F19
:107F200080819181873491050CF044E0E22FFF2796
:107F3000EE0FFF1FE951FA4F808191818A5B9F4FBD
:107F400074F480915606E82FFF27EE0FFF1FE951CA
:107F5000FA4F80819181863491050CF445E0842F9D
:107F60000E94DA0680915706E82FFF27EE0FFF1FC9
:107F7000E951FA4F808191810190F081E02DF7FF66
:107F800003C0F095E195FF4F7E97BCF480915606B3
:107F9000E82FFF27EE0FFF1FE951FA4F80819181F3
:107FA0008A5B9F4F54F481E08093130488EE93E042
:107FB0009093FF018093FE01B8C00E9415074CE624
:107FC00066E576E00E94BD0680E00E945C070E94A4
:107FD000AD668091620680FF10C080911B01909178
:107FE0001C01875B934038F480911B0190911C0128
:107FF0008E5E924010F40E943E1B1092FC010E9483
:108000005B3981E08093FC01579A86C08081918121
:10801000855B9F4F0CF087C0809121038F5F809319
:108020002103893C08F481C03C3010F4299801C038
:10803000299AA4E0B0E08FEF082E0E94156F1092ED
:1080400079021092210310925402109253020E945E
:108050005B39A4E0B0E08091DD029091DE0297FFF1
:1080600002C081509F4F892F990F990B082E0E94B3
:10807000156FA5E0B0E08091DD029091DE02082E40
:108080000E94156FA6E0B0E08091DB029091DC02C7
:1080900097FF02C081509F4F892F990F990B082E8F
:1080A0000E94156FA7E0B0E08091DB029091DC02A6
:1080B000082E0E94156F08E010E08091D502909183
:1080C000D602A091D702B091D802BC01CD010E9486
:1080D000A56DDC01CB019C0197FF02C021503F4FF1
:1080E000832F992787FD9A95D801082E0E94156F36
:1080F00009E010E08091D5029091D602A091D702BC
:10810000B091D802BC01CD010E94A56DDC01CB016C
:10811000D801082E0E94156F0E94150768E770E0CD
:108120000E94EF2F02C02093210380915806E82F70
:10813000FF27EE0FFF1FE951FA4F808191818B5A83
:108140009F4F0CF0C6C020917902E091590622237E
:1081500009F0A3C0FF27EE0FFF1FE951FA4F8081FE
:108160009181855B9F4F0CF095C0809122038F5FBA
:1081700080932203893C08F4ACC02093220381E061
:1081800090E0909354028093530281E080937902AF
:1081900010920B0310920C0310920D0310920E0319
:1081A00010929F021092A0021092A1021092A202BD
:1081B00010929B0210929C0210929D0210929E02BD
:1081C00080917106E82EFF24002711278091110766
:1081D000909112079C01442737FD4095542FC80108
:1081E000B7010E943C6EDC01CB018093AF029093FB
:1081F000B002A093B102B093B20280912107909196
:1082000022079C01442737FD4095542FC801B70130
:108210000E943C6EDC01CB018093A7029093A802E0
:10822000A093A902B093AA028091CF029091D002AC
:10823000A091D102B091D2028093AB029093AC0294
:10824000A093AD02B093AE028091C7029091C80294
:10825000A091C902B091CA028093A3029093A40294
:10826000A093A502B093A6021092030310920403F8
:108270001092050310920603109207031092080350
:108280001092090310920A03809152028860809331
:1082900052021FC0209322031CC0FF27EE0FFF1FB6
:1082A000E951FA4F808191818C34910584F080915D
:1082B00023038F5F80932303893C58F01092790247
:1082C00010922303109254021092530202C0109293
:1082D0002303809178018150809378018091780107
:1082E0008F3F21F08091520284FFD5C20E94F53B5E
:1082F00080912E0390912F03AC01440F551F480F1E
:10830000591F00915606A02FBB27AA0FBB1FFD01C6
:10831000E951FA4FF0906C06CF2CDD2480819181D9
:108320008C9D90018D9D300D9C9D300D1124420F30
:10833000531F57FF02C04D5F5F4F559547955595A9
:108340004795A55EB94F80916D06682F77278D916F
:108350009C91869FD001879FB00D969FB00D1124F0
:108360004A0F5B1F50932F0340932E0380916503A8
:10837000909166032091610330916203820F931FF5
:10838000481B590B50938102409380028091300327
:1083900090913103AC01440F551F480F591F1091A4
:1083A0005706A12FBB27AA0FBB1FFD01E951FA4FAA
:1083B000808191818C9DF0018D9DF00D9C9DF00D33
:1083C00011244E0F5F1F57FF02C04D5F5F4F559541
:1083D000479555954795A55EB94F8D919C91869F80
:1083E0009001879F300D969F300D1124420F531F2F
:1083F0005093310340933003809163039091640361
:1084000020915F0330916003820F931F481B590B2B
:1084100050937F0240937E0280915906E82FFF27F8
:10842000EE0FFF1FE951FA4F808191819095819560
:108430009F4F90937D0280937C028330910514F0CE
:10844000029705C03FEF8E3F930734F40296909356
:108450007D0280937C0204C010927D0210927C0207
:1084600080915806E82FFF27EE0FFF1FE951FA4FC2
:10847000C080D18048E750E0C40ED51ED0927B0268
:10848000C0927A0280918B019927AA2797FDA09527
:10849000BA2FBC01CD010E94C26DDC01CB0120E0EE
:1084A00030E040E251E4BC01CD010E94636DDC018B
:1084B000CB01BC01CD010E94A56DDC01CB018093F5
:1084C0001B0780918A018093F40680918901992786
:1084D000AA2797FDA095BA2FBC01CD010E94C26DBD
:1084E000DC01CB0120E030E040E251E4BC01CD01F1
:1084F0000E94636DDC01CB01BC01CD010E94A56D22
:10850000DC01CB018093CB06809188018093E20649
:1085100080911F0480FF61C080912407813808F496
:108520005CC080911804992787FD90954F2D5527A1
:10853000849F9001859F300D949F300D1124809170
:10854000800290918102820F931F90938102809309
:10855000800280911904992787FD9095849F90014E
:10856000859F300D949F300D112480917E02909153
:108570007F02820F931F90937F0280937E028091EF
:108580001A04282F332727FD309580917C02909183
:108590007D02820F931F90937D0280937C028091D5
:1085A0001C04282F332727FD3095809167069927D3
:1085B000289FB001299F700D389F700D1124709372
:1085C0007E0160937D0180911B0499278C159D0588
:1085D00024F490937B0280937A0280917A029091A6
:1085E0007B0297FF04C010927B0210927A02809166
:1085F000620682FF02C01092F40640918002509100
:108600008102CA0157FD03969C0135952795359542
:10861000279537FF03C0309521953F4F8091570232
:108620009091580282179307B4F4CA0157FF03C010
:10863000909581959F4F97FD039695958795959574
:10864000879590935802809357028536910544F0A0
:1086500084E690E001C001979093580280935702FE
:1086600040917E0250917F02CA0157FD03969C0102
:10867000359527953595279537FF03C0309521957A
:108680003F4F809155029091560282179307B4F4A0
:10869000CA0157FF03C0909581959F4F97FD0396A0
:1086A0009595879595958795909356028093550259
:1086B0008536910544F084E690E001C001979093DF
:1086C0005602809355028091520284FF08C0109296
:1086D0005802109257021092560210925502E12F42
:1086E000FF27EE0FFF1FE951FA4F40918E06242F0E
:1086F0003327808191812817390744F48091B3068C
:1087000082FF04C081E080936A0213C0E12FFF273B
:10871000EE0FFF1FE951FA4F842F992720918F0602
:10872000821B9109208131812817390714F4109296
:108730006A0240915706E42FFF27EE0FFF1FE95111
:10874000FA4F50918E06852F992722273327281B11
:10875000390B808191818217930744F48091B3068D
:1087600083FF04C081E08093690216C08091690292
:10877000882391F0E42FFF27EE0FFF1FE951FA4FF6
:1087800080918F069927851B91092081318182175D
:10879000930714F410926902E02FFF27EE0FFF1FDA
:1087A000E951FA4F40918E06242F33278081918121
:1087B0002817390744F48091B30680FF04C081E094
:1087C0008093670217C080916702882399F0E02F99
:1087D000FF27EE0FFF1FE951FA4F842F99272091B1
:1087E0008F06821B9109208131812817390714F4E3
:1087F0001092670240915606E42FFF27EE0FFF1FED
:10880000E951FA4F50918E06852F99272227332759
:10881000281B390B808191818217930744F4809142
:10882000B30681FF04C081E08093680216C0809186
:108830006802882391F0E42FFF27EE0FFF1FE95114
:10884000FA4F80918F069927851B910920813181EC
:108850008217930714F41092680280916A028823A9
:1088600019F480916902811181E080936B028091FB
:108870006702882321F480916802882351F081E007
:1088800080936C0210926B0210926A02109269023D
:1088900002C080936C0280916B02882321F4809146
:1088A0006C02882369F080918D069927A981BA818D
:1088B0008A179B0714F49A83898381E080938F023F
:1088C0008091520284FF1AC010927D0210927C02A5
:1088D000109281021092800210927F0210927E020A
:1088E0009AE590931B0788E78093F4069093CB0654
:1088F0008093E20610926B0210926C028091E50662
:108900009091E606A091E706B091E8062091CF028B
:108910003091D0024091D1025091D202820F931F28
:10892000A41FB51F8093E5069093E606A093E70683
:10893000B093E8068091ED069091EE06A091EF06C7
:10894000B091F0062090C7023090C8024090C90252
:108950005090CA02820D931DA41DB51D8093ED0693
:108960009093EE06A093EF06B093F0068091DA069E
:108970009091DB06A091DC06B091DD06E090CB0281
:10898000F090CC020091CD021091CE02EB82FC82DD
:108990000D831E838E0D9F1DA01FB11F8093DA06CD
:1089A0009093DB06A093DC06B093DD068091CC06A5
:1089B0009091CD06A091CE06B091CF06E090C30273
:1089C000F090C4020091C5021091C602EF82F886B1
:1089D00009871A878E0D9F1DA01FB11F8093CC069B
:1089E0009093CD06A093CE06B093CF06F0906C0284
:1089F000FB86FF2029F480916B02882309F460C074
:108A00001092BF021092C0021092C1021092C202D4
:108A10001092BB021092BC021092BD021092BE02D4
:108A20001092E5061092E6061092E7061092E8060C
:108A30001092ED061092EE061092EF061092F006DC
:108A40001092DA061092DB061092DC061092DD0618
:108A50001092CC061092CD061092CE061092CF0640
:108A60008091AF029091B002A091B102B091B20298
:108A70008093AB029093AC02A093AD02B093AE0290
:108A80008091A7029091A802A091A902B091AA0298
:108A90008093A3029093A402A093A502B093A60290
:108AA000109212021092110210926E0210926D0238
:108AB0001092700210926F020B85002309F0F2C130
:108AC00080916B02882309F0EDC18091A9059091F6
:108AD000AA05815092402CF480917902882309F4F0
:108AE000E1C190908E07A09071066091110770917E
:108AF00012077C8B6B8B80912107909122079A8BB8
:108B0000898B9FEF991609F4D9C0BB24CC24DD24AE
:108B1000CA01B901A60195010E94B06E79018A01CE
:108B2000EB89FC89CF01AA2797FDA095BA2FE81AF7
:108B3000F90A0A0B1B0BC201B101A60195010E94A3
:108B4000B06E59016A0129893A89C901AA2797FD9E
:108B5000A095BA2FA81AB90ACA0ADB0A292C33240D
:108B600027FC3094432C532CC801B701A20191017A
:108B70000E943C6E97FF04C061507E4F8F4F9F4F05
:108B80003B014C0109E095948794779467940A958A
:108B9000D1F7C601B501A20191010E943C6E97FF79
:108BA00004C061507E4F8F4F9F4F5B016C0119E0F5
:108BB000D594C794B794A7941A95D1F7809157028A
:108BC00090915802813491053CF480915502909126
:108BD000560281349105D4F0D401C30197FE03C03D
:108BE0000196A11DB11D3C014D0195948794779488
:108BF0006794D601C501D7FE03C00196A11DB11D22
:108C00005C016D01D594C794B794A79480915906DF
:108C1000E82FFF27EE0FFF1FE951FA4F8081918166
:108C20000190F081E02DF7FF03C0F095E195FF4F33
:108C30007A97A4F0C401B30123E030E040E050E0B3
:108C40000E94B06E39014A01C601B50123E030E04F
:108C500040E050E00E94B06E59016A018091900797
:108C6000282F332727FD3095432F532F26153705FF
:108C70004805590514F439014A01992787FD909553
:108C8000909581959F4FAA2797FDA095BA2F6816BA
:108C900079068A069B0614F43C014D012A153B0512
:108CA0004C055D0514F459016A01A816B906CA06F7
:108CB000DB060CF0CFC05C016D01CCC0EA2CFF24B8
:108CC00000271127CA01B901A80197010E94B06EBF
:108CD00039014A014B895C89CA01AA2797FDA095F1
:108CE000BA2F681A790A8A0A9B0AC201B101A8013F
:108CF00097010E94B06E59016A0169897A89CB0196
:108D0000AA2797FDA095BA2FA81AB90ACA0ADB0AA2
:108D1000D401C30197FE03C00F96A11DB11D3C01F4
:108D20004D01F4E09594879477946794FA95D1F780
:108D3000D601C501D7FE03C00F96A11DB11D5C0170
:108D40006D01E4E0D594C794B794A794EA95D1F760
:108D50008091570290915802813491053CF48091A2
:108D600055029091560281349105A4F0C401B301DB
:108D700023E030E040E050E00E94B06E39014A014B
:108D8000C601B50123E030E040E050E00E94B06E43
:108D900059016A0180915906E82FFF27EE0FFF1F46
:108DA000E951FA4F808191810190F081E02DF7FF28
:108DB00003C0F095E195FF4F7A97A4F0C401B30189
:108DC00023E030E040E050E00E94B06E39014A01FB
:108DD000C601B50123E030E040E050E00E94B06EF3
:108DE00059016A0171E267167104810491042CF043
:108DF00070E2672E712C812C912C80EE68168FEF1B
:108E000078068FEF88068FEF980644F460EE662EA2
:108E10006FEF762E6FEF862E6FEF962E91E2A916EA
:108E2000B104C104D1042CF050E2A52EB12CC12C08
:108E3000D12CA0EEAA16AFEFBA06AFEFCA06AFEF7D
:108E4000DA0644F440EEA42E4FEFB42E4FEFC42EBA
:108E50004FEFD42E8091AF029091B002A091B10259
:108E6000B091B20286199709A809B9098093AF0297
:108E70009093B002A093B102B093B2028091A70286
:108E80009091A802A091A902B091AA028A199B0907
:108E9000AC09BD098093A7029093A802A093A902F0
:108EA000B093AA0280911102909112028F3F910516
:108EB00009F008F4DEC5BB85BB2309F068C58091C5
:108EC0006B02882309F063C580918F02882309F023
:108ED0005EC5E0919606EC87EE2309F458C58091B3
:108EE000E5069091E606A091E706B091E806B7FF87
:108EF00004C081509F4FAF4FBF4FE92EFA2E0B2F6A
:108F0000112707FD1A95E092E506F092E606009318
:108F1000E7061093E8068091ED069091EE06A09189
:108F2000EF06B091F006B7FF04C081509F4FAF4FDE
:108F3000BF4F892F9A2FAB2FBB27A7FDBA958D87DF
:108F40009E87AF87B88B8093ED069093EE06A09333
:108F5000EF06B093F00680917106A82EBB24CC24B6
:108F6000DD242091BF023091C0024091C102509196
:108F7000C202C601B5010E943C6E97FF04C0615059
:108F80007F4F8F4F9F4F672E782E892E992487FC15
:108F90009A946092BF027092C0028092C102909235
:108FA000C2022091BB023091BC024091BD0250919F
:108FB000BE02C601B5010E943C6E97FF04C061501D
:108FC0007F4F8F4F9F4F272E382E492E552447FC19
:108FD0005A942092BB023092BC024092BD02509241
:108FE000BE028091B7029091B802A091B902B091EF
:108FF000BA02B7FF04C081509F4FAF4FBF4F892FB8
:109000009A2FAB2FBB27A7FDBA958093B7029093F9
:10901000B802A093B902B093BA02D801C701861969
:109020009709A809B9098093170390931803A0938F
:109030001903B0931A0320919506E22EFF2400270E
:109040001127BC01CD01A80197010E94B06E590102
:109050006A012093260330932703409328035093FB
:1090600029038D859E85AF85B88982199309A40946
:10907000B50980931B0390931C03A0931D03B09329
:109080001E03BC01CD01A80197010E94B06E209380
:109090002A0330932B0340932C0350932D03D601C6
:1090A000C501D7FE04C081509F4FAF4FBF4F892FDE
:1090B0009A2FAB2FBB27A7FDBA9590936E02809392
:1090C0006D0257FF04C021503F4F4F4F5F4FBB27EA
:1090D00057FDBA95A52F942F832F909370028093FC
:1090E0006F02809157029091580281349105DCF40F
:1090F000809155029091560281349105A4F480919B
:109100005906E82FFF27EE0FFF1FE951FA4F808124
:1091100091810190F081E02DF7FF03C0F095E1957A
:10912000FF4F7A97E4F080918E078F3FC1F48091D2
:109130006D0290916E0297FD01969595879590939B
:109140006E0280936D0280916F029091700297FD84
:109150000196959587959093700280936F02809108
:10916000DA069091DB06A091DC06B091DD06B7FF30
:1091700004C081509F4FAF4FBF4F892F9A2FAB2F05
:10918000BB27A7FDBA958093DA069093DB06A093E0
:10919000DC06B093DD068091CC069091CD06A091BF
:1091A000CE06B091CF06B7FF04C081509F4FAF4F9E
:1091B000BF4F892F9A2FAB2FBB27A7FDBA9580935E
:1091C000CC069093CD06A093CE06B093CF068091A7
:1091D000CF029091D002A091D102B091D2022B8106
:1091E0003C814D815E81281B390B4A0B5B0B209320
:1091F0000F03309310034093110350931203809197
:10920000C7029091C802A091C902B091CA02EF8032
:10921000F88409851A85E81AF90A0A0B1B0BE092F3
:109220001303F09214030093150310931603209375
:109230001703309318034093190350931A03E092D5
:109240001B03F0921C0300931D0310931E038091D7
:10925000AB029091AC02A091AD02B091AE02821B24
:10926000930BA40BB50B8093AB029093AC02A0932D
:10927000AD02B093AE028091A3029091A402A0919E
:10928000A502B091A6028E199F09A00BB10B809385
:10929000A3029093A402A093A502B093A602FC851A
:1092A000FF2371F120918D0230918E02213831051A
:1092B00094F08091E3029091E40201969093E4028D
:1092C0008093E3028091F1069091F20601969093CB
:1092D000F2068093F10620583F4F94F48091E30208
:1092E0009091E40201979093E4028093E3028091CD
:1092F000F1069091F20601979093F2068093F106A1
:1093000010928E0210928D0281E090E090933303D0
:1093100080933203E0901703F09018030091190333
:1093200010911A03D801C70117FF07C08827992792
:10933000DC018E199F09A00BB10B81509240A04017
:10934000B04034F084E090E0909333038093320394
:109350008091380390913903A0913A03B0913B0377
:109360002091E5063091E6064091E7065091E80627
:10937000821B930BA40BB50B815E914BAF4FBF4F7C
:109380008F539C49A040B04028F080918F078931CD
:109390000CF4FFC041E0E41640E1F40640E00407AD
:1093A00040E014070CF473C080913403882309F45F
:1093B0006AC0D801C70117FF07C088279927DC01B9
:1093C0008E199F09A00BB10B9C01AD01B7FF04C022
:1093D00021503E4F4F4F5F4FF9E0559547953795D8
:1093E0002795FA95D1F78091320390913303820F3C
:1093F000931F9093330380933203D801C70117FF63
:1094000003C00796A11DB11DE3E0B595A7959795FB
:109410008795EA95D1F78093260390932703A0932D
:109420002803B093290389589341A040B04064F0C9
:1094300088E893E1A0E0B0E08093260390932703AF
:10944000A0932803B093290320912603309127038A
:10945000409128035091290357FF04C021503F4FEA
:109460004F4F5F4F232F342F452F552747FD5A95D8
:1094700080916D0290916E02820F931F90936E0205
:1094800080936D0206C081E08093340302C0109285
:10949000340360E0E61660EFF6066FEF06076FEF45
:1094A00016070CF073C080913503882309F46AC055
:1094B000D801C70117FF07C088279927DC018E193B
:1094C0009F09A00BB10B9C01AD01B7FF04C0215057
:1094D0003E4F4F4F5F4F69E055954795379527951C
:1094E0006A95D1F78091320390913303820F931FD5
:1094F0009093330380933203D801C70117FF03C051
:109500000796A11DB11D23E0B595A7959795879561
:109510002A95D1F78093260390932703A0932803DD
:10952000B093290388579C4EAF4FBF4F64F488E730
:109530009CEEAFEFBFEF8093260390932703A09399
:109540002803B093290320912603309127034091EB
:1095500028035091290357FF04C021503F4F4F4F1C
:109560005F4F232F342F452F552747FD5A95809164
:109570006D0290916E02820F931F90936E02809302
:109580006D0211C081E0809335030DC01092350348
:109590000AC0109233031092320388EE93E0909346
:1095A0009E0180939D018C85282F33278091320363
:1095B000909133032817390724F430933303209311
:1095C000320310918F07112379F0212F332727FDC4
:1095D000309580913203909133032817390724F492
:1095E00030933303209332034091170350911803B3
:1095F0006091190370911A03413851056105710595
:1096000074F08091E7029091E8022091320330914A
:109610003303820F931F9093E8028093E702405830
:109620005F4F6F4F7F4F74F48091E7029091E80293
:109630002091320330913303821B930B9093E80205
:109640008093E70281E090E09093330380933203AC
:10965000C0901B03D0901C03E0901D03F0901E03EC
:10966000D701C601F7FE07C088279927DC018C19AE
:109670009D09AE09BF0981509240A040B04034F02E
:1096800084E090E0909333038093320310922A0396
:1096900010922B0310922C0310922D0380913C0307
:1096A00090913D03A0913E03B0913F032091ED06C0
:1096B0003091EE064091EF065091F006821B930B1D
:1096C000A40BB50B815E914BAF4FBF4F8F539C499D
:1096D000A040B04018F019310CF4FFC001E0C016F2
:1096E00000E1D00600E0E00600E0F0060CF473C0F4
:1096F00080913603882309F46AC0D701C601F7FEBA
:1097000007C088279927DC018C199D09AE09BF097C
:109710009C01AD01B7FF04C021503E4F4F4F5F4F3A
:1097200009E055954795379527950A95D1F780918A
:10973000320390913303820F931F909333038093EE
:109740003203D701C601F7FE03C00796A11DB11D64
:1097500013E0B595A795979587951A95D1F78093BE
:109760002A0390932B03A0932C03B0932D038958C5
:109770009341A040B04064F088E893E1A0E0B0E0FD
:1097800080932A0390932B03A0932C03B0932D0373
:1097900020912A0330912B0340912C0350912D03EB
:1097A00057FF04C021503F4F4F4F5F4F232F342F9F
:1097B000452F552747FD5A9580916F029091700271
:1097C000820F931F9093700280936F0206C081E016
:1097D0008093360302C01092360320E0C21620EFB9
:1097E000D2062FEFE2062FEFF2060CF073C0809145
:1097F0003703882309F46AC0D701C601F7FE07C002
:1098000088279927DC018C199D09AE09BF099C01A5
:10981000AD01B7FF04C021503E4F4F4F5F4FE9E00D
:109820005595479537952795EA95D1F7809132035D
:1098300090913303820F931F9093330380933203ED
:10984000D701C601F7FE03C00796A11DB11D73E045
:10985000B595A795979587957A95D1F780932A0323
:1098600090932B03A0932C03B0932D0388579C4E09
:10987000AF4FBF4F64F488E79CEEAFEFBFEF80932C
:109880002A0390932B03A0932C03B0932D032091D4
:109890002A0330912B0340912C0350912D0357FF45
:1098A00004C021503F4F4F4F5F4F232F342F452F80
:1098B000552747FD5A9580916F0290917002820F53
:1098C000931F9093700280936F0211C081E0809388
:1098D00037030DC0109237030AC010923303109261
:1098E000320388EE93E090939E0180939D014C8516
:1098F000242F33278091320390913303281739079F
:1099000024F4309333032093320380918F0788230C
:1099100079F0282F332727FD3095809132039091DD
:1099200033032817390724F4309333032093320389
:1099300040911B0350911C0360911D0370911E0305
:10994000413851056105710574F08091E5029091EF
:10995000E6022091320330913303820F931F9093DC
:10996000E6028093E50240585F4F6F4F7F4FCCF483
:109970008091E5029091E602209132033091330309
:10998000821B930B9093E6028093E5020AC010922B
:10999000700210926F0210926E0210926D0210927D
:1099A0008F028091F406882341F410927002109285
:1099B0006F0210926E0210926D028091E5069091F6
:1099C000E606A091E706B091E806809338039093ED
:1099D0003903A0933A03B0933B038091ED06909135
:1099E000EE06A091EF06B091F00680933C039093B1
:1099F0003D03A0933E03B0933F031092BF02109229
:109A0000C0021092C1021092C2021092BB021092C8
:109A1000BC021092BD021092BE021092B7021092C8
:109A2000B8021092B9021092BA021092E506109292
:109A3000E6061092E7061092E8061092ED061092E4
:109A4000EE061092EF061092F0061092DA061092CF
:109A5000DB061092DC061092DD061092CC06109206
:109A6000CD061092CE061092CF06109212021092DE
:109A70001102E0907C02F0907D02C701F7FE04C065
:109A8000882799278E199F0940976CF088EE93E0FC
:109A900090939E0180939D018091620684FD03C096
:109AA00081E08093250310916E06A12EBB24CC2467
:109AB000DD24B701882777FD8095982F9701F7FE61
:109AC00004C0222733272E193F09442737FD40952C
:109AD000542F0E943C6E9B01AC01C601B5010E944F
:109AE0003C6E97FF04C061507E4F8F4F9F4F59E0EF
:109AF00095958795779567955A95D1F79B01812F15
:109B000099278E9DD0018F9DB00D9E9DB00D112483
:109B1000CD01B7FD03969595879595958795280F67
:109B2000391F442737FD4095542F20930B03309362
:109B30000C0340930D0350930E0380919F0290916C
:109B4000A002A091A102B091A202821B930BA40BD0
:109B5000B50B80939F029093A002A093A102B093B3
:109B6000A2028155934CA040B04064F080E593EC94
:109B7000A0E0B0E080939F029093A002A093A10286
:109B8000B093A20280919F029091A002A091A102A5
:109B9000B091A202805B9C43AF4FBF4F64F480EB57
:109BA0009CE3AFEFBFEF80939F029093A002A0933E
:109BB000A102B093A20240909502509096024114E7
:109BC000510409F488C18091620683FF84C18091A9
:109BD000CF029091D002A091D102B091D202B7FFF2
:109BE00004C081509E4FAF4FBF4F09E0B595A79578
:109BF000979587950A95D1F76C0197FF04C0D0948B
:109C0000C194D108D3948091C7029091C802A091C9
:109C1000C902B091CA02B7FF04C081509E4FAF4F36
:109C2000BF4F19E0B595A795979587951A95D1F7E8
:109C3000BC0197FF03C0709561957F4FC616D7068C
:109C40000CF46B01B601D7FE02C0695F7F4F3B0188
:109C5000B3E075946794BA95E1F70894611C711CA0
:109C6000ACE1EA2EA2E0FA2E4E0C5F1C7201002736
:109C7000F7FC0095102F24EE3DEF420E531E80910D
:109C80001D0790911E07A0911F07B091200780909B
:109C9000790190907A01A0907B01B0907C01BC0189
:109CA000CD01A50194010E94B06EE21AF30A040BE3
:109CB000150BC801B70128E631E040E050E00E94F2
:109CC000B06EDC01CB018C01045B10408091160763
:109CD0009091170797FF03C0909581959F4F81380A
:109CE000910514F000E010E0E0909D01F0909E01DD
:109CF000E114F10489F539E1C316D1046CF58091C2
:109D00008D0290918E02800F911F90938E0280930E
:109D10008D02809125038823F9F0C201AA2797FDBF
:109D2000A095BA2FBC01CD01A50194010E943C6E03
:109D3000DC01CB0180931D0790931E07A0931F07A2
:109D4000B0932007BC01CD010E94B06E3093940205
:109D50002093930210922503C801F3E0880F991F06
:109D6000FA95E1F7B3010E947B6ECB01AA2797FD1C
:109D7000A095BA2F20911D0730911E0740911F0713
:109D800050912007280F391F4A1F5B1F20931D0782
:109D900030931E0740931F075093200710918E01A8
:109DA000612F7727C69EC001C79E900DD69E900D4D
:109DB000112497FD4F966C01E5E0D594C794EA9580
:109DC000E1F76C197D096B0177FD7FC0E114F104A7
:109DD00009F073C0E0905702F0905802809155024C
:109DE00090915602E80EF91EF7FE04C067E070E09D
:109DF000E60EF71E63E0F594E7946A95E1F780E4D8
:109E000090E0E80EF91ECA01B901A50194010E9473
:109E1000B06EDA01C9012091930230919402442777
:109E200037FD4095542F821B930BA40BB50B845E1A
:109E30009D4FAF4FBF4FBC01CD0128E631E040E060
:109E400050E00E94B06EDC01CB01845B90408C9DA1
:109E5000D0018D9DB00D9C9DB00D1124CD01B70199
:109E60000E947B6E83E0189F60011124C616D706FE
:109E700014F4B60108C0882799278C199D09681722
:109E800079070CF4BC019B01442737FD4095542F02
:109E900080919F029091A002A091A102B091A20294
:109EA000820F931FA41FB51F80939F029093A0025F
:109EB000A093A102B093A2020EC00894E108F10899
:109EC000F0929E01E0929D0106C084EF91E0909394
:109ED0009E0180939D0180912403815080932403EF
:109EE0008F3F09F0DCC088E18093240380917106E4
:109EF0009927880F991F880F991F7C010027F7FC6D
:109F00000095102F8091CF029091D002A091D102A4
:109F1000B091D202BC01CD01A80197010E94B06EA0
:109F200030936705209366058091C7029091C8021F
:109F3000A091C902B091CA02BC01CD01A80197014C
:109F40000E94B06E309369052093680580911107D7
:109F50009091120797FD039695958795959587950E
:109F600090936B0580936A05809121079091220759
:109F700097FD0396959587959595879590936D0593
:109F800080936C05809116079091170790936F0549
:109F900080936E058091750290917602A091770270
:109FA000B0917802BC01CD0125E030E040E050E006
:109FB0000E94B06E30937105209370058091A905C1
:109FC0009091AA059093730580937205509277053E
:109FD0004092760580912501909126019093790514
:109FE0008093780580918302992790937B058093D5
:109FF0007A0580911D0790911E07A0911F07B091CF
:10A0000020072091790130917A0140917B01509194
:10A010007C01BC01CD010E94B06E30937D05209380
:10A020007C05809113029091140290938B0580938C
:10A030008A0580911304992790938D0580938C0550
:10A040008091FA019091FB0190938F0580938E058A
:10A050008091930790919407909393058093920534
:10A060008091970790919807909395058093940518
:10A070008091910799279093A1058093A0058091E5
:10A080006503909166039093A3058093A205809148
:10A090006303909164039093A5058093A405809138
:10A0A0008F02882381F01092070310920803109208
:10A0B000090310920A0310920303109204031092F2
:10A0C000050310920603F0906C02FF20F1F48091DA
:10A0D000F406282F3327442755278091CF029091EB
:10A0E000D002A091D102B091D202BC01CD010E9458
:10A0F0003C6EDC01CB01BC01CD0128EF3AE240E02F
:10A1000050E00E94B06E490102C088249924E0907A
:10A110006B02EE20F1F48091F406282F33274427B8
:10A1200055278091C7029091C802A091C902B091B1
:10A13000CA02BC01CD010E943C6EDC01CB01BC0116
:10A14000CD0128EF3AE240E050E00E94B06E3901C4
:10A1500002C0662477248091C6069091C706893C88
:10A1600091051CF088EC90E005C088539F4F34F4B3
:10A1700088E39FEF9093C7068093C6068091D1062F
:10A180009091D206893C91051CF088EC90E005C0C6
:10A1900088539F4F34F488E39FEF9093D2068093C7
:10A1A000D1068091D3069091D406AA2797FDA09559
:10A1B000BA2F20911B07A22EBB24CC24DD24BC0186
:10A1C000CD01A60195010E943C6E9B01AC018091DE
:10A1D000C6069091C706AA2797FDA095BA2F17E04B
:10A1E000880F991FAA1FBB1F1A95D1F7280F391F77
:10A1F0004A1F5B1F57FF04C0215C3F4F4F4F5F4F0B
:10A20000A6E05595479537952795AA95D1F78401EE
:10A21000020F131F1093D4060093D3068091C40637
:10A220009091C506AA2797FDA095BA2FBC01CD0134
:10A23000A60195010E943C6E9B01AC018091D10664
:10A240009091D206AA2797FDA095BA2FF7E0880F24
:10A25000991FAA1FBB1FFA95D1F7280F391F4A1F54
:10A260005B1F57FF04C0215C3F4F4F4F5F4FE6E03D
:10A270005595479537952795EA95D1F72301420ED5
:10A28000531E5092C5064092C406809116079091C5
:10A290001707880F991FAA2797FDA095BA2F20911D
:10A2A000CB06332744275527BC01CD010E943C6EC5
:10A2B0005B016C0197FF08C02FE330E040E050E005
:10A2C000A20EB31EC41ED51E76E0D594C794B794D3
:10A2D000A7947A95D1F78091E206282F3327442757
:10A2E00055278091B3029091B402A091B502B0912C
:10A2F000B602BC01CD010E943C6EDC01CB01BC0169
:10A30000CD0120EF35E540E050E00E94B06EB50190
:10A31000620F731F70931707609316070150104464
:10A3200034F080E090E49093D4068093D30680913B
:10A33000D3069091D4068050904C34F480E090EC99
:10A340009093D4068093D30651E0451650E4550609
:10A3500034F080E090E49093C5068093C406809129
:10A36000C4069091C5068050904C34F480E090EC87
:10A370009093C5068093C4066150704434F080E029
:10A3800090E4909317078093160780911607909199
:10A3900017078050904C34F480E090EC90931707AE
:10A3A0008093160780910001482F55278091250141
:10A3B000909126014817590794F420912501309176
:10A3C000260109811A81049FC001059F900D149FE9
:10A3D000900D1124B9010E94676E7A8369832981E7
:10A3E0003A81220F331F220F331F3A832983409172
:10A3F000620640FF7AC5EE2009F077C5FF2009F01C
:10A4000074C5809144039091450390939105809386
:10A410009005809113029091140290938B05809384
:10A420008A052091E9023091EA022115310509F0EF
:10A430003FC080911B0190911C018959934058F0B5
:10A4400087B5853F20F480911502815011C081E0CD
:10A4500080934D034EC080911B0190911C01843666
:10A46000910508F587B58B30D0F0809115028F5F8C
:10A47000809315029AE08902900111248091B3051E
:10A48000821B87BD8CE291E09093FF018093FE01D7
:10A490008EE591E09093EA028093E9022AC081E080
:10A4A00080934C0326C0F0924C03F0924D0321C0E0
:10A4B0008091750290917602A0917702B091780216
:10A4C00054E0880F991FAA1FBB1F5A95D1F780939C
:10A4D000160290931702A0931802B09319021092DB
:10A4E000140210921302215030403093EA0220935C
:10A4F000E9022091910141FF24C02233D8F48091D8
:10A50000BE0181508093BE018F3FD9F51092900219
:10A510008091750290917602A0917702B0917802B5
:10A520008093710290937202A0937302B0937402AD
:10A5300081E004C081E08093900288EC8093BE01AA
:10A5400020C080917D0190917E01820F911D20910C
:10A5500067063327829FA001839F500D929F500D65
:10A560001124CA01AA2797FDA095BA2F80937102E2
:10A5700090937202A0937302B093740281E080936F
:10A5800090028091CF029091D002A091D102B0911F
:10A59000D202E0907901F0907A0100917B01109154
:10A5A0007C01BC01CD01A80197010E94B06E590148
:10A5B0006A018091C7029091C802A091C902B0912E
:10A5C000CA02BC01CD01A80197010E94B06EB90179
:10A5D000C5010E941E6D7C01CC971CF04CE3E42E5B
:10A5E000F12CC7010E9402627C01809190028823B5
:10A5F00009F407C38091520299279C0120713070A1
:10A6000084FDFFC26091B50660FD04C080916206C2
:10A6100081FD07C0C980DA80309341032093400355
:10A6200056C18091520281FF2EC14091BA015091D2
:10A63000BB01CA010F9620917A0230917B028217EA
:10A64000930784F580914C03882361F580914E0334
:10A6500081FF13C08D7F80934E038091750290918E
:10A660007602A0917702B091780280937102909364
:10A670007202A0937302B093740280914E038160C2
:10A6800080934E03241B350B2F50304037FF03C0FF
:10A69000309521953F4F8091400390914103820F67
:10A6A000931F34C0CA010F9728173907A4F580916A
:10A6B0004D03882381F580914E0380FF13C08E7F68
:10A6C00080934E038091750290917602A09177025B
:10A6D000B09178028093710290937202A0937302FA
:10A6E000B093740280914E03826080934E03241BCA
:10A6F000350B215F3F4F37FF03C0309521953F4F0A
:10A700008091400390914103821B930B90934103EE
:10A710008093400327C020914E03822F9927837096
:10A720009070892BF9F02C7F20934E0310924103F7
:10A73000109240038091750290917602A091770269
:10A74000B09178028093710290937202A093730289
:10A75000B093740261FF06C084EF91E09093FF0113
:10A760008093FE012091400330914103C90137FFDE
:10A7700004C088279927821B930B815092400CF4C8
:10A780006BC0809167069927289FD001299FB00D43
:10A79000389FB00D1124CD0160E075E00E947B6E02
:10A7A0009B01442737FD4095542F80917102909171
:10A7B0007202A0917302B0917402820F931FA41FC2
:10A7C000B51F8093710290937202A0937302B093AD
:10A7D000740210924103109240038091B50681FFEC
:10A7E00006C08BE490E09093FF018093FE0180917E
:10A7F0006B06882389F5409144035091450357FF28
:10A8000002C04D5F5F4F559547955595479580918F
:10A81000250190912601209100013327489FF001E6
:10A82000499FF00D589FF00D1124CF01B9010E94EE
:10A830007B6E7093BB016093BA01663471051CF4A2
:10A8400086E490E005C06739710534F086E990E050
:10A850009093BB018093BA018091E9029091EA0242
:10A86000892B89F18091750290917602A0917702EF
:10A87000B09178028093710290937202A093730258
:10A88000B093740220C08091750290917602A091DD
:10A890007702B091780280599140A040B0408093F7
:10A8A000710290937202A0937302B093740280912C
:10A8B0006B06882311F0992702C088E790E09093F7
:10A8C000BB018093BA01C0904403D090450320910E
:10A8D0007502309176024091770250917802809112
:10A8E000710290917202A0917302B091740282176A
:10A8F0009307A407B50724F08091B50680FDC3C176
:10A90000009175021091760280917102909172020D
:10A91000081B190B809190019927089F9001099FAE
:10A92000300D189F300D1124C90137FD0F9624E01A
:10A93000959587952A95E1F7C81AD90A20911302AF
:10A940003091140237FF02C0295F3F4FB3E03595C5
:10A950002795BA95E1F72930310514F028E030E069
:10A96000229FA001239F500D329F500D11241216DB
:10A97000130674F4CA0157FD03969595879595952E
:10A9800087952091130230911402280F391F0DC0B2
:10A99000CA0157FD039695958795959587952091C2
:10A9A000130230911402281B390B809192019927D0
:10A9B000AA27BB27442737FD4095542FBC01CD0162
:10A9C0000E943C6E97FF04C061587F4F8F4F9F4F8E
:10A9D000E7E09595879577956795EA95D1F79B017F
:10A9E0004FEF623874071CF421E83FEF05C06F3F5A
:10A9F000710514F02FEF30E0C21AD30A20909702AD
:10AA0000309098024090990250909A0257FE08C0E8
:10AA10006FE770E080E090E0260E371E481E591E5A
:10AA200057E055944794379427945A95D1F78091DD
:10AA30008F01282F332744275527C201B1010E94D7
:10AA40003C6E97FF04C0615E7F4F8F4F9F4F45E084
:10AA500095958795779567954A95D1F79B017FEFF7
:10AA6000223837071CF421E83FEF05C02F3F31059E
:10AA700014F02FEF30E0C21AD30A0B561F4F0B52BF
:10AA80001140E0F48091400390914103892BB1F48F
:10AA90008091440390914503181619067CF4809127
:10AAA0004603909147038C159D053CF48091BC01B1
:10AAB0009091BD01C816D9060CF06C018091E90295
:10AAC0009091EA02892B21F0C0904403D090450375
:10AAD00080918D019927AA27BB27209192073327C0
:10AAE00027FD3095432F532FBC01CD010E943C6EB2
:10AAF00097FF04C061587F4F8F4F9F4F37E0959568
:10AB00008795779567953A95D1F79B019FEF223806
:10AB100039071CF421E83FEF05C02F3F310514F041
:10AB20002FEF30E0C21AD30AC601AA2797FDA095DD
:10AB3000BA2F2DE0880F991FAA1FBB1F2A95D1F7A6
:10AB40009701442737FD4095542FBC01CD010E9449
:10AB5000B06E209313033093140340931503509366
:10AB60001603C0901303D090140380914203909178
:10AB700043039C01220F331F280F391F2C0D3D1D4D
:10AB800037FF02C02D5F3F4FA90155954795559559
:10AB90004795509343034093420380916306282FC7
:10ABA0003327220F331F220F331F241735076CF46E
:10ABB00080911507282F3327220F331F220F331FB1
:10ABC000205530404217530724F03093430320931D
:10ABD00042038091B50680FF0DC0809142039091A1
:10ABE0004303A981BA81A817B90724F4B09343039A
:10ABF000A0934203E0914203F0914303FA83E98377
:10AC000042C080916B06882301F5609144037091E6
:10AC1000450377FF02C06D5F7F4F7595679575950A
:10AC20006795409125015091260180910001282FC0
:10AC30003327649FC001659F900D749F900D112470
:10AC4000B9010E947B6ECB0101C099279093BB0193
:10AC50008093BA018091BA019091BB01863491052D
:10AC60001CF486E490E005C08739910534F086E94C
:10AC700090E09093BB018093BA0109811A811093EF
:10AC80004303009342038091520281FF2EC18091C1
:10AC9000520284FD2AC18091480390914903A091FA
:10ACA0004A03B0914B030097A105B105B1F4298186
:10ACB0003A81C901AA2797FDA095BA2FECE0880F29
:10ACC000991FAA1FBB1FEA95D1F780934803909361
:10ACD0004903A0934A03B0934B03809113029091D0
:10ACE0001402809113029091140297FF03C0909573
:10ACF00081959F4F843691050CF0F7C049815A81A8
:10AD0000CA01AA2797FDA095BA2F9701442737FDBE
:10AD10004095542FBC01CD010E943C6EDC01CB015B
:10AD20008093130390931403A0931503B093160319
:10AD3000B7FF04C08150904EAF4FBF4F7C018D01D3
:10AD40007DE015950795F794E7947A95D1F7E09211
:10AD50001303F092140300931503109316038091CC
:10AD600053029091540257E0803D9507F8F480918A
:10AD7000480390914903A0914A03B0914B039C0171
:10AD8000AD0169E056954795379527956A95D1F7B6
:10AD9000821B930BA40BB50BA801970113E0220FA4
:10ADA000331F441F551F1A95D1F722C06FE0803A18
:10ADB000960758F58091480390914903A0914A0362
:10ADC000B0914B039C01AD01FAE05695479537953C
:10ADD0002795FA95D1F7821B930BA40BB50BA8010D
:10ADE0009701E2E0220F331F441F551FEA95D1F768
:10ADF000820F931FA41FB51F8093480390934903AC
:10AE0000A0934A03B0934B033CC020914803309178
:10AE1000490340914A0350914B0380549F41C0F431
:10AE2000DA01C9017BE0B695A795979587957A9544
:10AE3000D1F7281B390B4A0B5B0BD801C7018E0DCC
:10AE40009F1DA01FB11F280F391F4A1F5B1F11C074
:10AE5000DA01C9016CE0B695A795979587956A9533
:10AE6000D1F7281B390B4A0B5B0B2E0D3F1D401FE2
:10AE7000511F209348033093490340934A03509352
:10AE80004B038091480390914903A0914A03B091EC
:10AE90004B035CE0B695A795979587955A95D1F7A2
:10AEA000909345038093440340916906442399F0AD
:10AEB00055279C01BA010E947B6EC901861B970B26
:10AEC0009093470380934603260F371F3093BD01AD
:10AED0002093BC010AC010924703109246038FEFE3
:10AEE00093E09093BD018093BC013090D806232D50
:10AEF0003327C901880F991F880F991F8896A98148
:10AF0000BA818A179B0714F09A83898340901507AA
:10AF1000842D9927880F991F880F991F805590407D
:10AF2000E981FA818E179F0714F49A8389838091AF
:10AF300047028823A1F08091530290915402029716
:10AF4000C09768F4E980FA801E141F0444F481E07D
:10AF500090E090935402809353023A8329830981AD
:10AF60001A81109375050093740580910B039091DD
:10AF70000C03A0910D03B0910E0312E0880F991FEE
:10AF8000AA1FBB1F1A95D1F700911607109117073A
:10AF9000081B190B29813A81213A31058CF0C9012E
:10AFA00037FD019695958795801791070CF48C01D4
:10AFB000909581959F4F081719076CF48C010BC071
:10AFC0000135110514F000E510E03FEF003B1307D9
:10AFD00014F400EB1FEF242D3327220F331F220F11
:10AFE000331FC90149815A81841B950B8017910732
:10AFF0000CF48C0169817A81621B730B06171707A9
:10B000000CF48B018091D3069091D406609180025C
:10B0100070918102861B970B9093E4068093E30660
:10B02000D090F4062091030330910403409105036E
:10B0300050910603DD2041F0861A970AC401AA2721
:10B0400097FDA095BA2F04C0AA2797FDA095BA2F07
:10B05000280F391F4A1F5B1F2093030330930403FB
:10B0600040930503509306038091030390910403DA
:10B07000A0910503B091060381509A4FA040B040C3
:10B0800064F080E09AEFA0E0B0E080930303909337
:10B090000403A0930503B0930603809103039091EA
:10B0A0000403A0910503B091060380509640AF4F72
:10B0B000BF4F64F480E096E0AFEFBFEF80930303EF
:10B0C00090930403A0930503B0930603809093012B
:10B0D000909094019401442737FD4095542F80911E
:10B0E000030390910403A0910503B0910603BC01F2
:10B0F000CD010E94B06EE090E306F090E406E20E0F
:10B10000F31EB0907F016B2D772788279927980130
:10B1100017FF04C022273327201B310B37FF02C043
:10B120002F5F3F4F3595279549815A81240F351F51
:10B13000442737FD4095542F0E943C6E97FF04C072
:10B14000615C7F4F8F4F9F4F56E095958795779520
:10B1500067955A95D1F79B016E157F050CF47B011D
:10B16000309521953F4FE216F3060CF4790180915A
:10B17000C4069091C50660917E0270917F02861B85
:10B18000970B9093C3068093C206209107033091DA
:10B1900008034091090350910A03DD2041F0661A2B
:10B1A000770AC301AA2797FDA095BA2F04C0AA2742
:10B1B00097FDA095BA2F280F391F4A1F5B1F2093B8
:10B1C0000703309308034093090350930A038091C7
:10B1D000070390910803A0910903B0910A038150DD
:10B1E0009A4FA040B04064F080E09AEFA0E0B0E059
:10B1F0008093070390930803A0930903B0930A0375
:10B200008091070390910803A0910903B0910A036C
:10B2100080509640AF4FBF4F64F480E096E0AFEFB0
:10B22000BFEF8093070390930803A0930903B093A3
:10B230000A039401442737FD4095542F809107035A
:10B2400090910803A0910903B0910A03BC01CD01BC
:10B250000E94B06EC090C206D090C306C20ED31E2C
:10B260006B2D772788279927980117FF04C022277D
:10B270003327201B310B37FF02C02F5F3F4F35951F
:10B280002795A981BA812A0F3B1F442737FD409596
:10B29000542F0E943C6E97FF04C0615C7F4F8F4F1C
:10B2A0009F4F26E095958795779567952A95D1F7D5
:10B2B0009B016C157D050CF46B01309521953F4F7A
:10B2C000C216D3060CF4690186EB682E85E0782E51
:10B2D000B4E9AB2EB3E0BB2EABE05A2EF5EF8F2EC8
:10B2E000F6E09F2EF501258512160CF0ABC04981C2
:10B2F0005A81CA01AA2797FDA095BA2F332727FDA7
:10B300003095432F532FBC01CD010E943C6E97FF17
:10B3100004C0615C7F4F8F4F9F4FE6E09595879506
:10B3200077956795EA95D1F77C8B6B8BC701AA2738
:10B3300097FDA095BA2FF5012685332727FD309577
:10B34000432F532FBC01CD010E943C6E97FF04C0D8
:10B35000615C7F4F8F4F9F4F56E09595879577950E
:10B3600067955A95D1F72B893C89260F371F3C8B5F
:10B370002B8BC601AA2797FDA095BA2FF50127852B
:10B38000332727FD3095432F532FBC01CD010E9459
:10B390003C6E97FF04C0615C7F4F8F4F9F4F46E02C
:10B3A00095958795779567954A95D1F72B893C892F
:10B3B000260F371F3C8B2B8BC801AA2797FDA09522
:10B3C000BA2FF5012089332727FD3095432F532FBE
:10B3D000BC01CD010E943C6EDC01CB01B7FF03C074
:10B3E000CF96A11DB11D36E0B595A7959795879588
:10B3F0003A95D1F7F401608171812B893C89820FE4
:10B40000931F0E94DD2FD4018D939C9397FD03968B
:10B4100095958795959587959C8B8B8B832D9927F3
:10B42000EB89FC89E817F9073CF0842D99272B89D3
:10B430003C898217930714F49C8B8B8BEB89D30187
:10B44000EC9302C0D3011C925A94E2E0F0E08E0E1D
:10B450009F1E24E030E0A20EB31E620E731E57FE44
:10B4600041CFE2E1CC5E0C94E76E80915B0390915A
:10B470005C03A0915D03B0915E03809353039093AE
:10B480005403A0935503B0935603809157039091B2
:10B490005803A0915903B0915A0380934F0390939E
:10B4A0005003A0935103B093520308951092660382
:10B4B000109265031092640310926303089584B19F
:10B4C000806A84B93D9A82E58CBD1DBC459A81E0B5
:10B4D000809327078AEA8093370783E880933807A9
:10B4E0008AE08093390710923B0710923A07109236
:10B4F0003D0710923C07109291071092590708954A
:10B50000EF92FF920F931F93809171069927880FF6
:10B51000991F880F991F7C010027F7FC0095102FB9
:10B520008091CF029091D002A091D102B091D2022D
:10B53000BC01CD01A80197010E94B06E30933B077A
:10B5400020933A078091C7029091C802A091C90246
:10B55000B091CA02BC01CD01A80197010E94B06E52
:10B5600030933D0720933C0720911D0730911E0723
:10B5700040911F0750912007DA01C901E3E0880FCD
:10B58000991FAA1FBB1FEA95D1F7820F931FA41F13
:10B59000B51F820F931FA41FB51F20917901309111
:10B5A0007A0140917B0150917C01BC01CD010E9448
:10B5B000B06E3093430720934207E091D902F09197
:10B5C000DA028091EA069091EB06BF010E947B6E41
:10B5D000CB019B01220F331F220F331F280F391F6E
:10B5E000280F391F37FF02C02D5F3F4F3595279534
:10B5F0003595279530933F0720933E078091190793
:10B6000090911A07BF010E947B6E9B01220F331F8E
:10B61000220F331F260F371F260F371F37FF02C099
:10B620002D5F3F4F359527953595279530934107E9
:10B63000209340071092DA021092D9021092EB0682
:10B640001092EA0610921A07109219078091390792
:10B6500099278D30910509F463C08E3091055CF413
:10B660008B30910509F48BC08C3091050CF00CC126
:10B670000A9761F08BC18F30910509F45FC18F305B
:10B6800091050CF44BC1409781F180C18091660215
:10B6900080934A078091650280934B0780916402F2
:10B6A00080934C078091630280934D0780916202E2
:10B6B00080934E078091610280934F0780916002D2
:10B6C0008093500780915F028093510780915202CE
:10B6D0008093520780915202837F80935202A2E0AE
:10B6E000B0E00E94086F802D4FC180919307909128
:10B6F000940790934B0780934A0780919707909106
:10B70000980790934D0780934C0780912501909165
:10B71000260180934E078091000180934F0736C128
:10B720008091A20680934A078091A30680934B07DD
:10B730008091A40680934C078091A50680934D07C5
:10B740008091A60680934E078091AA0680934F07AA
:10B750008091AB06809350078091AC06809351078F
:10B760008091AF06809352078091AD068093530776
:10B770008091AE06809354078091B006CCC0F894B7
:10B7800080915806E82FFF27EE0FFF1FE951FA4F6F
:10B790000190F081E02DE038F1051CF0EFE7F0E0DA
:10B7A00006C02FEFE138F20714F4E1E8FFEFE09371
:10B7B0004A0780915906E82FFF27EE0FFF1FE95136
:10B7C000FA4F0190F081E02DE038F1051CF0EFE731
:10B7D000F0E006C06FEFE138F60714F4E1E8FFEFA0
:10B7E000E0934B0780915706E82FFF27EE0FFF1FCE
:10B7F000E951FA4F0190F081E02DE038F1051CF09D
:10B80000EFE7F0E006C08FEFE138F80714F4E1E865
:10B81000FFEFE0934C0780915606E82FFF27EE0FCD
:10B82000FF1FE951FA4F0190F081E02DE038F1055A
:10B830001CF0EFE7F0E006C02FEFE138F20714F458
:10B84000E1E8FFEF7894E0934D07809184028093C4
:10B850004E078091850280934F07809186028093E6
:10B8600050078091870280935107809188028093CE
:10B870005207809189028093530780918A028093B6
:10B88000540780918B0247C080911304863018F0D2
:10B890001092130485E080934A078091B10680934B
:10B8A0004B07809170059091710590934D0780939F
:10B8B0004C078091710290917202A0917302B09135
:10B8C0007402BC01CD0125E030E040E050E00E9470
:10B8D000B06E30934F0720934E078091A706809358
:10B8E00050078091A806809351078091A906809304
:10B8F0005207809183028093530780918202809344
:10B900005407809174059091750597FD0396959560
:10B910008795959587958093550738C010924A076B
:10B920008EE480934B0781E080934C078CE08093FA
:10B930004D078091020180934E0728C080918906AF
:10B9400080934A078091B40680934B0780918501CC
:10B9500080934C078091820680934D0780918306E7
:10B9600080934E078091840680934F0780918401D5
:10B9700080935007809186068093510780918706B7
:10B9800080935207809188068093530780915907CE
:10B99000882309F4B0C040915B0750915C07CA014D
:10B9A00081509E4F8F5F9340C8F420915D07309186
:10B9B0005E07C90181509E4F8F5F934078F480915C
:10B9C000620685FF0BC05093660340936503309376
:10B9D0006403209363038AEF809368038091610777
:10B9E0009091620721E08936920724F490939602A1
:10B9F00080939502809195029091960220919302F6
:10BA000030919402821B930B845E9D4F68E671E037
:10BA10000E947B6E845B904090939202809391028F
:10BA200020916507309166078091FE019091FF019A
:10BA30008217930740F480911304882321F43093F4
:10BA4000FF012093FE0180915A07992788369105BE
:10BA500001F18936910524F48736910529F053C008
:10BA60008936910559F14FC08091670780938E0701
:10BA700080916807809390078091690780938F0772
:10BA800080916A078093910780916B07809392075A
:10BA90003AC080916707809331078091680780934F
:10BAA0003207809169078093330780916A078093FA
:10BAB000340780916B078093350725C08091670715
:10BAC00080932807809168078093290780916907F0
:10BAD00080932A0780916B0790916C0790932C07B5
:10BAE00080932B0780916D0790916E0790932E079E
:10BAF00080932D0708C01092660310926503109280
:10BB00006403109263031F910F91FF90EF900895CB
:10BB100080912707882309F43BC0459887E397E085
:10BB20009093300780932F0790916703E92FFF27A9
:10BB3000E154FE4F9F5F90936703808180933907A4
:10BB4000993010F010926703109227070E94805AD4
:10BB500081E0809336070000000000000000000034
:10BB600000000000000000000000000000000000D5
:10BB700000000000000000000000000000000000C5
:10BB800000000000000080913707809356078EBDAB
:10BB9000089530912707332309F085C00DB407FEBF
:10BBA00082C084E08093FD01459A2EB5809169039F
:10BBB00099278130910589F0823091051CF4892BF9
:10BBC00021F03EC00297B9F03BC030935807209354
:10BBD0006A032138A9F581E008C0253549F4809130
:10BBE0006A03820F80936A0382E08093690328C00E
:10BBF0003093690325C080915807E82FFF27EC5840
:10BC0000F84F20838F5F8093580790916A038A31A1
:10BC1000A0F0291769F48AE1A4E7B7E0EAE5F7E0C4
:10BC20000D9001928A95E1F781E08093590702C057
:10BC3000309359071092690303C0920F90936A03DF
:10BC400020913607203208F028C0459800000000F7
:10BC500000000000000000000000000000000000E4
:10BC600000000000000000000000000000000000D4
:10BC7000000000000000000000000000E0912F071D
:10BC8000F0913007E20FF11D80818EBD8091560743
:10BC90009081890F8093560703C081E08093270726
:10BCA0002F5F20933607089587B18C6087B942983B
:10BCB000439810926C0380E88093C90110926B0343
:10BCC0008093C8010895809171038150809371031E
:10BCD0008F3F09F0F4C094E0909371038091520279
:10BCE000807BE1F08091A006882349F08091740365
:10BCF000882311F490936C0381E080937403809106
:10BD0000A1068823B9F080917503882319F484E093
:10BD100080936B0381E0809375030CC08093740360
:10BD20008093750380919C068093720380919E0698
:10BD30008093730380917403882309F040C080913D
:10BD4000B306282F332724FF07C080917902882368
:10BD500019F425FD4DC04EC090919D06983F50F0BE
:10BD60008091EC068D3D30F08091720388230CF4B5
:10BD70003FC040C0983F48F08091EC068A3028F4DC
:10BD8000809172038823B4F133C080916C03815099
:10BD900080936C038F3F79F58091EC0681508093FE
:10BDA0006C038091C901813011F480E801C086954F
:10BDB0008093C9018091C9019091720317C080914D
:10BDC0006C03815080936C038F3FA9F489E08093CA
:10BDD0006C038091C901813011F480E801C086951F
:10BDE0008093C9018091C9019091A006892311F027
:10BDF000429A01C0429880917503882309F043C09C
:10BE00008091B306282F332724FF07C08091790241
:10BE1000882319F426FD50C034C090919F06983FA6
:10BE200050F080911407873E30F08091730388238F
:10BE30000CF442C026C0983F48F0809114078A3025
:10BE400028F4809173038823E4F036C080916B035B
:10BE5000815080936B038F3F91F58091140781503F
:10BE600080936B038091C801813011F480E801C098
:10BE700086958093C8018091C801909173038923AE
:10BE8000D9F44398089580916B03815080936B039C
:10BE90008F3FA9F489E080936B038091C8018130C2
:10BEA00011F480E801C086958093C8018091C80193
:10BEB0009091A106892311F0439A0895439808951B
:10BEC0004FB724E130E0F8948091C9008F778093D8
:10BED000C9008091C9008F7B8093C9008091C900FF
:10BEE0008F7D8093C9005A9A52985B9A539A832FF8
:10BEF00099278093CD002093CC008091C800826068
:10BF00008093C80080E18093C9008091CA008F7738
:10BF10008093CA008091CA008F7B8093CA00809171
:10BF2000CA008F7D8093CA008091CA008F7E809363
:10BF3000CA008091CA00877F8093CA008091C9009F
:10BF40008B7F8093C9008091CA0084608093CA006F
:10BF50008091CA0082608093CA008091C80087FFE8
:10BF600003C08091CE00F9CF8091C9008068809392
:10BF7000C9004FBF0895FF920F931F93CF93DF9394
:10BF800080E197E20E94F016EC01FF248091C90045
:10BF90008F778093C9008091C9008F7E8093C900FC
:10BFA0005A9881ED99E09F938F9307E213E11F93D5
:10BFB0000F93E0919203F091930309950F900F90E6
:10BFC0000F900F9002C04A996CC0CE010E94F916E2
:10BFD0008823C9F3E0919203F0919303FF2009F4C1
:10BFE00068C087E09AE09F938F931F930F93099502
:10BFF000529A0F900F900F900F90CE010E94F91659
:10C000008823D9F383E690E05A9A019797FFFCCFF3
:10C010008FE891E05A98019797FFFCCF89E090E074
:10C020005A9A019797FFFCCF89E090E05A980197C0
:10C0300097FFFCCF8FE891E05A9A019797FFFCCFCA
:10C040008FE891E05A98019797FFFCCF89E090E044
:10C050005A9A019797FFFCCF89E090E05A98019790
:10C0600097FFFCCF8FE891E05A9A019797FFFCCF9A
:10C070008FE891E05A98019797FFFCCF89E090E014
:10C080005A9A019797FFFCCF89E090E05A98019760
:10C0900097FFFCCF8FE891E05A9A019797FFFCCF6A
:10C0A00013C08AE590E00E94F016EC0191E0F92EB1
:10C0B00091CF8DE09AE09F938F931F930F930995F3
:10C0C0000F900F900F900F9052985A980E94605FB7
:10C0D000E5E0CDB7DEB70C94F46EEF92FF920F93CC
:10C0E0001F93CF93DF93482F00E010E08091CA01A7
:10C0F000813061F41092CA0184E480937603109237
:10C10000780310927703109279032BC18091760304
:10C11000882319F421E030E001C098019091770361
:10C12000992371F4232B11F081E010C084E48093F3
:10C130007603909378039093770390937903FAC0F2
:10C14000913069F4232B09F0EBC082E080937703F0
:10C15000809178038F5F8093780383E0E9C0923009
:10C16000D1F4232B09F0DCC083E080937603409365
:10C17000790390917803923039F410927A0347FF53
:10C1800003C081E080937A0383E0809377039F5F0D
:10C1900090937803CFC0933009F0C2C0232B09F0ED
:10C1A000BFC09093760382E08093770380917803F9
:10C1B0008F5F8093780320917903822F9927782FBE
:10C1C0006627842F9927682B792B80917B068130F5
:10C1D00049F47370CB018050924063E070E00E949C
:10C1E0007B6E17C0823061F47770CB018050944031
:10C1F00066E070E00E947B6E2695269526950BC022
:10C20000737068567140CB0177FD0196BC0175953E
:10C21000679526952695022F11270F7010700F5FD6
:10C220001F4F0D30110508F074C07801E00EF11EAB
:10C23000F701E951FA4F808191819B01281B390B4D
:10C24000C90137FF03C0909581959F4F069794F4DD
:10C2500080918302883C30F480918302865F8093D2
:10C26000830208C088EC8093830280916F008F7DE9
:10C2700080936F00F701E951FA4F808191819C0111
:10C28000220F331F280F391F260F371F37FF02C019
:10C290002D5F3F4FE901D595C795D595C795CB0142
:10C2A00001968C179D0714F4219706C061507040C9
:10C2B000C617D7070CF4219680918302843BD0F0F7
:10C2C000F701E951FA4F80819181FE01E81BF90BDA
:10C2D000CF0163E070E00E947B6ECB01880F991F55
:10C2E000860F971F2BE136E0E20EF31EF7019183D4
:10C2F000808307C02BE136E0E20EF31EF7011182C6
:10C300001082000F111F09511A4FF801D183C08309
:10C3100011C00231110570F081E08093CA010AC09A
:10C3200081E08093CA011092780310927A0384E42A
:10C330008093760380917803803198F080917A031E
:10C34000882331F48091CA01882311F48093780105
:10C350001092780310927A031092770384E480930A
:10C360007603E6E0CDB7DEB70C94F36ECF93FC0115
:10C3700097FF05C0CFEFF095E195FF4F01C0C1E0F9
:10C3800028E631E0CF01B9010E947B6EFC018B35BC
:10C39000910554F08B5590408A35910538F484EB23
:10C3A00090E08E1B9F0BFC0141E00DC0CF01855B2F
:10C3B00090408A35910518F4E45BF04003C02E1BD1
:10C3C0003F0BF9014FEFEE0FFF1FE85EF54F259190
:10C3D00034918C2F992787FD9095289FB001299F34
:10C3E000700D389F700D1124842F992787FD90952B
:10C3F000689FA001699F500D789F500D1124CA01BC
:10C40000CF9108952AE530E0281B390BC9010E941D
:10C41000B6610895CF93DF9380E00E946E658091AE
:10C420002501909126016AE070E00E947B6E9F9347
:10C430008F9380912501909126016AE070E00E941F
:10C440007B6E7F936F9386EE9AE09F938F93C1E606
:10C45000D5E6DF93CF93E0919203F0919303099592
:10C460002DB73EB7285F3F4F2DBF809168038823CB
:10C4700039F187E00E946E658FED90E09F938F9376
:10C4800080912D0790912E079F938F9380912B077A
:10C4900090912C076AE070E00E94676E7F936F9323
:10C4A0008FEE9AE09F938F93DF93CF93E091920367
:10C4B000F091930309958DB79EB70A968DBF12C070
:10C4C00087E00E946E658CEF9AE09F938F93DF93D5
:10C4D000CF93E0919203F091930309950F900F9001
:10C4E0000F900F9080E10E946E658091D001909135
:10C4F000D1016CE370E00E94676E9F938F938091EF
:10C50000D0019091D1016CE370E00E94676E7F933F
:10C510006F9380919707909198079F938F9383E0F3
:10C520009BE09F938F93DF93CF93E0919203F091E1
:10C5300093030995809162062DB73EB7265F3F4F62
:10C540002DBF80FF24C08BE10E946E658091750233
:10C5500090917602A0917702B0917802BC01CD0152
:10C5600024E630E040E050E00E94B06E3F932F930D
:10C5700081E19BE09F938F93DF93CF93E0919203B0
:10C58000F091930309958DB79EB706968DBFDF9105
:10C59000CF910895CF93DF9380E00E946E6586E18E
:10C5A0009BE09F938F93C1E6D5E6DF93CF93E09115
:10C5B0009203F0919303099580E10E946E650F90BC
:10C5C0000F900F900F9080911D0790911E07A091E2
:10C5D0001F07B09120072091790130917A01409195
:10C5E0007B0150917C01BC01CD010E94B06E3F9354
:10C5F0002F938091C7029091C802A091C902B09177
:10C60000CA02B7FF04C081509C4FAF4FBF4F3AE002
:10C61000B595A795979587953A95D1F79F938F9361
:10C620008091CF029091D002A091D102B091D2021C
:10C63000B7FF04C081509C4FAF4FBF4F2AE0B59564
:10C64000A795979587952A95D1F79F938F9385E224
:10C650009BE09F938F93DF93CF93E0919203F091B0
:10C66000930309958DB79EB70A968DBFDF91CF9141
:10C6700008950F931F9380E00E946E652AE030E0DA
:10C680008091930790919407B9010E94676E9F93E0
:10C690008F938091930790919407B9010E94676EE0
:10C6A0007F936F938091250190912601B9010E949B
:10C6B0007B6E9F938F938091250190912601B90104
:10C6C0000E947B6E7F936F9381E39BE09F938F9398
:10C6D00001E615E61F930F93E0919203F091930307
:10C6E000099580E10E946E658DB79EB70C968DBF4F
:10C6F00080919707909198079F938F9380919507CA
:10C70000909196079F938F9384E49BE09F938F93E0
:10C710001F930F93E0919203F091930309958DB7C6
:10C720009EB708968DBF1F910F9108950F931F9389
:10C73000CF93DF9380916803C1E6D5E6882309F49F
:10C7400090C080E00E946E658091290799279F9391
:10C750008F9380E59BE09F938F938E01DF93CF9320
:10C76000E0919203F091930309958DB79EB70696D9
:10C770008DBF80912A0799278230910579F0833007
:10C7800091051CF4892B21F019C0039789F016C07C
:10C7900087E00E946E6589E59BE005C087E00E9406
:10C7A0006E658FE59BE09F938F93DF93CF930FC0D0
:10C7B00087E00E946E6585E69BE0F5CF87E00E94EA
:10C7C0006E658BE69BE09F938F931F930F93E09191
:10C7D0009203F091930309950F900F900F900F9093
:10C7E0008091280781FF14C089E00E946E6581E76F
:10C7F0009BE09F938F9381E695E69F938F93E091C3
:10C800009203F091930309950F900F900F900F9062
:10C8100080E10E946E658FED90E09F938F938091F1
:10C820002D0790912E079F938F9380912B079091C6
:10C830002C076AE070E00E94676E7F936F9387E732
:10C840009BE09F938F9381E695E69F938F93E09172
:10C850009203F091930309958DB79EB70A968DBF09
:10C8600012C082E00E946E6589E89BE09F938F93DF
:10C87000DF93CF93E0919203F091930309950F908A
:10C880000F900F900F90DF91CF911F910F9108950E
:10C89000CF93C82F20917B0320937C0399278F325D
:10C8A0009105E1F0803391051CF44F9779F027C092
:10C8B0008F349105D9F08F38910509F586E0289FCE
:10C8C000F0011124E253F54F849117C086E0289FB0
:10C8D000F0011124E153F54F84910FC086E0289FA9
:10C8E000F0011124E053F54F849107C086E0289FA2
:10C8F000F0011124EF52F54F849180937B039091C6
:10C900007B0380917C039813C0E00E947465909132
:10C910007B0386E0989FF0011124EE52F54F25919C
:10C9200034918C2FF9010995CF91089510929407B5
:10C9300010929307109298071092970710929607FB
:10C94000109295078AE090E00E94F01690937E0383
:10C9500080937D030895CF93DF9380917D03909121
:10C960007E030E94F916882309F4A8C080917D03F4
:10C9700090917E030A9690937E0380937D03E0E07E
:10C98000F0E09F0190E0A6EBB5E04BE0ED0189817E
:10C9900087FF07C09F5F8A81E80FF11D8C91280FE8
:10C9A000311D4150149647FFF1CF232B41F52091C3
:10C9B0008303309184034091850350918603BB2704
:10C9C000A52F942F832F9093820380938103AA270E
:10C9D000BB27281B390B4A0B5B0BCF01AA27BB27B0
:10C9E000280F391F4A1F5B1F209383033093840352
:10C9F0004093850350938603E5E0F0E013C0209157
:10CA00008103309182032E173F0718F4E21BF30BCA
:10CA100002C0E0E0F0E0892F9927880F991FE80F06
:10CA2000F91F3596F0939407E0939307EF3FF105D4
:10CA300078F480912501909126018E9F90018F9F1F
:10CA4000300D9E9F300D1124C90164E670E013C0C3
:10CA5000CF019695879596958795209125013091E0
:10CA60002601289FA001299F500D389F500D1124A9
:10CA7000CA0169E170E00E94676E70939607609347
:10CA8000950720917F03309180032E0F3F1F309335
:10CA9000800320937F035EE02131350778F0809199
:10CAA000970790919807019690939807809397071E
:10CAB00020513E403093800320937F03DF91CF913C
:10CAC000089590918803933240F4E92FFF27E756A9
:10CAD000F84F80839F5F909388030895833218F402
:10CAE0008D5F80938803089590E2ECE9F7E08FE191
:10CAF0009193815087FFFCCF0895CF93CFB723E068
:10CB000031E0F8948091C9008F778093C9008091BB
:10CB1000C9008F7B8093C9008091C9008F7D80936D
:10CB2000C9005A9A52985B9A539A832F99278093F7
:10CB3000CD002093CC008091C80082608093C80013
:10CB400088E18093C9008091CA008F778093CA00E2
:10CB50008091CA008F7B8093CA008091CA00806256
:10CB60008093CA008091CA0080618093CA0080913E
:10CB7000CA0088608093CA008091C9008460809355
:10CB8000C9008091CA0084608093CA008091CA0065
:10CB900082608093CA008091C80087FF03C08091A3
:10CBA000CE00F9CF8091C90080688093C900809140
:10CBB000C90080648093C9000E947465CFBFCF9183
:10CBC0000895282F99278F709070892B31F4209524
:10CBD00080918703822B8093870308958091CB01F6
:10CBE000882309F43FC08091520285FF0AC082E980
:10CBF0008093990783E280939A0785E580939B074A
:10CC000002C01092990780918703882321F48091B4
:10CC10009907882339F18091CC018F3021F48091DC
:10CC200087030E9448641092CB018091C80085FF61
:10CC3000FCCF8091C9008F7E8093C9008091C9008C
:10CC40008E7F8093C90080919907882311F48EEF1D
:10CC500001C08EE78093CE00809187038093CC0142
:10CC60001092870308951F920F920FB60F9211240E
:10CC70008F939F93EF93FF939091CB019923E1F5CD
:10CC800080918903882341F480919907882399F43E
:10CC900083E0809389030FC0833099F480919907D2
:10CCA000882349F0909399078091C9008E7F8093E3
:10CCB000C9008EEF1EC08091C90081608093C900B9
:10CCC0000EC0833261F48091C9008E7F8093C900C9
:10CCD0008FEF8093CE0081E08093CB0114C08091D0
:10CCE0008903E82FFF27E756F84F8F5F809389036A
:10CCF00080818093CE0007C0109289038091C90083
:10CD000080618093C900FF91EF919F918F910F9067
:10CD10000FBE0F901F9018959FB7F8948091C9008F
:10CD2000877F8093C9008091C9008F7E8093C9005E
:10CD30008091C9008F778093C9008091C9008F7B53
:10CD40008093C9008091C9008F7D8093C90052985B
:10CD50005A9A53985B9A9FBF0895CF93DF9380911F
:10CD60008A03882309F49FC090917B068091CF01AC
:10CD7000981709F498C08091CE01823071F48091A7
:10CD8000C800803241F48091CA00863021F481E0ED
:10CD90008093CE0102C01092CE0182E89CE09F9366
:10CDA0008F93C7E2D3E1DF93CF93E0919203F091A9
:10CDB000930309950F900F900F900F9080917B0631
:10CDC00099278230910501F1833091052CF4009769
:10CDD00061F0019769F024C084309105D9F0843066
:10CDE0009105ACF00597C9F01BC082E79CE002C03A
:10CDF00080E69CE09F938F93DF93CF93E091920323
:10CE0000F0919303099519C087E49CE0F3CF84E285
:10CE10009CE0F0CF86E19CE0EDCF8EE09CE0EACF95
:10CE20008FE89CE09F938F93DF93CF93E0919203E1
:10CE3000F0919303099510927B060F900F900F903D
:10CE40000F908091CE018823A9F00E948C6690916A
:10CE50007B06892F8150833018F40E94605F1FC0C9
:10CE6000943019F40E947D651AC09530C1F40E9477
:10CE7000526815C080917B06882389F085EA9CE082
:10CE80009F938F9387E293E19F938F93E091920317
:10CE9000F091930309950F900F900F900F90809150
:10CEA0007B068093CF01DF91CF9108950F931F935D
:10CEB00081E080938A034091CD01EEEBFBE020E01E
:10CEC00030E05FE4849199272F5F3F4F829FB0014C
:10CED000839F700D929F700D1124462751503196FB
:10CEE00057FFF0CF4093CD01E6E9FBE020E030E0D2
:10CEF00057E2849199272F5F3F4F829FB001839F14
:10CF0000700D929F700D112446275150319657FF96
:10CF1000F0CF4093CD01433459F088E190E029E20D
:10CF20000FB6F894A895809360000FBE2093600020
:10CF300080E59AE6909393038093920380EC9CE0C3
:10CF40009F938F9307E213E11F930F93E091920356
:10CF5000F091930309950F900F900F900F9082E638
:10CF600090E09F938F938EE490E09F938F931F9216
:10CF70001F92809102016AE00E945B6E892F9927BF
:10CF80009F938F93809102010E945B6E99279F93DC
:10CF90008F9386EE9CE09F938F931F930F93E09166
:10CFA0009203F091930309958EEB9BE09F938F93EF
:10CFB0001F930F93E0919203F0919303099586E9F3
:10CFC0009BE09F938F931F930F93E0919203F091B7
:10CFD000930309958DB79EB746968DBF8AE19DE074
:10CFE0009F938F931F930F93E0919203F09193037C
:10CFF000099582EC8093810080916F00806280931C
:10D000006F000F900F900F900F901F910F91089548
:10D0100080918A03882361F080917B06843011F42B
:10D020000E94EE658091CD01833411F010928A0345
:10D0300008951F920F920FB60F9211242F933F93D2
:10D040004F935F936F937F938F939F93AF93BF9310
:10D05000EF93FF932091CE0090917B06892F815012
:10D06000833020F4822F0E946D600BC0943021F435
:10D07000822F0E94E16505C0953019F4822F0E942D
:10D08000BE69FF91EF91BF91AF919F918F917F9179
:10D090006F915F914F913F912F910F900FBE0F9025
:10D0A0001F9018954FB720E430E0F8948091C900A4
:10D0B0008F778093C9008091C9008F7B8093C900CE
:10D0C0008091C9008F7D8093C9005A9A52985B9ACB
:10D0D000539A832F99278093CD002093CC00809181
:10D0E000C80082608093C80088E18093C900809165
:10D0F000CA008F778093CA008091CA008F7B80938B
:10D10000CA008091CA008F7D8093CA008091CA00B6
:10D110008F7E8093CA008091CA00877F8093CA0067
:10D120008091C9008B7F8093C9008091CA00846080
:10D130008093CA008091CA0082608093CA00809167
:10D14000C80087FF03C08091CE00F9CF8091C9004D
:10D1500080688093C9004FBF08950F931F93CF93AA
:10D16000DF93482F4F5F893108F089C08091E60531
:10D17000841710F44093E605CB0183539B4268E18A
:10D1800070E00E947B6EA42FBB27FD01EA0FFB1FFE
:10D19000E951FA4F808191819B01281B390BC9010C
:10D1A00037FF03C0909581959F4F069794F4809127
:10D1B0008302883C30F480918302865F80938302EF
:10D1C00008C088EC8093830280916F008F7D8093EC
:10D1D0006F00FD01EA0FFB1FE951FA4F8081918139
:10D1E0009C01220F331F280F391F260F371F37FFCF
:10D1F00002C02D5F3F4FE901D595C795D595C795DD
:10D20000CB0101968C179D0714F4219706C061503D
:10D210007040C617D7070CF4219680918302843B97
:10D22000D8F08D010A0F1B1FF801E951FA4F8081D8
:10D230009181FE01E81BF90BCF0163E070E00E94D1
:10D240007B6ECB01880F991F860F971F055E194FC4
:10D25000F8019183808307C0AA0FBB1FA55EB94F59
:10D2600011961C921E92E42FFF27EE0FFF1FE9512B
:10D27000FA4FD183C083443011F410927801DF91CA
:10D28000CF911F910F910895CF93DF932091BC0709
:10D29000822F9927807F9070409709F06CC02F31C2
:10D2A00009F046C08091BD0780938B032091BF0792
:10D2B00020938D038091C00780938C03822F992740
:10D2C0009093E8058093E705222309F054C08091EC
:10D2D0005606282F3327220F331FF901E55EF94F39
:10D2E0001182108280915706A82FBB27AA0FBB1F5F
:10D2F000FD01E55EF94F1182108280915906E82FF9
:10D30000FF27EE0FFF1FCF01855E994FEC011982B9
:10D31000188229513A4FE90119821882A951BA4F4E
:10D3200011961C921E92E951FA4F1182108223C06D
:10D33000C22FCF70CA30F8F48091BD078093C30725
:10D340008091BE078093C2078091BF078093C50775
:10D350008091C0078093C4076091C2077091C30792
:10D360008C2F0E94AD686091C4077091C5078C2F07
:10D370008F5F0E94AD68DF91CF910895CF93C82F42
:10D380008F3F49F480918E038F3F29F410929003D0
:10D3900010928F0332C020919003222339F4CF31B1
:10D3A00011F485E001C084E08093910380919103A2
:10D3B00090918F038217A0F4892F809580938F031B
:10D3C0008F3F19F48EEF80938F0380918F03C817DE
:10D3D00011F40E9444691092900310928F030BC0C5
:10D3E000E22FFF27E454F84FC0832F5F2093900370
:10D3F0009C0F90938F03C0938E03CF910895EF926B
:10D40000FF920F931F93CF93DF937C018B01EA016F
:10D41000452B39F0F80181918F01F701099521978A
:10D42000C9F7E6E0CDB7DEB70C94F36EEF92FF924A
:10D430000F931F93CF93DF937C018B01EA01452B60
:10D4400041F0F8010F5F1F4F8491F7010995219773
:10D45000C1F7E6E0CDB7DEB70C94F36E0F931F93E0
:10D46000CF938C01C62F161634F480E2F80109958B
:10D47000C1501C16D4F3CF911F910F9108950F93B3
:10D480001F93CF938C01C62F161634F480E3F80156
:10D490000995C1501C16D4F3CF911F910F91089597
:10D4A000A2E3B0E0E6E5FAE60C94CB6E29962EAC4A
:10D4B0003FAC29971DA61EA61FA618AAFBE46F2E37
:10D4C000712C6C0E7D1E2B96AEACBFAC2B97809151
:10D4D0008A03882329F485B7816085BF82E085BFF0
:10D4E000B50105C0053239F00894A11CB11CF50145
:10D4F00004910023B9F7A501461B570B19F0C10190
:10D500000E94166A002309F43FC20894A11CB11CB2
:10D51000552459AA5CA61FEF59A6F5010894A11C31
:10D52000B11C0491053721F0802F80628837F1F417
:10D5300050FE0EC0F30124E030E0620E731E8081C5
:10D540009181A281B3818DA79EA7AFA7B8AB0EC072
:10D55000F301A2E0B0E06A0E7B1E808191819C0104
:10D56000442755272DA73EA74FA758AB003221F4DB
:10D5700089A5882391F61DC0033211F438E083C0D9
:10D580000A3211F00D3299F40A3261F4F30142E0EB
:10D5900050E0640E751EE081ECA7EE230CF0BDCFC9
:10D5A000E195ECA750E1552A8FED5822B6CF0B320A
:10D5B00011F409A7B2CF0E32C1F5F5010894A11CF0
:10D5C000B11C04910A3279F4F301A2E0B0E06A0ED2
:10D5D0007B1E40815181BFEF4F3F5B0714F44FEF3B
:10D5E0005FEF142F9ACF40E050E0802F80538A30B5
:10D5F000A0F4CA01E3E0880F991FEA95E1F7840FD0
:10D60000951F480F591F400F511D40535040F501C1
:10D610000894A11CB11C0491E8CFEFEF4F3F5E07C7
:10D6200014F44FEF5FEF142F7DCF003329F454FC37
:10D6300074CFF0E25F2A71CF802F81538930D8F404
:10D6400040E050E0CA0173E0880F991F7A95E1F736
:10D65000840F951F480F591F400F511D40535040D4
:10D66000F5010894A11CB11C0491802F80538A30CD
:10D6700048F34CA757CF083619F424E0522A4DCF6F
:10D680000C3619F431E0532A48CF033661F44E01C9
:10D690000894811C911CF30142E050E0640E751E59
:10D6A000808189831CC1043421F0043611F00936CD
:10D6B000B1F5043411F451E0552A50FE0AC0F301CB
:10D6C00084E090E0680E791E20813181428153818F
:10D6D0000CC0F30142E050E0640E751E8081918120
:10D6E0009C01442737FD4095542F2DA73EA74FA7F7
:10D6F00058AB8DA59EA5AFA5B8A9B7FF0DC0B09535
:10D70000A095909581959F4FAF4FBF4F8DA79EA736
:10D71000AFA7B8AB8DE289A76AE0462E7BC00F3475
:10D7200011F00F3639F40F3411F491E0592A58E012
:10D73000452E6FC00037A1F4F301A2E0B0E06A0EFD
:10D740007B1E808191819C01442755272DA73EA7F0
:10D750004FA758AB40E1442E30E4532A08E759C0A4
:10D760000337C1F5F30142E050E0640E751E80807E
:10D7700091808114910489F44E010894811C911CBC
:10D7800088E289838EE6F401818385E78B838CE6CA
:10D790008C838D8389E28E831F8217FD13C0812FB6
:10D7A000992787FD9095AC0160E070E0C4010E946C
:10D7B000556D009729F0D82ED8181D150CF091C082
:10D7C000D12E8FC0F40101900020E9F73197DE2EB1
:10D7D000D81887C0053511F0053739F4053511F42F
:10D7E000F1E05F2A3AE0432E14C0083519F00837FB
:10D7F00009F06DC020E1422E53FE0BC02DA53EA5C1
:10D800004FA558A9211531054105510511F030E406
:10D81000532A19A619AB17FD02C04FED542299E205
:10D82000892E912C8C0E9D1E8DA59EA5AFA5B8A905
:10D830000097A105B10521F499A9992309F440C0E5
:10D84000C42CDD24EE24FF241AAA2DA53EA54FA545
:10D8500058A92C153D054E055F0510F031E03AAB97
:10D860006DA57EA58FA598A9A70196010E948E6E31
:10D87000DC01CB01182F8A3010F4105D04C0195A56
:10D88000083509F41F7DD4011E934D016DA57EA5B9
:10D890008FA598A9A70196010E948E6E2DA73EA77D
:10D8A0004FA758ABBAA9BB2379F6E8E04E1641F46E
:10D8B00053FE06C0103321F080E3D4018E934D0156
:10D8C000CE010196D82ED818B8E2DB0E0BC000238B
:10D8D00009F45AC04E010894811C911C098381E00F
:10D8E000D82E19A61D2DC9A8CD18C7FCCC2489A5F2
:10D8F000882311F01F5F02C056FC1E5F1C0DE52C33
:10D90000FF24C70180739070892B31F48CA5811B93
:10D91000682FC1010E942E6A89A5882331F041E059
:10D9200050E0BE01675D7F4F0AC0E6FE0BC080E39A
:10D930008AA70BA742E050E0BE01665D7F4FC101A0
:10D940000E94FF69C70180739070809731F48CA5A5
:10D95000811B682FC1010E943F6A6C2DC1010E948A
:10D960003F6A8D2D992787FD9095AC01B401C101C7
:10D970000E94FF69E4FEB4CDECA5E11BECA76E2F7D
:10D98000C1010E942E6AACCDE2E1CE5C0C94E76E40
:10D99000002422273327442751E0BB27EE27FF2707
:10D9A000A0E1660F771F881F991F001C221F331FDD
:10D9B000441F660F771F881F991F001C221F331FEB
:10D9C000441F2AF4050E2B1F3E1F4F1F04C0051ACB
:10D9D0002B0B3E0B4F0B550FBB1FEE1F587F556097
:10D9E00047FD5250AA95E9F6E695B7955795E69505
:10D9F000B7955795852F9B2F08952227332741E010
:10DA0000552768E0880F991F221F331F880F991F21
:10DA1000221F331F1AF4240F351F02C0241B350B9D
:10DA2000440F551F487F456037FD42506A9551F7B6
:10DA30005695479556954795842F0895AA2797FFA1
:10DA400004C0809590958A1F9A1F77FF04C0609547
:10DA500070956A1F7A1F669F9001779FA001679F4C
:10DA6000300D411D5A1F300D411D5A1F889FF00176
:10DA7000999F2E0F3F1F401D511D899F300D411D45
:10DA80005A1F300D411D5A1FCA01B901112480CF00
:10DA9000FB01DC0140FF05C002C005900D9205901E
:10DAA0000D9242505040C8F70895FC01415050403B
:10DAB00030F001900616D1F73197CF0108958827ED
:10DAC000992708955058192EA6D001D08CC0BA17A6
:10DAD0006207730784079507B1F188F40EF4109478
:10DAE0000B2EBA2FA02D062E622F202D072E732F5E
:10DAF000302D082E842F402D092E952F502DFF27D5
:10DB00005523B9F0591B49F0573E98F04695379583
:10DB10002795A795F0405395C9F776F0BA0F621F85
:10DB2000731F841F30F4879577956795B795F040FC
:10DB3000939517FA0F2E0895BF1BBB27BA0B620BE4
:10DB4000730B840BF6CFDEF692C097FB70D09F3735
:10DB500038F0FEE9F91B982F872F762F6B2F05C021
:10DB600083C09695879577956795F150D0F73EF4E9
:10DB700090958095709561957F4F8F4F9F4F089539
:10DB8000E89403C097FB0EF4F3DFB62F672F782FCE
:10DB9000892F9EE9002427C00ED05EF004C00BD070
:10DBA00026F001C008D019F020F48FEF089580E02E
:10DBB000089581E0089597FB092E052600F86894E2
:10DBC0002DD0E89407FC07C06217730784079507F8
:10DBD00021F008F400940794989408959A95BB0F47
:10DBE000661F771F881F11249923A1F08823B2F79D
:10DBF0009F3F59F0BB0F48F421F4002011F460FF5F
:10DC000004C06F5F7F4F8F4F9F4F881F97958795F9
:10DC100097F9089529C0052E092607FA440F551FC4
:10DC20005F3F79F0AA27A51708F051E04795880FC4
:10DC3000991F9F3F31F0BB27B91708F091E08795F6
:10DC400008959F919F91112414C097FB880F991FED
:10DC50009F3F31F0BB27B91708F091E087950895F1
:10DC60009F919F91112405C06627772788279927C0
:10DC700008959FEF80EC0895629FD001739FF0019B
:10DC8000829FE00DF11D649FE00DF11D929FF00D4C
:10DC9000839FF00D749FF00D659FF00D9927729F83
:10DCA000B00DE11DF91F639FB00DE11DF91FBD010E
:10DCB000CF0111240895991B79E004C0991F96178C
:10DCC00008F0961B881F7A95C9F780950895AA1BBE
:10DCD000BB1B51E107C0AA1FBB1FA617B70710F057
:10DCE000A61BB70B881F991F5A95A9F78095909589
:10DCF000BC01CD01089597FB092E07260AD077FDB8
:10DD000004D0E5DF06D000201AF4709561957F4FAE
:10DD10000895F6F7909581959F4F0895A1E21A2EE8
:10DD2000AA1BBB1BFD010DC0AA1FBB1FEE1FFF1FBF
:10DD3000A217B307E407F50720F0A21BB30BE40B0F
:10DD4000F50B661F771F881F991F1A9469F7609556
:10DD50007095809590959B01AC01BD01CF01089510
:10DD600097FB092E05260ED057FD04D0D7DF0AD029
:10DD7000001C38F450954095309521953F4F4F4FFA
:10DD80005F4F0895F6F790958095709561957F4F58
:10DD90008F4F9F4F08952F923F924F925F926F92B5
:10DDA0007F928F929F92AF92BF92CF92DF92EF922B
:10DDB000FF920F931F93CF93DF93CDB7DEB7CA1BAC
:10DDC000DB0B0FB6F894DEBF0FBECDBF09942A88D7
:10DDD000398848885F846E847D848C849B84AA847F
:10DDE000B984C884DF80EE80FD800C811B81AA810C
:10DDF000B981CE0FD11D0FB6F894DEBF0FBECDBFD7
:10DE0000ED010895EE0FFF1F0590F491E02D0994A8
:10DE1000F999FECFB2BDA1BDF89A119600B408954C
:10DE2000F7DF01921A94E1F70895F999FECFB2BD98
:10DE3000A1BD00BC11960FB6F894FA9AF99A0FBEDC
:0CDE400008950190F2DF1A94E1F70895B4
:10DE4C005E010A0151756164726F00000164FF018B
:10DE5C00FFFF01FC01FC0101737373FF03007D00E4
:10DE6C0000C409C40964001048616C6C6F205765CC
:10DE7C006C740000000000000000000000000000B6
:10DE8C000000000000000000000000000000000086
:10DE9C000000000000000000000000000000000076
:10DEAC000000000000000000000000000000000066
:10DEBC000000000000000000010B050000ECFF64F6
:10DECC0040415A4664640A02969696960840403A37
:10DEDC0010FB30380190D0030090D00300F40164A3
:10DEEC000053706F727400004E6F726D616C0000A5
:10DEFC00426567696E6E657200007800FF03640B03
:10DF0C000A0D0B0C0E0B0F10010101010F7002FF1B
:00000001FF
